:10B6E800414952434F54454300405053332E35305F
:10B6F8004048554E00414B4B5500532F4E21464173
:10B70800494C555245005245454E54455221532FF8
:10B718004E00434F4E5441435420414952434F54E5
:10B7280045430047505300403244400040334440B2
:10B73800004B492021554A20404D454E75000A16B8
:10B74800000180000300007E0000FE00001E0000D3
:10B75800360003E60001C4000000000FFFE053417B
:10B76800545320404B4552455300204750534056B0
:10B77800414C49442000404B455932004B45504507
:10B78800524E596F00534F5252454E440054455241
:10B798004B45502020005445524D494B202000561F
:10B7A8004152494F202020004241524F4752414DBB
:10B7B800005554564E414C2020004B6F5A454C4979
:10B7C80020200046504F4E544B2020004A454C45FF
:10B7D8004B20202000414C415020202000202020D8
:10B7E8002141544C212020202054415600205452FD
:10B7F80041434B21424520200020545241434B21D4
:10B808004B492020004D41524B004952414E592D81
:10B8180046454E540045535A414B2D46454E54001B
:10B82800214B494C45502020015554564F4E405607
:10B83800414C014D4147204245414C4C2001524565
:10B8480050754C45534B68690146504F4E544F4B09
:10B85800206869015554564F4E414C4B6869014C5C
:10B86800454754455220206869014245414C4C499E
:10B878005420686900472D464F52434520686900A7
:10B888004D4147204245414C4C20004241524F40D7
:10B898004D4147202000475053204D41472020006C
:10B8A800514E4820202020402148504100464C005D
:10B8B8005245504E41504C4F207552455320003E42
:10B8C800214B494C4550202000214B494C45500103
:10B8D800564A4154535A014B554C44202001544F69
:10B8E800524F4C2000214B494C45502020012055F7
:10B8F8005342204F4E4C592001544E4320312320AF
:10B9080035374B01544E4320312320392E3601015F
:10B91800505743403130234035374B01505743404F
:10B928003130234031394B01014D585040313023DB
:10B938004035374B014D58502034232035374B01C3
:10B948004D58502031232035374B014D5850403148
:10B9580030234031394B014D5850203123203139A3
:10B968004B0021564953535A412001465020554A0D
:10B978002020202020014650204D4153494B2020B3
:10B9880001465020546F524C2020200101434F4D56
:10B998003A0146505420464F4741442001465054EE
:10B9A800204B754C442020016F535A404650544058
:10B9B8004B754C01014650544F4B205441562001C1
:10B9C8004D494E40465040546F524C0049524E59D2
:10B9D80021544156004D454E542000414B54554189
:10B9E8004C5340504F5A2E005441524F4C20202067
:10B9F80020002053544F52452157505420002046D0
:10BA0800554C4C20002140546F524C455300535A1A
:10BA18004552004952444100555342200055534273
:10BA280020004C495354004B754C44002041545657
:10BA38004954454C492E48494241202000214B4950
:10BA48004C45502020015554564E4C4056414C010F
:0DBA5800554A204650202020202001555442
:10BA65005620535A45524B2001464F5244495420C3
:10BA750055545601465020546F524C45532001559C
:10BA8500545620546F524C45530143594C20524152
:10BA95004449555301434F4D3A0155545620464F9D
:10BAA5004741442001555456204B754C44202001F4
:10BAB500505245434845434B005554562156414C39
:10BAC50020200055404A40200020554A2040504F34
:10BAD5005A4021002140464F5244495420400046D7
:10BAE5004F524449540021404650544B40544F5204
:10BAF5004C005554564E40544F524C004E454D2027
:10BB0500755245532020002140555456404B754CE5
:10BB15004400202052414449555300214B494C458E
:10BB250050014C4547545240546F4C5421014C45EB
:10BB3500475452404E455A20014F53535A214C47C2
:10BB450021544F520101434F4D3A014C4547545240
:10BB550020464F4744014C45475452204B754C44B1
:10BB6500004C45475452204E455A20202020202085
:10BB7500004D4F5A4741542000464F5247415344C8
:10BB850020202000534B414C202020582F5920566F
:10BB95004953535A0054415620546F524C00415555
:10BBA500544F2E424520004155544F2E4B492000FD
:10BBB5002020534B414C4100544156204B4D200011
:10BBC500544156204E4D2000214B494C45502020D4
:10BBD50001564152494F20202068690158432D42A2
:10BBE50045414C4C6869015645522D4245414C68CA
:10BBF5006901414C544C414E4F536869014B4550C6
:10BC050045524E596F6869010101414C41502D4D16
:10BC15004F4420014759415249204245414C015466
:10BC250045535A545245502000214B494C4550200C
:10BC3500200153754C5948414E470153754C5921C4
:10BC45002D0153754C59404D4F440153754C594086
:10BC5500494E56015641522054434020204023016D
:10BC650048414E4745526F01564152494F204E5566
:10BC75004C4C0148414E474D4147200150455249E2
:10BC85004F445553015641522041564020304023E0
:10BC9500014E4554544F2D0148414E475445535A82
:10BCA50054200053754C5948414E4700532D484187
:10BCB5004E47214B49004E494E4353214455414C73
:10BCC50000564152494F204E554C4C005641524A60
:10BCD500203130205045524349472020004E554CD5
:10BCE5004C415A41532020202020202000214B493F
:10BCF5004C45502020015554564F4E414C20014192
:10BD050055544F43454E54010141544C2F5441560F
:10BD1500200153494B4C204B414C0153535A0101CF
:10BD2500535A454C21542D55500143454E542154E9
:10BD35002D55500157415950542142524700214B2E
:10BD4500494C455020200153544152544049446FB9
:10BD55002001454C536F200144454C54413A200184
:10BD6500546F42535A6F526F53200155544F4C53E1
:10BD75000143594C5349474020204023015554560F
:10BD85004056414C4C200101010143594C5201439D
:10BD9500594C21495246454C00214B494C455020B0
:10BDA50020010145475347014B41545440302C4035
:10BDB5002023014B4F4E5452535A54014E4D454189
:10BDC5002131383301494D50454C4C455201494DBF
:0DBDD500502D43414C01432D564152494F22
:10BDE2000154454320202040303040250141004E7F
:10BDF2004F20414750532F464C00414C54492D4748
:10BE02005053202000464C47542D4C4556454C007B
:10BE120041475053203C3E20464C00205741495454
:10BE2200004E4F20464C494748540040455849541B
:10BE3200204C4F47403F40004D4D2E595900206045
:10BE42006869003C2D20202020202D3E202020202B
:10BE520053454C003C2D20202020202D3E20202028
:10BE620045584954003C52454320205245433E2008
:10BE7200202053454C00522D4F464600202052456B
:10BE82004300414343454C455241542E00472D55F2
:10BE92004E49545300214B494C45502020015245F4
:10BEA200434D4F4445202058015245432E20313501
:10BEB2002F23015245432E2036302F230152504C5E
:10BEC20041592F53454E4401546F524C45534046FD
:10BED200505401434F4D3A00205C2020202053450E
:10BEE2004E44004046504E54204C4554455A494B0E
:10BEF200202020400046504F4E5420202000204B4E
:10BF0200494C455020202100464F47414420200003
:10BF1200535A414240003C2D204C495354202D3E5F
:10BF22002020455849540053454C004E4558540072
:10BF32004B6F56204650202000454C6F5A6F2046CA
:10BF42005000535A415240546F524C006F53535A4F
:10BF520040546F524C004B492020202020202020AA
:10BF62002000204B4920004750532048494241209D
:10BF72002000205441524F4C202020005554564E50
:10BF82004C004B4F5A454C49004C495354410045D3
:10BF92005445004D41474030007552455320555499
:10BFA2005620200054554C40534F4B202000214036
:10BFB2004C49534056414C20002046504056414C7B
:10BFC2004C2120002140464F474144202040002080
:10BFD20020404F4B4540202021004F4B4500564109
:10BFE2005200464958004741544521580053545283
:10BFF20054564E4C20202000535443594C200040AC
:10C002004B49200054502000406A40494E200040D5
:10C0120067404F55540020204849424120202100CA
:10C02200204B494C5000535A4552004947454E0057
:10C03200554A20202020414C4C2020535A45524B37
:10C04200004B4F56202020202056414C2020204BD0
:10C0520049005843542D464C4947485420005553F3
:10C06200454400454E54455220004D4D2E4D4D4DF8
:10C0720020004D4D2753532E530057475321383438
:10C08200002040554054404D402000554054404D02
:10C09200002055544320004C4F43414C0053574914
:10C0A2005353474400414C540053554940580041B2
:10C0B200564740203040230035303000313634308E
:10C0C20000205D203130404B632F70005D20202026
:10C0D2003140632F2300205D202035404B54530014
:10C0E2005D203230304046504D00406340204B636B
:10C0F200004654204B6300406340204E4D0046549E
:10C10200204E4D004D2F53003230305E003530301E
:10C112005E00312200322200332200352200382212
:10C1220000464C3700464C313600464C333300460D
:10C132004C3635004631303000463136300046321A
:10C142003630005E252640534F47005E2526405478
:0DC15200415300414C540056415200225E02
:10C15F002F24004B545300532F4E002224004B54D6
:10C16F0000225E004E4D00302C3500312C30003255
:10C17F002C3000302C3600312C3200322C3500336D
:10C18F002C3800372C35004031350040333000401B
:10C19F003630005441534B00464C2D44415445001A
:10C1AF00545000544F46005354410046494E004CE2
:10C1BF00414E00534554204F464653455400495372
:10C1CF004120484549474854004155544F2D474F4A
:10C1DF00200053544152540020434845434B4041A3
:10C1EF004C4C005241442044495354004053454C59
:10C1FF00404845494748543A0047505340424152FE
:10C20F004F40414C4C0053494E4B40312D3221632E
:03C21F002F2300CA
:106F3B00304D2475A7049005C2E0F51CE0F51DE06B
:106F4B00F51EE0F51FE0F56DE0F56EE0F56FE0F591
:106F5B0054127AFD12753B2275C70375C6E475B9D9
:106F6B0001E5BCB48143127AFD1261158E628F6309
:106F7B007568F9756900127011203C2D203B2B129E
:106F8B00714612711A856D1C856E1D856F1E855499
:106F9B001F12707D203C12203243201D231271469C
:106FAB0012753BE532242850DC2212707D203CF90F
:106FBB00203DF6203205201DBD80EF301DB880EA44
:106FCB0012714612753B856D1C856E1D856F1E8576
:106FDB00541F12713012753B203DCE80991273698C
:106FEB00201D0D75531074001272CC203DBB808692
:106FFB00E553540FC553C4540F2035051271E1806E
:10700B00031272CC808BC23CD23B1270CDFD12703E
:10701B00CDFC1270CDC39573F565EC9574F564EDED
:10702B009575600504600A800EE56424E0501180BC
:10703B0006E564242040091270CD1270CD0270CD8C
:10704B001270CDFD1270CDFC1270CDC39576F56725
:10705B00EC9577F566ED9578600904600122E5669D
:10706B00F48002E5668562F0A474E025F04002C26C
:0D707B003B22C23C1270CDA2E7923DA2E67E
:10708800921DA2E592324026A2E492E592E692E7AA
:10709800FC1270CD2565F565EC3564F5641270CD8C
:1070A800FC1270CD2567F567EC3566F56622A2E41B
:1070B8009235540F79C6F71270CD09F7301D0512B5
:1070C80070CDF55322E5697023E5686030240440EB
:1070D8002CE56875F004A485F0C7F5C675B901E517
:1070E800BCB4811985BD68756902801E540370108F
:1070F80005C675B901E5BC056953690F22D23C2262
:10710800147004E5BD80F0147004E5BE80E9E5BFA5
:1071180080E575A7009006F6E56DF0A3E56EF0A38F
:10712800E56FF0A3E554F02275A7009006F6E0F5A8
:107138006DA3E0F56EA3E0F56FA3E0F55422E564D6
:10714800B2E7F56D85656EAB67E566FC30E707C3AA
:10715800E49BFBE49CFCAA62A963125E0FE566301F
:10716800E707C3E49DFDE49EFEEEB2E7F56F8D549C
:107178002275380C1273D212741DD553012275383A
:107188000C1273A3127413D55301227538001273AD
:0E719800BB1273E2D55301227538001273A3A7
:1071A6001273E2D55301227538031273D212744E4C
:1071B600D55301227538031273A3127444D55301B3
:1071C6002275380F1273BB127473D55301227538AA
:1071D6000F1273A3127473D55326229071E623738C
:1071E6008091807780688059804A803B802C801D02
:1071F600800E80DA80CB80BC80AD809E808F8080C0
:107206007538151273D2127495D553012275381537
:107216001273A312748AD55301227538091273BBEF
:1072260012745BD55301227538091273A312745B6D
:10723600D55301227538061273D2127405D553013F
:10724600227538061273A31273FAD55301227538C4
:10725600121273BB12742BD5530122753812127396
:10726600A312742BD5530122027179753815127346
:10727600D2127495D553012275380F1273A3127466
:1072860073D553012275380F1273BB127473D5531D
:1072960001227538031273A3127444D55301227563
:1072A60038031273D212744ED55301227538001268
:1072B60073A31273E2D55301227538001273BB1201
:1072C60073E2D55326229072D12373809E80A980C3
:1072D600B480BF80CA80D580E08010801B80268065
:1072E60031803C80478052805D806875380C12730F
:1072F600A3127413D553012275380C1273D212746B
:0E7306001DD55301227538121273A312742B79
:10731400D55301227538121273BB12742BD5530145
:10732400227538061273A31273FAD55301227538E5
:10733400061273D2127405D55301227538091273DB
:10734400A312745BD55301227538091273BB1274EE
:107354005BD55301227538151273A312748AD55361
:10736400012202727178C686040886037AED125DE2
:10737400CD78CAA60408A60378C686040886037ACC
:1073840062125DCD78CCA60408A60378C6860408EC
:1073940086037AB5125DCD78C8A60408A6032275C3
:1073A4001A6A751B0A78CA86180886191275E6784F
:1073B400CC86060886072278C88618088619E4F55C
:1073C4001AF51B1275E678C886060886072278C661
:1073D4008618088619751A00751B010275E6E51DE5
:1073E4002519F51DE51C3518F51CC3E51F9FF51F70
:1073F400E51E9EF51E22C3E51F9FF51FE51E9EF5A3
:107404001EC3E51D9519F51DE51C9518F51C22E50F
:107414001D2FF51DE51C3EF51CC3E51F9519F51F31
:10742400E51E9518F51E22C3E51D9FF51DE51C9E5E
:09743400F51CC3E51F9519F51FB5
:10743D00E51E9518F51E22E51F2FF51FE51E3EF5DD
:10744D001EE51D2519F51DE51C3518F51C22C3E596
:10745D001D9519F51DE51C9518F51CE51F2FF51F3C
:10746D00E51E3EF51E22E51D2FF51DE51C3EF51C06
:10747D00E51F2519F51FE51E3518F51E22C3E51D5F
:10748D009FF51DE51C9EF51CE51F2519F51FE51E35
:10749D003518F51E22E51A7009E51B70058C068D51
:1074AD000722ED851BF0A4A2F792D5ED851AF0A465
:1074BD00AEF0FFEC851BF0A4A2D53FEE35F0FF92A8
:1074CD00D5EC851AF0A42FFFE435F030D50104FE7C
:1074DD0022E4F51AF51BEF4E7003051B22EF65191B
:1074ED007006EE65187001227808C3EF33FFEE3396
:1074FD00FEEF9519F5F0EE95184003FEAFF0E51A85
:10750D0033F51AD8E5F4F51A751BFF7805C3EF337B
:10751D00FFEE33FEEF9519F5F0EE95184003FEAF33
:03752D00F0E51B6B
:1075300033F51BD8E5F4C403F51B22E51D9511E5D1
:107540001C9510500BE56E9511E56D9510500122BC
:10755000E51F9511E51E9510500BE5549511E56F4B
:107560009510500122E51D9513E51C9512400BE581
:107570006E9513E56D9512400122E51F9513E51EEA
:107580009512400BE5549513E56F95124001225377
:107590002CF8C3E51F9554FFE51E956FFE926050D1
:1075A00007C3E49FFFE49EFEC3E56E951DF519E554
:1075B0006D951CF5189261500BC3E49519F519E40B
:1075C0009518F518C3E5199FE5189E9262500AE5D3
:1075D00018CEF518E519CFF5191274DEE52C54070D
:1075E00075F003A4F538E5389075EC730276040263
:1075F000761802762602763E02765102766402768C
:107600007202768A851C16851D17C3E4951FF51531
:10761000E4951EF51402769D851C16851D17851EA2
:1076200014851F158077C3E4951DF517E4951CF5A7
:1076300016C3E4951FF515E4951EF514805FC3E4A9
:05764000951DF517E4A3
:10764500951CF516851E14851F15804CC3E4951FE2
:10765500F517E4951EF516851C14851D15803985CD
:107665001E16851F17851C14851D15802BC3E495D3
:107675001FF517E4951EF516C3E4951DF515E4955C
:107685001CF5148013851E16851F17C3E4951DF57B
:1076950015E4951CF5148000C3E5179513E51695BB
:1076A5001210D70122E5159513E514951210D7018F
:1076B50022E519F92517FFE518F83516FED3EF95DC
:1076C50011EE9510500122E5119517FDE51095165F
:1076D500FC402A4D60271274A2E5152FF515E51417
:1076E5003EF514E5159513E514951210D70122E51D
:1076F500199DF9E5189CF8851016851117E51729C8
:10770500FFE51638FEE5139FE5129E500BC3E51302
:107715009517F9E5129516F8E51A700AE51B700636
:10772500AA00AB018013E9851AF0A4E5F0FBE88512
:107735001AF0A42BFBE435F0FAE5152BFBE5143A1A
:06774500FAE5119BE510BE
:10774B009A10D70122EB9515FDEA9514FCC3E515AC
:10775B009511E514951010D717E5139BE5129A5068
:10776B0036E5139515FFE5129514FE127A1A80274C
:10777B00EB9511FFEA9510FEAA00C001127A1AD000
:10778B0003E5172BFBE5163AFAEB99F517EA98F593
:10779B0016851115851014C2D5E5466002D2D5AAFF
:1077AB0056E98AF0A4ABF0E88AF0A42B30D5047527
:1077BB00F00384F8700122E5172513FDE516351249
:1077CB00FCED8AF0A4ABF0EC8AF0A42B30D5047559
:1077DB00F00384FEE5152513FDE5143512FCED8A47
:1077EB00F0A4ABF0EC8AF0A42B30D50475F0038435
:1077FB00F9E5389078027302781A02782602782F0E
:10780B0002783802783E02784A027851027856C3E1
:10781B00743E9EFFC3743E99FE8032C3743E9EFF3E
:10782B00AE018029AF06C3743E99FE8020AF06AE31
:0D783B0001801AC3743E9EFEC3743E99FF87
:10784800800EC3743E99FF8007C3743E9EFEAF014D
:1078580008EF2437FFE51B7007E51A700CE8800E67
:10786800A2E7E51A50030460F488F0A4E5F060018B
:1078780004F923FA98FBC3E998C333F990788AE5A9
:1078880038730278A20278CF02790402793102793A
:107898005E02798B0279B80279E505A7800BEB3097
:1078A800E7032A8002291E1FFBEEC45403F583EE6A
:1078B8005408C42FF582EE5407243883F5F0E045C8
:1078C800F0F0D8DA05A72205A7800BEB30E7032AEA
:1078D8008002290E1FFBEEC45403F583EE5408C43E
:1078E8002FF582EE5407240B83F5F0E045F0F0D82D
:1078F800DA05A722804020100804020105A7800BA2
:10790800EB30E7032A8002291E0FFBEEC45403F56F
:1079180083EE5408C42FF582EE540724EC83F5F067
:10792800E045F0F0D8DA05A72205A7800BEB30E791
:05793800032A80022972
:10793D000E0FFBEEC45403F583EE5408C42FF582ED
:10794D00EE540724BF83F5F0E045F0F0D8DA05A733
:10795D002205A7800BEB30E7032A8002291F1EFBAF
:10796D00EEC45403F583EE5408C42FF582EE54078C
:10797D00249283F5F0E045F0F0D8DA05A72205A7AB
:10798D00800BEB30E7032A8002291F0EFBEEC45457
:10799D0003F583EE5408C42FF582EE540724658356
:1079AD00F5F0E045F0F0D8DA05A72205A7800BEB3E
:1079BD0030E7032A8002290F1EFBEEC45403F58322
:1079CD00EE5408C42FF582EE5407243883F5F0E009
:1079DD0045F0F0D8DA05A72205A7800BEB30E703B9
:1079ED002A8002290F0EFBEEC45403F583EE5408D2
:1079FD00C42FF582EE5407240B83F5F0E045F0F02B
:107A0D00D8DA05A7228040201008040201EC701F6F
:087A1D00ED20E740D2E023CF89
:107A250023CF30E7F980357B08801A7B1080167BE1
:107A35002080127B40800E20E4ED20E3EE20E2EF73
:107A450020E1F07B80EE8BF0A4CF8BF0A4E5F02F46
:107A5500FFEC8BF0A4CD8BF0A4E5F02D2499838F5A
:107A6500F0A433E5F033FBE98BF0A4E5F0C88BF027
:107A7500A428F9E435F0F822FFFEFCFAF8F6F4F252
:107A8500F0EFEDEBEAE8E6E5E3E1E0DEDDDBDAD9B0
:107A9500D7D6D4D3D2D0CFCECCCBCAC9C7C6C5C40E
:107AA500C3C1C0BFBEBDBCBBBAB9B8B7B6B5B4B328
:107AB500B2B1B0AFAEADACABAAA9A8A8A7A6A5A414
:107AC500A3A3A2A1A09F9F9E9D9C9C9B9A999998D8
:107AD5009797969594949392929190908F8F8E8D7F
:107AE5008D8C8C8B8A8A898988878786868585840B
:107AF500848383828281818075A700907B23E546FC
:107B0500FA24FA50027A05EA2323F978107F0493C0
:107B1500F60809E9DFF9907B3BEA93F556227FC227
:107B2500803E7F4680BA7E8C81747D1882E87A30EB
:107B350085D074608BA0808040201008127B47029E
:107B45007D9DD215D274D273C219C23A1261158EB7
:107B550047757D0075460575520212AA001201DCB3
:107B6500E53524EB500E12AA007F1990BB9A1281BD
:107B75003712F19BE55275F016A4F570127D537519
:107B85007E15127C1E7F237E0990BB7612814912D9
:107B9500F19B10000810010D10021280E2127CC644
:107BA50075330180DA127D0B75330180D2757E0045
:107BB500127C1E7E0090BB8912817C7F237E0590FE
:107BC500BB7E128149127C6F12F19BE55210000FAA
:107BD50010010510028780D5045403F55280CE129A
:107BE5007C1E7F237E0B90BBB7128149E54660075B
:107BF50014600414124D2212F19BE5461000081082
:107C0500010B10021180D860D6154680D2B405024A
:107C150080CD054680C9027B6275320012F3127F62
:107C2500017E1190BB6612817C7E0012E9D1E57E52
:107C3500D26612EA2875170812EE5E124D6175714B
:107C450000C20612EB78741BFFF5177E0F90BBBDC3
:107C5500305D0390BBC512817C12AA4312674612A0
:107C650052C7C206126F63022829E55260141460D8
:107C75001E1460297F647E2D791C127CB91E1FD9C4
:107C8500F9227F6A7E1F7928127CB91FD9FA227FD3
:107C9500487E2D791C127CB90F1ED9F9227F567E9C
:107CA5003379281F12F22D0F0F12F22D1F12F22D0C
:107CB5001ED9F0221E12F22D0E0E12F22D1E02F208
:107CC5002DE552605514606814606D800075709ED6
:107CD500127D408003757000E5732540F573E4352A
:107CE50074F574E43575F57522757016127CDD80B2
:107CF5000375702DE5762542F576E5773541F577FF
:107D0500E43578F57822E55260CB1460DC1460E147
:107D15008000757044127CF9800375705AE573957F
:097D250040F573E5749400F57457
:107D2E00E5759400F57522757071127D22800375CC
:107D3E007088E5769542F576E5779541F577E578A5
:107D4E009400F57822E546907D6993F540FEAD47A7
:107D5E00E4FFFC125EA28E418F4222020C183060AC
:107D6E00C07F4012189812283F12F19B128018EB18
:107D7E00700590B8C0800B127E2690BFD150039034
:107D8E00C0187F3F7E0412814912F19B12F15012EE
:107D9E00F19175370990BB20122725907DAD7302A6
:107DAE00023D027F6D027B41028049027D9D027D74
:107DBE00C5027DDE027D6F7F2E1220CD80D17F36F3
:107DCE007E0490BFA612814912F19B12F15080BF22
:107DDE007F3712189812283F12F19B127FFC125413
:107DEE0057D2AC1000A9306DFA127ED6203BCF4090
:107DFE00ED7568F9751600127F2340FB1280BF7F68
:107E0E00367E29E51612E7AF12F19B05161281EEAA
:107E1E0078C6B6F7E2027FF67C0512545712EFF4DD
:107E2E00744112F005745312EFB5EB12EFE31282A8
:107E3E00005003DCE5227515F975160010000EE5ED
:107E4E00156025127E784005127E9F5002D3227F48
:107E5E003F7E29E51612E7AF12F19B7F1412F167F0
:107E6E000516E51664F870D4C3221287BD75B901E4
:107E7E00E5BCB4811AE5BDF51570037516F778C625
:0B7E8E00A6161289061288FE1288FE5C
:107E9900C30288FED3227F0575F019D5E0FDD5F020
:107EA900FA12545712EFF4744112F005744212EFAA
:107EB900B57E0F78C6E60812EFB5DEF912EFE612C5
:107EC9008200400122DF012275F00080CEC23B1200
:107ED9005457D2AC12F02D204C3CB440F712F0327A
:107EE900B4400312F032B4412DF53812F032B453D4
:107EF9002512F032FA12F032E538701A12F032B463
:107F09000D1412F032B40A0EC3E5169A4003028129
:107F1900E5C2ACD23B22C2ACD322128244125457DE
:107F2900D2AC1000F112F02D204CEBB440F412F059
:107F390032B4400312F032B441DCF53812F032B4F5
:107F490042D47E1078C612F032F608DEF9E53870B0
:107F5900C512F032B40DBF12F032B40AB9C2ACC3C3
:107F690022027D9D7F0A12189812283F12F19B1256
:107F79007FFC125473D2AC1000E712F032B440F512
:107F8900F53812F032B46EED12F032E538600A12AB
:107F99005473744F12EFC180DC125473744012F0A1
:107FA90005E51612EFC112EFD17568F975160012C1
:107FB9005473D2AC10003912F032B440F7F53812CC
:107FC900F032B44EC07E1078C612F032F608DEF9EF
:107FD900125473E5386007744F12EFC180D11280D3
:107FE900BF0516745112EFC178C6B6F7C212805C8C
:0C7FF900027D9D7515007516031287B4FB
:1080050075B901E5BC30E70205160515E51524200F
:1080150050EB227B007515F91287BD75B901E5BCDA
:10802500B481010B0515E515240450EC75150112F5
:1080350087B475B901E5BCB481010B0515E51524B7
:108045002050EC227F1C12189812289C40067515AA
:10805500F912805C027D9DE51560372404401A24E1
:108065001E5019E5152407400280271287BD12808E
:10807500980515E515240450F27515011287B47598
:10808500B901E5BC30E7031280980515E5152420F4
:1080950050EA221280AD1255F705C61255F705C6EE
:1080A5001255F705C60255F774FF80057404800163
:1080B500E4F5BCF5BDF5BEF5BF22E568606AF515CA
:1080C5000515E5152404501D7515011287B475B9FC
:1080D50001E5BC30E70280190515E515242050EBB4
:1080E500751500800C241C60F750E0E5152406503A
:1080F50037E56875F004A485F0C7F5C675BC81E55C
:1081050015F5BDF56878C6B6F70375BD000812818B
:108115002212811C12811C86BC0886BD0886BE08F9
:0981250086BF081255F705C622B9
:10D4070012CCE312D506128CC112D48B128CC9121E
:10D41700D49802CCE712CCE312D506128CC17F5AFE
:10D42700C23C128BA3128D9F783F79437F607EEABF
:10D4370012D4FA128CC97F65128BA3128D9F783D87
:10D4470079417F207E4E12D4FA303C2012D6BC128E
:10D45700D517783F794312D476783D794112D4763F
:10D4670012D6BC78D7E65480F675370002C3D4C30A
:10D47700E796FF1819E796FE0809C3E69FF71819FC
:10D48700E69EF7227F5B7E0690C0AB12817C1F80F1
:10D497000A7F667E14745912E8CA1F128A2C7E39D5
:10D4A700E402E8E97866E620E73418C3E6947208F0
:10D4B700E694045029C318E6941F08E69404401E16
:10D4C7007869E620E71818C3E6940E08E694015039
:10D4D7000DC318E6947508E694004002D322C322D0
:10D4E700E67D0030E7011D08E62BFB18E63CFCE46F
:0ED4F7003DFD22C3EB9FF6F71819EC9EF6F7E9
:10D505002212D4AB400CE47842F608F67840F608CF
:10D51500F6227864C3E6946AF55708E6944CF55606
:10D525000808C3E69458F55B08E694AEF55A7539D4
:10D5350000AC56AD57EC12D079784C12D107AC5AE5
:10D54500AD5BEC12D079785012D1077F2B7E867DAA
:10D55500777C1812D03E785012D0FB12CF4A12D0E9
:10D565003E785012D0FB12CF4A12D03E785012D0DE
:10D57500FB12CF4A12D03E7F367E847D257C641215
:10D58500D03E785012D0FB12CF4A12D03E784C12C2
:10D59500D0FB12CF4A12D03E7F3F7EA27D607C8BAE
:10D5A50012D03E785012D0FB12CF4A12CD3812CD90
:10D5B5003812D1137F3F7E807D057CE6053912CF79
:10D5C5004A784812D1077F2C7E937D477C7F12D005
:10D5D5003E785012D0FB12CF4A12D03E785012D06E
:10D5E500FB12CF4A12D03E784C12D0FB12CF4A1212
:10D5F500D03E7F357EB47DF87CDF12D03E78501268
:10D60500D0FB12CF4A12D03E785012D0FB12CF4A2F
:10D6150012D03E7F3F7EED7D227CCD12D03E784CF0
:10D6250012D0FB12CF4A12CD3C12CD38784412D11C
:10D63500077F317E397D9D7CE712D03E784C12D034
:10D64500FB12CF4A12D03E784C12D0FB12CF4A12B1
:04D65500D03E784407
:10D6590012D0FB12CD3C12D03E7F2C7E377D0C7C44
:10D66900A312D03E784C12D0FB12CF4A12D03E788A
:10D679004C12D0FB12CF4A12D03E784C12D0FB127A
:10D68900CF4A12CD3C12D1137F3F7E807D027C9F11
:10D69900053912CF4A784412D107784812D0FB12C3
:10D6A900D0B08E428F43784412D0FB12D0B08E4056
:10D6B9008F4122753900AC42AD43EC12D0797848DC
:10D6C90012D107AC40AD41EC12D079784412D107A0
:10D6D9007F2B7E537D507C0912D03E784812D0FBB7
:10D6E90012CF4A12D03E784812D0FB12CF4A12D03C
:10D6F9003E784412D0FB12CF4A12D03E7F347EF2DC
:10D709007DCD7CA312D03E784812D0FB12CF4A12AD
:10D71900D03E784812D0FB12CF4A12D03E7F3F7ECE
:10D729000A7D2E7CAE12D03E784412D0FB12CF4A2D
:10D7390012CD3812CD38784C12D1077F2B7E4F7D10
:10D74900AF7CB212D03E784812D0FB12CF4A12D029
:10D759003E784812D0FB12CF4A12D03E784812D0F8
:10D76900FB12CF4A12D03E7F357EB17D4B7C95129C
:10D77900D03E784812D0FB12CF4A12D03E784412DC
:10D78900D0FB12CF4A12D03E7F3F7E497DCD7C45EA
:10D7990012D03E784812D0FB12CF4A12CD3C12CD9E
:10D7A90038785012D107784C12D0FB12D0B08D5571
:10D7B9008E568F57785012D0FB12D0B08D598E5A91
:04D7C9008F5B786496
:10D7CD00E557246AF608E556344CF608E555340459
:10D7DD00F608E55B2458F608E55A34AEF608E4354C
:03D7ED0059F622C8
:10C2220012CCE312C8B312CCE77F6690C08D1281A4
:10C232007A12C2907F5A78C412C26C12C27478C643
:10C2420012C26C12C2577F6578C812C26C12C274D5
:10C2520078CA12C26C7E2DE51B12E8E97E33E51A1C
:10C2620012E8E97E39E51902E8E986040886030244
:10C272005D6C7E15E51C12E8E97E1BE51B12E8E900
:10C282007E21E51A12E8E97E27E51902E8E97F5ADC
:10C292007E01E53A12E7FD7E0B90CCA7E53B9302C7
:10C2A200E8FCE6FF08E6FE08E6FD339217E45001DB
:10C2B200F4FC12D12475130A75390112D32278D7EE
:10C2C200E6C2E775F00A84F9303D02A9F012D124E2
:10C2D2008913053912D2FB30170A053912D30E051C
:10C2E2003912D30EA80302D10712CCE312C8B3C28B
:10C2F2003C7F5A7E03128F5012C29012F19B1000A3
:10C302000810011510022080EFE53A146004153A76
:10C312008003753A3CD23C80DFE53AB43C05753A7D
:10C322000180F2053A80EE7E03128F4B7E0B128F54
:10C332005012C29012F19B10000810011510022039
:10C3420080EFE53BB40205753B158002153BD23CFC
:10C3520080DFE53BB41505753B0280F2053B80EEBC
:10C362007E0B128F4B7F5A78C412C26C12C27412A7
:07C37200C3DD128DAF78C49A
:10C3790012C43578C612C26C12C25712C40F751C8A
:10C3890000128DAF78C612C4357F6578C812C26CA9
:10C3990012C27412C3DD128DAF78C812C43578CABF
:10C3A90012C26C12C25712C40F751C00128DAF78DD
:10C3B900CA12C435303C14E53B24F4500B78C9E665
:10C3C9002410F618E63427F612C43B12CCE712897A
:10C3D9003102F19BC2247E15E51C128EA0F51CD2F8
:10C3E900247E1BE51B128EA0F51B1023E77E21E599
:10C3F9001A128EA0F51A1023E67E27E519128EA0CF
:10C40900F5191023E822C2247E2DE51B128EA0F512
:10C419001BD2247E33E51A128EA0F51A1023E77E6B
:10C4290039E519128EA0F5191023E622ECF608EB6E
:10C43900F62212CCBF78C8E6FE0886073395E0FDE0
:10C44900FC12D03E7FE87E037D007C0012D32212CD
:10C45900D03E78CAE6FE0886073395E0FDFC12D285
:10C46900FB12D03E7F807E697D677CFF12D2FBEC98
:10C4790012D07512D03E7F3F7E807D0D7C1D12CF7C
:10C489004A12D03E7F3D7E407D007C0012D03E782E
:10C49900BC12D0FB12CF4A12D03E7F3E7E807D0077
:10C4A9007C0012CD3C12D03E78BC12D0FB12CF4A90
:09C4B90012D03E7F3F7E807D0021
:10C4C2007C0012CD3812D03E78B412D0FB12CF4A83
:10C4D20012CFC2783C12D1077F407E807D007C0063
:10C4E20012D03E783C12D0FB12CF4A12D1A112D008
:10C4F2003E7F3F7EA87D007C0012D03E78B812D0ED
:10C50200FB12CF4A12CF4A12D03E7F407E007D00FE
:10C512007C0012D03E783C12D0FB12CF4A12D1A13D
:10C5220012D03E7F3F7EC07D007C0012CF4A12CDEA
:10C532003C12D03E78B812D0FB12CF4A12D03E78CD
:10C542003C12D0FB12CD3C785412D10712D18B7819
:10C552005812D10712D03E12CF4A12D03E78C012E2
:10C56200D0FB12CF4A784412D107785412D0FB1272
:10C57200D1A1783C12D10712D03E12CF4A12D03E3E
:10C5820078BC12D0FB12CF4A783C12D1077F3E7E94
:10C59200C07D007C0012D03E783C12D0FB12CF4A04
:10C5A20012D03E7F3F7E007D007C0012CD3C12D037
:10C5B2003E783C12D0FB12CF4A12D03E7F3F7E80A3
:10C5C2007D007C0012CD3C12D03E78B412D0FB121A
:10C5D200CF4A787012D10778C4E6FE0886073395F1
:10C5E200E0FDFC12D03E7FE87E037D007C0012D38A
:10C5F2002212D03E78C6E6FE0886073395E0FDFC9F
:10C6020012D2FB12D03E7FE07E5E7DF87CFF12D21A
:10C61200FBEC12D07512D03E7F3F7E7F7DE57CC958
:05C6220012D03E78700B
:10C6270012D0FB12CF4A12CFC2785012D1077F3FE8
:10C637007EF07D007C0012D03E783C12D0FB12CFFA
:10C647004A12D03E7F3F7EC07D007C0012CD3C1257
:10C65700D03E783C12D0FB12CF4A12D03E7F3F7EAD
:10C66700807D007C0012CD3C783C12D10778BC124B
:10C67700D0FB12D03E7F3F7E807D007C0012CD38FC
:10C6870012D03E783C12D0FB12D03E78B412D0FBC9
:10C6970012CF4A12CF4A784012D107785412D0FBF2
:10C6A70012D1D9783C12D10712D03E12CF4A7874F2
:10C6B70012D1077F417E107D007C0012D03E78C0EA
:10C6C70012D0FB12CF4A12D03E7F407E807D007C85
:10C6D7000012D03E784412D0FB12CF4A12D03E7FD0
:10C6E700417E207D007C0012CD3812D03E78441266
:10C6F700D0FB12CF4A12D03E7F407E407D007C00A7
:10C7070012D03E787412D0FB12CF4A12D03E7F402F
:10C717007EA07D007C0012CD3C12CD3C12CD38129C
:10C72700D03E785012D0FB12CF4A12D03E7850122A
:10C73700D0FB12CF4A12D03E7F3D7E2A7DAA7CAB2A
:10C7470012CF4A12D03E7F3F7E007D007C0012CD83
:10C757003812D03E783C12D0FB12D03E787012D0FF
:10C76700FB12CF4A12D03E784012D0FB12CFC21232
:10C77700D03E785012D0FB12CF4A12D03E785012DA
:10C78700D0FB12CF4A12CF4A12D03E785412D0FBB8
:0CC7970012CD3812D03E7F4A7E517DD278
:10C7A3007CCB12CF4A12D0B078AC12D1077F407E37
:10C7B300007D007C0012D03E787412D0FB12CF4A69
:10C7C30012D03E7F3F7E807D007C0012CD3C12D094
:10C7D3003E784412D0FB12CD3C12D03E785012D09A
:10C7E300FB12CF4A12D03E785012D0FB12CF4A121E
:10C7F300D03E785012D0FB12CF4A12D03E7F3E7EFD
:10C803002A7DAA7CAB12CF4A12D03E785012D0FBBD
:10C8130012CD3812D03E785812D0FB12CFC212D0AC
:10C823003E7F4A7E517DD27CCB12CF4A12D0B012CA
:10C83300D03EAF3AEF3395E0FEFDFC12D03E7F4091
:10C843007E7E7D057C0012D32212D03E7F607E75F2
:10C853007D587CFF12D2FB12D2FB78B012D107783D
:10C86300AC751B6412C88A8F1C78B0751B6712C81D
:10C873008AE51C75F00AA42FFF249C50027F0078E0
:10C88300D7E654802FF62275390012D0FB12D03E22
:10C893007F0A7E007D007C0012D3CEA81BE513F631
:10C8A30008E512F608E511F6335004EFF404FF220D
:10C8B300C23D78647BAC12C2A4D23D78677BB012D0
:10C8C300C2A412CCBF7F007EE47D577C0012D03E11
:10C8D30078AC12D0FB12D2FB12D03E7F007E537D88
:0EC8E300077C0012D3CE12D05D85133B7F8000
:10C8F1007ECB7DA47C0012D03E78B012D0FB12D248
:10C90100FB12D03E7F407E7E7D057C0012D3CE128D
:10C91100D05DE513F56F04F53A85126E85116D85CD
:10C92100106C7F407E7E7D057C0012D03E786C12BB
:10C93100D0FB12D32212D03E7F607E0C7DA27C0000
:10C9410012D03E78B012D0FB12D2FB12D30E786C0B
:10C9510012D10778AC12D0FBEC12D07512D03E7F09
:10C96100347E9C7D2B7C5F12CF4A785412D1071202
:10C97100D18B785012D107786C12D0FBEC12D075A4
:10C9810012D03E7F347E9C7D2B7C5F12CF4A12D029
:10C991003E785012D0FB12CF4A784012D1077F4027
:10C9A1007E007D007C0012D03E785412D0FB12CF65
:10C9B1004A12D1A112D03E7F3D7EC07D007C001283
:10C9C100D03E78BC12D0FB12CF4A12D03E7F3E7EC1
:10C9D100C07D007C0012CD3C12D03E78BC12D0FB51
:10C9E10012CF4A12CF4A12D03E7F3D7E407D007C5D
:10C9F1000012D03E78BC12D0FB12CF4A12D03E7F3B
:10CA01003E7E807D007C0012CD3C12D03E78BC126F
:10CA1100D0FB12CF4A12D03E7F3F7E807D007C004A
:10CA210012CD3812D03E785412D0FB12CF4A12CD1B
:10CA31003812D03E7F407E807D007C0012D03E784F
:10CA41005412D0FB12CF4A12D1A112D03E7F3D7EAB
:10CA5100707D007C0012D03E78BC12D0FB12CF4A10
:10CA610012D03E78BC12D0FB12CF4A12CF4A12CD5F
:10CA71003C12D03E78B412D0FB12CF4A785812D172
:10CA810007785412D0FB12D1A1783C12D107785407
:10CA910012D0FB12D1D9785412D107783C12D0FBB5
:10CAA10012D03E12CF4A12D03E78BC12D0FB12CF28
:10CAB1004A783C12D1077F3E7EC07D007C0012D0B7
:10CAC1003E783C12D0FB12CF4A12D03E7F3F7E000F
:10CAD1007D007C0012CD3C12D03E783C12D0FB127E
:10CAE100CF4A12D03E7F3F7E807D007C0012CD3C3C
:10CAF10012D03E78B412D0FB12CF4A787012D1070F
:10CB0100785012D0FB12D03E12CF4A12D03E78C0DC
:10CB110012D0FB12CF4A784412D107785412D0FBBD
:10CB210012D03E12CF4A787412D107784012D0FB4E
:10CB310012D03E12CF4A783C12D1077F407E807DD1
:10CB4100007C0012D03E784412D0FB12CF4A12D0A2
:10CB51003E7F417E107D007C0012CD3C12D03E789C
:10CB61004412D0FB12CF4A12D03E787412D0FB127D
:10CB7100D03E7F407EA07D007C0012CD3812CD3C9E
:10CB810012D03E783C12D0FB12CF4A12D03E7F3DEC
:10CB91007E2A7DAA7CAB12CF4A12D03E7F3F7E0017
:10CBA1007D007C0012CD3C12D03E785412D0FB1295
:10CBB100D03E787012D0FB12CF4A12D03E783C1290
:10CBC100D0FB12CF4A12CF4A12D03E785812D0FB76
:10CBD10012CD3C12D03E7F3F7E7F7DE57CC912CFD6
:01CBE1004A09
:10CBE20012D03E7F4B7E187D967C8012CD3C12D0B7
:10CBF200B012D03E7FE87E037D007C0012D3CE12BD
:10CC0200D05D78C8A61208A61308A60608A607785B
:10CC12007412D0FB12D03E7F3F7E807D007C0012DA
:10CC2200CD3812D03E784412D0FB12CD3C12D03E09
:10CC32007F3E7E2A7DAA7CAB12CF4A12D03E78403C
:10CC420012D0FB12CF4A12D03E783C12D0FB12CF48
:10CC52004A12D03E784012D0FB12CD3C12D03E7F19
:10CC62003F7E7F7DE57CC912D03E787012D0FB12E8
:10CC7200CF4A12CF4A12D03E7F487EF47D247C00F8
:10CC820012CD3C12D0B012D03E7FE87E037D007CF4
:10CC92000012D3CE12D05D78C4A61208A61308A63D
:10CCA2000608A607223F3F4344454647484A4B4CA5
:10CCB2004D4E5051525354555657583F3FE4F53953
:10CCC200F5A790CCD3791078B4E493F6A308D9F9F8
:10CCD2002232A5C24A4A19DC3A885CDB3BFFD6DC29
:01CCE2003B16
:10CCE300D2D58002C2D575A70490040078107F0BBB
:10CCF30012CD0F78267F0512CD0F783C7F2212CDFF
:10CD03000F786A7F0F12CD0F75A7002230D506E684
:10CD1300F008DFFB22E0F608DFFB22DA0CD9028001
:10CD23000BD906303701B3500502CEAB923702CE92
:10CD330097D9F680F9D2368002C23612CEDC30366D
:10CD430006C86002B237C89236DAD0D9E4B8000A0E
:10CD530012CF23A236923702CE8060FBB513004078
:10CD63000F12CF23A23692F7A2379236A2F7923749
:10CD7300C398F40424E740DF2419AD29AC28AB277A
:10CD83007A00C394084008CDCCCBCAE4CD80F42408
:10CD9300086010F9C3ED13FDEC13FCEB13FBEA136E
:10CDA300FAD9F1A236303701B340308A17E5102B98
:10CDB300F518E5113CF519E5123DF51A501A13F56E
:10CDC3001AE51913F519E51813F518E51713F517EF
:10CDD3000513E5137002051402CE36E4C39AF51762
:0CCDE300E5109BF518E5119CF519E51210
:10CDEF009DF51A500DB237C378177F04E496F608F5
:10CDFF00DFFA7A047019E513C39408F5135002157E
:10CE0F0014E4C517C518C519F51ADAE802CED720EC
:10CE1F00E7BAE5137002151415137817C37F04E6EC
:10CE2F0033F608DFFA80E8E51A20E7137817C37F97
:10CE3F0004E633F608DFFAE513700215141513E54F
:10CE4F00173378187F03E63400F6500E08DFF775B6
:10CE5F001A800513E51370020514E51420E75470CA
:10CE6F0027E513604E046020851A12851911851865
:10CE7F00105326F0AC10AD11A237E51313FFE512D6
:10CE8F0092E7FEA81302D05DE4F512F511F510F547
:10CE9F00147513FF5326F043260580D8E5FFF512CE
:10CEAF00F511F510751400F513D2375326F04326FC
:10CEBF000980C15326F0432603E4F512F511F5104E
:10CECF00F514F513C23780AC5326F080EC79017A54
:10CEDF00018512F0E513A2F7339237751400F5139D
:10CEEF006002D2F785F012A813B8FF0809E512C245
:10CEFF00E76001098C278D288EF0A2F7EF330470BD
:01CF0F000A17
:10CF10000AC2F705F00AD5F0011A146002D2F785AB
:10CF2000F02922C88813C512C529C512C511C52804
:10CF3000C511C510C527C51022DA03B8000302CEFB
:10CF4000ABD9028002D9F702CE9712CEDC3037017E
:10CF5000B392377004D9E78005DADEB8000302CE59
:10CF6000D7D9E2C3947E500215142513F51350024D
:10CF700005147815760008B81BFA78277915E608A5
:10CF8000FAE8FC78108AF0E608A427F709E5F037FC
:10CF9000F7500989F00907E760FBA9F0B813E61913
:10CFA00019ECF8B82AD802CE3602CEC2B8FFFA027F
:10CFB000CEABD9FB02CE97DAF6B800F002CED7128C
:10CFC000D11312CEDC303701B392377007D9E3B8F2
:10CFD00000E280DBDAE1B8000280E1D9D5C8C3986D
:10CFE00050021514247F50020514F513781A7600A8
:10CFF0007A1A7B80C3E5109527E5119528E51295EF
:10D00000294016C3E5109527F510E5119528F5116F
:10D01000E5129529F512E64BF6DA0302CE36EB035C
:0AD02000FB30E703187600C3E510AB
:10D02A0033F510E51133F511E51233F51240CA3024
:10D03A00E7DD80B6E53905396010D0F0D0E0C010E0
:10D04A00C011C012C013C0E0C0F08F138E128D1130
:10D05A008C1022E539146010D0F0D0E0D013D01231
:10D06A00D011D010C0E0C0F01539227920800C7997
:10D07A0010800479087D007E007F003392D550032A
:10D08A0012D0EDEC33400FEF33FFEE33FEED33FDFC
:10D09A00EC33FCD9EE22EECCF5F0747E29A2D5133E
:10D0AA00FF92F7AEF022EF8EF0A2F7D2F73392D5C5
:10D0BA00C3947F5006E4FFFEFDFC229420400474D2
:10D0CA00FF80F304CCFEE4FFFAE5F0CC6012C3CC97
:10D0DA0013CCCD13CDCE13CECF13CF0450EEDAEC52
:10D0EA0030D5D7C3E49FFFE49EFEE49DFDE49CFC9B
:0CD0FA0022E6FC08E6FD08E6FE08E6FF62
:10D1060022ECF608EDF608EEF608EFF622CFC51388
:10D11600CFCEC512CECDC511CDCCC510CC22E4F5EF
:10D1260013F512F511F51022E493FCA3E493FDA385
:10D13600E493FEA3E493FFA322C0E012D03E12CFF5
:10D146004A12D17212D12ED0E0C0E012D03E12D1D6
:10D156006912CF4A12D03E12D12E12CD3CD0E0D564
:10D16600E0E722AC48AD49AE4AAF4B228C488D4928
:10D176008E4A8F4B2274FF7809FFFEFDFCE526548C
:10D18600F048F5262212D23204A2E1927F1420E062
:10D196001590D2B3740412D13F802912D23230E1F5
:10D1A60002B27F20E0EB8C4C8D4D8E4E8F4F90D28D
:10D1B600C7740412D13F12D03EAC4CAD4DAE4EAF4B
:10D1C6004F12CF4A307F04EF6480FFEE33EF3370A7
:10D1D60001FF2212D232C0E08C4C8D4D8E4E8F4F05
:10D1E60090D2EB740312D13F12D03EAC4CAD4DAE93
:10D1F6004EAF4F12CF4AECC54CFCEDC54DFDEEC50A
:05D206004EFEEFC54FD4
:10D20B00FF90D2DB740312D13FD08212D03EAC4CD4
:10D21B00AD4DAE4EAF4FE58230E00712CFC2B27FBD
:10D22B00809D12CFBF8098EE33EF3324605007D030
:10D23B00E0D0E002D17BEFA2E7547F927FFF12D0C8
:10D24B003E7C837DF97E227F3E12CF4AEE33EF3355
:10D25B002481501012D03E12D0B012D075EFB2E72D
:10D26B00FF12CD3CEE33EF33602A2403F8C313FFD8
:10D27B00EE92E7FEE82481E4501A12D03E12D0B0B1
:10D28B00EF04C2E0FCF58212D07DEFB2E7FF12CDC6
:10D29B003CE58203FAEE33EF33600B148FF0A2F709
:10D2AB0013FFEE92E7FEEA2283FA703AE4E9AABC96
:10D2BB00F8E0813EE6E99DBF0000803F1A3C28392B
:10D2CB00666999BBE335A33DE75D25BFDB0FC93F1E
:10D2DB00CCDB8D41EE3649C43F91C9453DF8B0C515
:10D2EB000000803F34F517C373FA2F45DDFD0AC6E6
:10D2FB00EF2513FFEE3512FEED3511FDEC3510FC6D
:10D30B0002D05DC3EF9513FFEE9512FEED9511FD67
:10D31B00EC9510FC02D05DEFF88513F0A4FFE5133C
:10D32B00C5F0CEF9A42EFEE435F0CDFA88F0E51267
:09D33B00A42EFEED35F0FDE433F3
:10D34400CC8513F0A42CFCE5128AF0A42CFCE51186
:10D3540089F0A42CFCE51088F0A42CFC89F0E512DB
:10D36400A42DFDEC35F0FCE51188F0A42DFDEC3581
:10D37400F0FC8AF0E513A42DFDEC35F0FC02D05D41
:10D38400E4CCF8E4CDF9E4CEFAE4CFFB75F020C3A5
:10D39400E51333F513E51233F512E51133F511E511
:10D3A4001033F510EF33FFEE33FEED33FDEC33FCB9
:10D3B400EF9BEE9AED99EC98400CFCEF9BFFEE9AF4
:10D3C400FEED99FD0513D5F0C622C2D5EC30E70574
:10D3D400B2D512D0EDE51030E70DB2D512D3F1126B
:10D3E400D38412D0ED800312D38430D515C3E495D1
:10D3F40013F513E49512F512E49511F511E4951063
:03D40400F51022FE
:108F9E00E57124885002D2191261158E4712E60D22
:108FAE0012AA431264D1305E0F12646F12A12F12F7
:108FBE0063A0129D6F124E5C124578125403103648
:108FCE0026301219E4129121129136129231129218
:108FDE00533051030292DD1295AE205109C251E475
:108FEE00F552F545F5442275A700758307E559C47A
:108FFE0054F0F582E0F538A3E0F518A3A3A3E0F54D
:10900E001E74FF1291211261158E1C8F1B7510DFBD
:10901E00751100E51164B470061290EC7511101202
:10902E0090B94028AE1CAF1B12619D20321EAC03BE
:10903E00AB027A0C125DA4ED701275A70075830455
:10904E00851182ECF00583E510F00511D510C412E0
:10905E0090EC75C70375C6E075A7049005007F04F4
:10906E001290A7DFFB75A70012385712646FE4F554
:10907E00A7F8F559758307E8C4F582E065387011D5
:10908E00A3E06518700BA3A3A3E0651E70038859B7
:10909E002208C3E5589850DC22E0F5BCE0F5BDE0AF
:1090AE00F5BEE0F5BF1255F705C622E51075F004C2
:1090BE00A4F5C685F0C775B901E5BC33401F05C6DA
:0B90CE0005C675B90185BE6485BF654D
:1090D90005C675B90185BC6685BD6785BE6885BF4E
:1090E90069C322E51124FE502E75A7007F10AE1129
:1090F9001E7583048E82E0FD1582E0CDB505005012
:1091090012F00582CDF00583E0FD1582E0CDF00572
:1091190082CDF0DEDCDFD7227FB475A7549004003E
:1091290005A7900500F0F0DFFC75A7002212993918
:10913900C2517B077AFFE47F00F5A79004001292E1
:109149001DED244C4035EC603075A7008D8205A7D4
:109159001291E37583058D82E02410401CF005A768
:10916900E02CF0500505A7E004F0BA000CBB00099B
:10917900D251EF24DC50027F23DFC3EA600512914C
:10918900968006EB60031291CE75A7002230E004A9
:109199007553082230E1047553182230E2047553DF
:1091A900282230E3047553382230E40475534822E9
:1091B90030E5047553582230E6047553682230E7C8
:1091C900037553782230E0047553882230E1047521
:1091D90053982230E2037553AA22ED54F0C4232395
:1091E9009091ED735302FE225302FD225302FB229A
:0791F9005302F7225302EFBD
:10920000225302DF225302BF2253027F225303FE66
:10921000225303FD225303FB225303FB22129833F4
:1092200012B191E4F5F7E4ADF7F5F7E4ACF7D2B29B
:109230002290050078B4E06015FD54F0C4CD7C00A8
:10924000540FFE1583E0FF125EA2EFF00583058246
:10925000D8E42275830478FF088882E060FAF5D3A9
:109260008812E512244C50012285D3D288D488126A
:1092700079FF0512E51260F00908E875F0B484A8DA
:10928000F08882E060ECF5D3B9000280D5B9230004
:1092900050D0C395D292D15002F40409FEE4FFFCF1
:1092A000AD01125EAF7401FA25D475F0B484A8F054
:1092B000AC06AB07125D96EB30E7010CE5D22C3023
:1092C000D1029C9C8882F00AEAB501DCE512244CAC
:1092D00050012285D3D28512D4A812809390040025
:1092E00012939C8C068B0512939CE4FFF512F511EA
:1092F0008C148B13C3ED9BF9EE9CFA4012E5119987
:0B930000E5129A500A8C148B138A129D
:10930B0089118F528F82E0F9C3ED99FDEE9400FE27
:10931B00E582245A5002244C75F0B48485F082E027
:10932B00FA2DFDEE3400FEEB9AFBEC9400FCE92BDE
:10933B00FBEC3400FC0FBFB4B0E55224D340022445
:10934B00B4F552C3E51333FBE51433FCE511FE2BE7
:10935B00FBE512FF3CFC125F04E9F89093AE93F52A
:10936B0011FDEBF513FFECF514FE7C00125EA28FE2
:10937B0044E89094AE93FAAB13AC14125DCDAF03EB
:10938B00AE04AD117C00125EA2EF7002F552F545F2
:10939B00227C007B007F5AE02BFBEC3400FC058227
:1093AB00DFF522B4B4B4B4B4B4B4B4B4B4B4B4B498
:1093BB00B4B4B4B4B4B3B3B3B3B3B3B3B3B3B3B36D
:1093CB00B3B3B2B2B2B2B2B2B2B2B2B1B1B1B1B175
:1093DB00B1B1B0B0B0B0B0B0B0AFAFAFAFAFAEAE89
:1093EB00AEAEAEAEADADADADADACACACACACABABA7
:1093FB00ABABAAAAAAAAA9A9A9A9A9A8A8A8A8A7D0
:10940B00A7A7A7A6A6A6A5A5A5A5A4A4A4A4A3A300
:10941B00A3A2A2A2A2A1A1A1A0A0A0A09F9F9F9E38
:10942B009E9E9D9D9D9D9C9C9C9B9B9B9A9A9A9975
:10943B0099999998989897979796969695959594B4
:10944B009494939393929292919191919090908FF7
:10945B008F8F8E8E8E8D8D8D8C8C8C8B8B8B8A8A39
:10946B008A8989898888888787878686868585857E
:10947B008484848383838282828181818080807FC4
:10948B007F7F7E7E7E7E7D7D7D7C7C7C7B7B7B7A05
:10949B007A7A797979787878777777767676757549
:1094AB00757474000203050608090B0C0E101113DA
:1094BB00141617191A1C1D1F2122242527282A2BA5
:1094CB002D2E303133343637393A3C3D3F40424311
:1094DB00454648494B4C4E4F505253555658595A86
:1094EB005C5D5F606163646667686A6B6C6E6F700E
:1094FB007273747677787A7B7C7E7F8081838485A8
:10950B008688898A8B8D8E8F909192949596979859
:10951B00999B9C9D9E9FA0A1A2A4A5A6A7A8A9AA22
:10952B00ABACADAEAFB0B1B2B3B4B5B6B7B8B9BA08
:10953B00BBBCBDBEBFC0C0C1C2C3C4C5C6C7C7C804
:10954B00C9CACBCCCCCDCECFD0D0D1D2D3D4D4D51D
:10955B00D6D7D7D8D9DADADBDCDCDDDEDEDFE0E04C
:10956B00E1E2E2E3E4E4E5E5E6E7E7E8E8E9EAEA95
:10957B00EBEBECECEDEEEEEFEFF0F0F1F1F2F2F3F2
:10958B00F3F4F4F4F5F5F6F6F7F7F8F8F8F9F9FA69
:10959B00FAFAFBFBFBFCFCFDFDFDFEFEFEFEFFFFF6
:1095AB00FFFFFFC251E4F544F814FB900400A9003F
:1095BB007C0FC2D11296C9E82405F8B8B4F08B130E
:1095CB00E5122403FA244C5001FABBFF012275115A
:1095DB002C8A191297008F16203D12AA1975112388
:1095EB001297008F15751600303DE280117511230F
:1095FB001296A8751500303D05E82F13F51575115A
:01960B00124C
:10960C001296A8751400303D05E82F13F514EA24C2
:10961C0004F552244C5002F552E4F51AF51BF51CD6
:10962C00E516600AFB7A00AF137EFF12966EE51505
:10963C00600AFB7A4FAF137EFF12966EE516600D33
:10964C00FB7A00E5146006FF7ECF12966EAE1CAF5F
:10965C001B7C00AD1A125EA28F45EF2513F544D288
:10966C005122EFF5F0A4FCADF0EBF5F0A49CFCE579
:10967C00F09DFDEB8AF0A4FAABF0EF8EF0A49AF813
:10968C00E5F09BF9E833F8E933F97B00125F480504
:10969C001AE51B2BF51BE4351CF51C22EA2511F9E8
:1096AC00244C5001F9C2D11296C7303D428F00C3F1
:1096BC00EA9511F9500324B4F9D2D17C09E4FDFEEA
:1096CC00FF8982E060062FFFE43EFE0D09B9B4026B
:1096DC007900DCEDED20D118F51E24FE923D500FE3
:1096EC00125EAFEFB503005006851E1FFB881222D9
:1096FC00F51D80E61296A8203D43740212979F1226
:02970C0096A81D
:10970E00203D3874041297A71296A8203D2D74069A
:10971E0012979F1296A8203D2274081297A71296B0
:10972E00A8203D17740A12979F1296A8203D0C741C
:10973E000C1297A71296A8203D0122C3E89F6050F5
:10974E0088148F158A1640081ABAFF0A7AB3800653
:10975E000ABAB4027A001296A8303D34C3E89FF9D3
:10976E00602EC3E5149515FB6930E7D4E930E703A5
:10977E00F404F9EB30E702F404C3995002AA16E59B
:10978E00142515C82F28FFE4FC33FE7D04125EA2BB
:10979E00222AFA244C5001FA22C3CA9AFA50032400
:1097AE00B4FA2212188E85BF6C85BE6B756A0002E4
:1097BE00B174129CEB852E72E55F030354C0F8E57D
:1097CE005E543F28F57C3055062212B0ED80031210
:1097DE00B0DD7410256A54F0F56AE4356BF56BE470
:1097EE00356CF56C24815003756C0022756A00E4AB
:1097FE00D380E8E54B75F010A4256A54F0F56AE5C0
:10980E00F080D8E56A24F054F0F56AE56B34FFF584
:0E981E006BE56C34FFF56C24815003756C7E95
:10982C0022E56A24FF80E4E56D24F054F0F56DE543
:10983C006E34FFF56EE56F34FFF56F2481500375C0
:10984C006F7E221298AB129908C22DC254C255E5F4
:10985C007F7002D255147002D254E54A30E00122D6
:10986C00B4062120540C129811129BBD129C6C0250
:10987C009D02129DE37E0412F15D754A0112F157AF
:10988C00756A202220550C1297E0129C3D129CEB1D
:10989C00029B96129DE37E0412F15D754A0522121D
:1098AC00B17C7870E4F5F7E4A6F708B880F6D2B28C
:1098BC0022129939756D1012B191E4F5F7E4E5F7C0
:1098CC00D2B264C0702D756D1E12B191E4F5F7E43F
:1098DC00E5F7C4F9E4F5F7E4E5F7D2B2C4F8E954D6
:1098EC000FFD5301F0E8540F49FCE854F0FB7F03E3
:1098FC00129B28056EE56E540370B922E575F85479
:10990C001F30E40244E0F57585722EA2779226E5AD
:10991C007C543F30E50244C0F55EE57C54C0232303
:10992C00F55FE57FC2E779BCF709A77E22856C6FEE
:10993C00856B6E856A6D22856F6C856E6B856D6A25
:10994C0022FA7420303B0274608510F0A4256EF569
:01995C004DBD
:10995D00E5F0356FF54EEA2323303B0475F003A493
:10996D00254DF54DE5F0354EF54E754C00227580C3
:10997D0000C2B212F165D2B222758000C2B2F5F703
:10998D00A4D2B222758000C2B2F5F7A48DF7A48CD3
:10999D00F7A48BF722EB241054F0FBE43CFCE43DE0
:1099AD00FD22EB24F054F0FBEC34FFFCED34FFFD15
:1099BD0022758000C2B2F5F7A4856FF7A4856EF706
:1099CD00A4856DF722E56D241054F0F56DE4356E28
:1099DD00F56EE4356FF56F22756D00E56E24045458
:1099ED00FC80EDE56D24F054F0F56DE56E34FFF57A
:1099FD006EE56F34FFF56F22756D00E56E24FC5436
:109A0D00FC80EC758000C2B2F5F7A4854EF7A485F5
:109A1D004DF7A4854CF722740F254CF54CE4354DCC
:109A2D00F54DE4354EF54E2274F1254CF54CE54DD2
:109A3D0034FFF54DE54E34FFF54E22754C00E54DE6
:109A4D0024FC54FC80EC7403129A1075A70090044A
:109A5D000075F700A4E5F7F0A3E58324F850F2753F
:039A6D00F700A45B
:109A7000E5F7D2B2C23C30E602D23C754C00E54D6F
:109A8000240454FC80A77403129A1075A700900454
:109A9000007F22129ABB8010E54C2411FBAC4D0CC8
:109AA0000CAD4E740312999175A7009004117F00BC
:109AB000129ABB7FEF129ABBD2B22275F700A4E5CF
:109AC000F7F0A3DFF622D23CE4F56FF56EF56D7486
:109AD000031299BEE4F5F7A4E5F7D2B204600BC215
:109AE0003C1299D2E56F24FE50E5923D227F107919
:109AF000B8740612998674021299BE87F709DFFBC3
:109B0000D2B280337F1079B874031299BEE4F5F7AE
:109B1000A4A7F709DFF7D2B278B9793A12DBA40229
:109B20009C8AAD6FAC6EAB6D74061299867402128E
:109B300099918FF7A4D2B2758000C2B275F705A4CF
:109B400075F705A4E5F7D2B220E0EC227403129970
:109B500091E4F5F7A4E5F7D2B222E4FEFF740775AD
:109B6000A704F5838E8274FFF0DFFD75A7002274D1
:109B7000067E007FB0129B5FE4F55AF55B2275A765
:109B800004758306E55A600A75F00A84E5F07002F0
:0B9B9000740AC4F58222307720E55AE9
:109B9B0024024002055A129B7EE55AF0E573F0E56C
:109BAB0074F0E575F0E576F0E577F0E578F075A7FC
:109BBB0000223077F9129B7E7F1074FFF0DFFDE5FA
:109BCB005A24F55003129BE8155AE55AB4FF0205C7
:109BDB005AC3E55A955B50D6755B0080D112993903
:109BEB007F0A056D056D12B191E4F5F7E4E5F7D247
:109BFB00B230E704DF02800512983380E5056D1261
:109C0B00B191129B7EE55A24F6F07F06E4F5F7E45A
:109C1B00E5F7F0DFF7D2B275A700227F42129C2E38
:109C2B00DFFB22302B0C0542E542247C40012275E0
:109C3B004280053FE53FB43C17753F00053EE53ECE
:109C4B00B43C0D753E00053DE53DB41803753D0074
:109C5B00802D302B0C1542E5422483500122754296
:109C6B0080153FE53FB4FF17753F3B153EE53EB40E
:109C7B00FF0D753E3B153DE53DB4FF03753D177874
:109C8B00ABA63A08A63B08A63C121875E5BF253DC6
:109C9B00240C75F0188478AEA6F018600564026089
:109CAB00182216E670121816E67004760C18167841
:099CBB00ACE6909CDE9308F62251
:109CC4000618E608909CDE930466700D760118066B
:109CD400E6640D70047601180622001F1D1F1E1F66
:109CE4001E1F1F1E1F1E1F0542E542B43C0F754276
:109CF400000541E541B43C0575410005402215428B
:109D0400E542B4FF0F75423B1541E541B4FF0575CB
:109D1400413B154022AC40AB41A842EC75F03CA459
:109D24002BFBE435F0FC7A3C125D96EB28FBE43C1B
:109D3400FC22AC3DAB3EA83F80E178AE8604AB3E4E
:109D4400E53FC313F8800C7800121857E5BE75F090
:109D540005A4FBE5BF75F03CA42BFBE435F0FC7ACD
:109D64001E125D96EB28FBE43CFC22129D4BAE04D4
:109D7400AD03129D3E8C148B13121861E5BFFF24B2
:109D8400F650027F01E5BE75F096A4AAF0F9C3ED82
:109D94009513FBEE9514FC924E4B701120110E306E
:109DA400480B75364B3003037536FFD22E304E0206
:109DB400DF1F7A02125D9675A7009004EEECF0A303
:109DC400EBF0C3E5BF9F04BF0102D2E79005CBF0DF
:049DD40022ED29FD56
:059DD800EE3AFE80B52B
:10F14A0012F15312F15312F1537E0480067E0280AB
:10F15A00027E017F0080087F6480027F017E00EFCB
:10F16A004E6012E4FD0D1D0DEDC394AD40F7EF1F87
:10F17A0070ED1E80EA2212F31290C0227F001281E3
:10F18A003712F19B12F153753500C200C201C20257
:01F19A002252
:10F2FE00F5D8D2DCE5F520E7FBE5DA540FFEAFD901
:04F30E0075D800228C
:10EF06007F767E0690B6FD128149740412F2FE7C6D
:10EF1600007D52125EA2EFF875F00A84C0F07F768B
:10EF26007E2312E8E97E29742E12E8FC7E2ED0E0BC
:10EF360012E8E97E35745612E8FC7F6B7E1190EF7D
:10EF46006F12E928E824E04001220423F824E75060
:10EF560002781812EF5FD8FB227F6CE82411FE7945
:10EF66000512F22D0E0FD9F922071DFFFFFFE080D3
:10EF7600000020C0000038E0000008F0000038F86B
:07EF8600000020FFFFFFE087
:10F00A0012F03230E6022409540F75F00AA4F515FD
:10F01A0012F03230E6022409540F25152212F0327A
:10F02A00540F2275F000800875F044800375F007CC
:10F03A00E4206D09D5E0FAD5F0F7D24C229247C206
:10F04A00ACE54F623885504FA26E926D859950C2D9
:10F05A006FD2ACC24CA2472212F06CC4FA12F06C06
:10F06A002A2212F03220E603540F225407240922DE
:10EF8D00E612EF9418E608FAC412EF9AEA540F4409
:10EF9D0030F924C6E950112407800D75F00A84C09C
:10EFAD00F012EFB3D0E0443030530975F00085E036
:10EFBD00E0D5F0FA3099FD75F019D5F0FDC299F54F
:10EFCD0099623822E53880EC742A12EFC16238E577
:10EFDD003812EF94800812EFB5E53812EFB5740DC5
:10EFED0012EFB5740A80C1744012EFB5744080B849
:0DEFFD00742C80B4742E80B075380080AB89
:10F3240085A0835383FE438380858384F0758400A2
:01F3340022B6
:10EDB30074A212F32474A112F32474A612F324741C
:10EDC300A412F32474C012F324742512F32412EE54
:10EDD3004475C70375C6FC75B90112AA637408129A
:10EDE300F2FEEE75F020A4FEEF54F80303032E2485
:10EDF30092C313FE24EA50027E16EE90EE2D932565
:10EE0300BCFE24E6502024E8401C748112F324EE57
:10EE130012F32412EE51744012F324742F12F324CC
:10EE230074AF12F324227E2680E0F7F7F8F8F9FA9C
:10EE3300FBFCFDFEFF0000000001010202020303D0
:10EE430003A8BCA9BDAABEABBFACC7ADC62288BCD4
:0BEE530089BD8ABE8BBF8CC78DC62214
:10F19B00C006C007C5F075A7019000007EB7E58CCF
:10F1AB00240340FA12F1BD1EBEAFF3C5F0D007D059
:10F1BB00062275A700EE12F324741012F3247404C4
:10F1CB0012F32485A08343838185838475A7517FA4
:10F1DB0020E0F0E0F0E0F0E0F0DFF6E4F5A7F584F6
:01F1EB002201
:10F3120075A711900000E4C583F0C58330E2F8F5CB
:02F32200A72220
:10F22D00EF20E723EE20E71F20E61C05A7C45403BB
:10F23D00F583EE5408C42FF582EE5407240983F5A7
:10F24D00F0E045F0F005A7228040201008040201EF
:10F25D00EF20E723EE20E71F20E61C05A7C454038B
:10F26D00F583EE5408C42FF582EE5407240983F577
:10F27D00F0E055F0F005A7227FBFDFEFF7FBFDFEB5
:10E8A700FDA42582F582E5F03583F583ED227E0010
:10E8B700906AE57A0475F00512E8A77D05805E7A0F
:10E8C7000580027A04547FC0E0C083C082C39420CD
:10E8D7005001E4906A9512E8BC802E906BF37A059C
:10E8E7008005906CB07A0675F00712E8A77D07805F
:10E8F7002C7A0580027A06C0E0C083C082C39420C8
:10E907005001E4906C4012E8EED082D083D0E02230
:10E91700906A0975F00A12E8A77D0A7A07C2D180C2
:10E9270002D2D1C0A7C082C083C007C006C0E030F2
:10E93700D10975A704E493FDE493FAEEFB75A704E8
:10E94700EBFEEAFC7901D9067908E493F5D4E5D41E
:10E9570023F5D420E01612F25D0EDCEA0FDDE1D0DC
:10E96700E0D006D007D083D082D0A72212F22D8024
:10E97700E890694975F00E12E8A77D0E7A0812E94A
:10E98700249069F175F00212E8A7E493FDE4A393DC
:10E99700FACE2408CE7C0812E9A57C06AD02ED2349
:10E9A700FD20E00712F25D0FDCF42212F22D80F752
:10E79200F5D2C2D58036F5D2D2D58030F5D224F664
:10E7A20050090E0E24A650030E0E0EE5D2F5D275B8
:10E7B200F0648485F0D3C2D57009D2D5742012E8F2
:10E7C200FC800312E8E9CE2406CEE5D375F00A8474
:10E7D20085F0D3700A30D507742012E8FC8003124A
:10E7E200E8E9CE2406CEE5D312E8E9E5D222F5D255
:10E7F20075F0648485F0D3C2D58022F5D2C2D5806B
:10E8020025F5D2D2D5801FF5D275F0648485F0D378
:10E81200C2D57009D2D5742012E8FC800312E8E256
:10E82200CE2405CEE5D375F00A8485F0D3700A3084
:10E83200D507742012E8FC800312E8E2CE2405CE4C
:10E84200E5D312E8E2E5D222F5D2C2D58035F5D27F
:10E85200D2D5802F30E70DF404C0E0742D12E8CA3F
:10E862000E0ED0E0F5D275F0648485F0D3C2D57077
:10E8720009D2D5742012E8CA800312E8B7CE240464
:10E88200CEE5D375F00A8485F0D3700A30D50774CB
:10E892002012E8CA800312E8B7CE2404CEE5D312D0
:05E8A200E8B7E5D222F9
:10812E0090B9F012813702F19B7E00800E7405FE2D
:10813E00F51EE4FFF51DF51F203C3375A700E493F3
:10814E00700122A3B40204051D8003B4010A051FA9
:10815E00EF2409FFAE1E80E612E8FC7D06B4400255
:10816E007D03B421027D02EE2DFE80D27E0075A726
:10817E0000E493700122A3B40204051D8003B40130
:10818E000F051FEF2407FFAE1E80E612E8C680081B
:10819E00B45B0050F612E8CA0EB4210280D30EB4BE
:1081AE00400280CDB42C0280C80E0EB45F0280C196
:1081BE00B45B0040BC0E80B9E60812E8FCEE240663
:1081CE00FED513F42290B72B30740990B72F30736D
:1081DE000390B73402814975F019D5E0FDD5F0FA58
:1081EE0012545712EFF4744F12F005744B12EFE362
:1081FE00C322C250128244125457D2AC12F02D3008
:10820E004C1212F02D304C0C12F02D304C06D25078
:10821E00C2ACD322B440E512F032B4400312F032B5
:10822E00B44FED12F032B44BE712F03212F03212BC
:10823E00F032C2ACC32230530975F008D5E0FDD53B
:10824E00F0FA227F0575F019D5E0FDD5F0FA12543B
:10825E005712EFF4745712F005745012EFB5748183
:0A826E0012EFB5E56312EFB5E5620B
:1082780012EFB578D0E612EFB508B8D7F8E6F87976
:108288005F30E702792FE912EFB512EFB512EFB5BB
:1082980012EFB5745812EFB5744312EFB5E412EF4C
:1082A800B5E8C2E775F00A84C425F012EFB5786422
:1082B800E612EFB508B869F8E612EFE3128200405B
:1082C8000122DF02800A20508B75F0008080D25096
:1082D800C2ACD322128244C250125457D2AC2002EC
:1082E800EF12F02D204CE7B440F412F032B4400302
:1082F80012F032B457DAF53812F032B450D212F024
:108308003212F032F56312F032F56278D012F032A0
:10831800F924A0500353015FE924E04002795FA6E5
:108328000108B8D8E8780612F032D8FB12F032FC0F
:1083380053040FC4540F75F00AA42CFC249C50025B
:108348007C0078D78601E4B92F02D2E72CF678644E
:1083580012F032F608B86AF812F032E53860030213
:1083680082D812F03212F032C2ACC32290BEE5803D
:108378000390BA347F2012817A12F19B02F15B7567
:108388003400C26B12844312F15B1287FAE516605F
:108398000312839F020211128A4F12287312F19B53
:1083A80010002010010280F8128865501312287EF0
:1083B80012837410000D10010280F812281980D75A
:0483C8001285E62212
:1083CC00C26BD22775480A12384B753400128925B6
:1083DC00C26A123FDD106A0512020280ED1202021F
:1083EC0012878C1288E412893178D0E664266044B6
:1083FC00128A4F12287312F19B1000381001028060
:10840C00F8128865501BE96515601812287E1283D6
:10841C007412F15310001D10010280F812281980FB
:10842C00BCD26B1289107516078559171238C47592
:10843C00350080960202111287FA12846512893176
:10844C007F1912847F90BF127E1212817C7E23E5ED
:10845C001602E86690C06080EF7862E41284767849
:10846C00D0745F12847618E4F6227F08F608DFFCDD
:10847C00227F7B7E007810742012E8CACE2404FE82
:10848C00D8F5221220C37F197E0812817C7E289099
:10849C00BA2030530390BA1B02817CC26B128465E4
:1084AC001284B2020211C25112893190BF0A128495
:1084BC008F12283F1287FA7F2012844E12F19BE50F
:1084CC0016700512F150803675A6FF3051031281DB
:1084DC00EE125457D2AC200025306DFA1282DF40D8
:1084EC000C12886540111285E6D25180BB105003E6
:1084FC00128379C25180D1D25112837480CAC2AC1A
:10850C0022D22775480A12384B753400C26B128977
:10851C0025C26A123FDD106A0512020280EB1202BC
:0F852C000212878C1288E412893112853E50DAD0
:10853B0002021190BA2F12848F12285812F19BC38A
:10854B0010001310010510020E80F412825140012D
:10855B002212837980DDD3C2AC22D227C26B75483D
:10856B000A12384B753400128925C26A123FDD108E
:10857B006A0512020280EDD26B12878C1288E4120C
:10858B0087B475B901E5BCB2E7F5BC1255F77516A2
:10859B00078559171238C480CB1287FAE516601F6E
:1085AB0078D0E53D1285D7E53E1285D7E53F12859C
:1085BB00D7765A08765F12DB9A1289100287CB7F27
:1085CB003E7E1190BA0612814902F19B75F00A8426
:1085DB004430F608E5F04430F60822D26B128910CD
:1085EB001287CBE51775F01084240AF54824E85060
:1085FB000375480A12385785585922D22075320014
:10860B00129B5A75A7049007007515001287B47555
:10861B00B901E5BC20E705E515F0801004600D6499
:10862B0082600975BCFF75B90575B9020515E515AD
:10863B00242050D8E58224FE40030286E1A882184C
:10864B007F0075A7007583078882E0FE75F004A490
:10865B0012875FA9BCAABDABBEACBF1582E0FD758E
:10866B00F004A412875FC3E995BC404C7052EA95A5
:0D867B00BD4045704BEB95BE403E7044EC99
:1086880095BF4037703DEE75F004A40412875FA9CA
:10869800BCAABDABBEACBFED75F004A40412875FE5
:1086A800C3E995BC4015701BEA95BD400E7014EBEC
:1086B80095BE4007700DEC95BF5008EEF00582EDB1
:1086C800F01582E5826009C3EF9582500302865552
:1086D8000FC3E89F400302864D75A70490070075F5
:1086E800C70375C6A8E0F5BCE0F5BDE0F5BEE0F54A
:1086F800BF75B90575B90205C6E58224204006E5AF
:10870800C6242050E00875C70375C68075B901E511
:10871800BC128749F5BCE5BD128749F5BDE5BE1217
:108728008749F5BEE5BF128749F5BF75B90205C689
:10873800E5C6245850D6E5320470FB75A700C22060
:1087480022B4FF0122F975A704900700E58268604A
:1087580005E06970F7E922F5C685F0C775B901E546
:10876800BC645F700375BC27E5BD645F700375BDAD
:1087780027E5BE645F700375BE27E5BF645F7003BD
:1087880075BF272275C703E54875F004A42480F552
:10879800C6E55975F00484A8F00825C6F5C675B96C
:0787A80001A9BCAABDABBE94
:1087AF00ACBF861522E515242050037515DFE5159E
:1087BF0075F004A454FCF5C685F0C722E5172420F4
:1087CF004028E51775F00484A8F00824A8F5C675AD
:1087DF00C70375B901A9BCAABDABBEACBFA61589AD
:1087EF00BC8ABD8BBE8CBF1255F722E4F516F5156A
:1087FF0079FF1287B475B901E5BCB4FF040516A95A
:10880F00150515E515242050E9891579FF75C7035E
:10881F0075C6A875B90109E5BC04601B09E5BD045F
:10882F00601509E5BE04600F09E5BF04600905C6C0
:10883F00E5C6242050DD098917227516007515012C
:10884F001287B475B901E5BC20E70205160515E5D9
:10885F0015242050EB227900E975F004A454FCF59F
:10886F00C685F0C775B901E5BC20E73078D06670D2
:10887F002B08E5BD66702508E5BE66701F08E5BFCD
:10888F0066701905C675B90108E5BC66700E08E576
:10889F00BD66700808E5BE667002D32209E9242080
:1088AF0050B6C3221288D31288BBA8017F08E0F606
:0C88BF0008DFFB221288D31288CBA8012E
:1088CB007F08E6F008DFFB2278D0796275A7047584
:1088DB008307EBC454F0F582221287B478D0128848
:1088EB00FEE5BCF9C23C20E702D23C1288FE78625E
:1088FB001288FE75B901A6BC08A6BD08A6BE08A6BF
:10890B00BF0805C622D2201287B478D012811C1260
:10891B00811C786212811C02811C12646F12F3128B
:10892B00129F2502F19B12F3127F007E0990BEF776
:10893B001281497F0A7E12E5150412E79E7F1412FD
:10894B00DD8B1228197F277E0875130778D01281CB
:10895B00C6E6793E30E702792F7E34E912E8FC7FD8
:10896B003D7E0190C07C12817C20311B3030031284
:10897B00C222C23B128BE1128997D23B128BE112BE
:10898B0089A9128C28807C12D40780E6C23B7F44D5
:10899B007453201702744E7E0012E8FC8017D23BF2
:1089AB007F4F745720170274457E0012E8FC7E0639
:1089BB00E51E12E8E97E0CE51D12E8E97E12E51CC6
:1089CB0012E8E97E17748112E8FC7E1CE51B12E8A5
:1089DB00E97E22E51A12E8E97E28742E302602740D
:1089EB002712E8FC7E2DE51912E8E97E33E5181213
:1089FB00E8E97E39302607742C12E8F87E3BE53720
:108A0B0002E8E9742D201702742B7F707E1512E893
:068A1B00FC128A2C7E3AD9
:108A210012E7477E0190C0A70281497E1BE51C1217
:108A3100E8E97E21E51B12E8E97E27E51A12E8E95B
:108A41007E2DE51912E8E97E33E51802E8E9128A7C
:108A5100CD128AF8128DCF128931128E2720171E5E
:108A610010021B12B23B12DB9A128AB51228247F24
:108A7100347E2F1281D312896A12F19B80E212286F
:108A810019203026203128C23B128BE1128B0D7840
:108A910066128CE1D23B128BE1128B227869128C27
:108AA100E1128C28128B9C028D8412C2EB80F2128F
:108AB100D41C80EDE57D75F01084AAF075F00AA450
:108AC1002A547FFA78D7E654802AF6227F277E0837
:108AD10079D08700C001D224B9D002C224128EAE4F
:108AE100D001A70010230909EE2406FEB9D7E3221D
:108AF10019EE24FAFE80DB7E3479D7E7A2E79217DC
:108B0100128E5B79D7E7A21792E7F722C224C23B04
:108B1100751E007F447E00128E6B801E1023ED8037
:108B21002AD23BC2247F4F7E00128E73D2247E064E
:108B3100E51E128EA0F51E1023E7D2247E0CE51D42
:108B4100128EA0F51D303BD41023E1D2247E12E514
:108B51001C128EA0F51C1023E17E1CE51B128EA0B9
:108B6100F51B1023E67E22E51A128EA0F51A1023BA
:038B7100E87E2D6E
:108B7400E519128EA0F5191023E87E33E518128E3C
:108B8400A0F5181023E87E393026027E3BE5371223
:108B94008EA0F5371023E3227F707E15128E63C2F8
:108BA400247E1BE51C128EA0F51CD2247E21E51B1D
:108BB400128EA0F51B1023E77E27E51A128EA0F56E
:108BC4001A1023E67E2DE519128EA0F5191023E85C
:108BD4007E33E518128EA0F5181023E82278D7E624
:108BE400C2E775F00A847866F537303B0578698505
:108BF400F037128C5130262BE53775F003A40404AA
:108C040075F00584FBE51975F00AA4251875F006BE
:108C1400A42BFBE435F0FC125FBEF537125FBEF502
:108C2400188B1922E563FC339217AB625003126070
:108C34002F305C0A7AD2125DA47840125F46AE04EB
:108C4400AF037C277D10125EAF8F1C8037E6FD33A7
:108C5400921718860418860350031260377A09792C
:108C64002778C0125F438B1EADD3ACD2AB0679EA32
:108C74007860125F418B1DAF06AED27C177D7012F7
:108C84005EAF8F1CAF05AE047C037DE8125EAF8F30
:108C94001BAF05AE047C007D64125EAF8F1AED75C8
:0A8CA400F00A84F51985F01822EC9F
:108CAE00339217500312602F751D30301786751DC5
:108CBE002D808178427B607CEA800678407B207C28
:108CCE004E12D4E779277810125F418B1CAF06AE97
:108CDE00D280AB30262AE51975F00AA4251875F056
:108CEE000AA42537FBE435F0FC7A05125D968C0656
:108CFE008B077C007D03125EA28E048F03128C1BE9
:108D0E00E51E75F00AA4251D75F00AA4251C75F044
:108D1E0006A4251BFBE435F0FC7A0A125D96EB25C2
:108D2E001AFBE43CFC7A0A125DA4EB2519FBE43C29
:108D3E00FCE43DFD7A0A125DB6EB2518FBE43CFC23
:108D4E00E43DFD301703126037A60518A60418A6D9
:108D5E000378D7E6A2E7923DC2E775F00A84FCAB32
:108D6E00F0303B0EAB37EC75F00AA42BA23D92E728
:108D7E00F622AC3780F0128D9F305C0A7A40125D7D
:108D8E00A478D2125F4630170312602F8C638B6269
:108D9E0022128DAF7A0A125D96EB2518FBE43CFC8D
:108DAE0022E51C75F00AA4251B75F00AA4251AFBF2
:068DBE00E435F0FC7A0A26
:108DC400125D96EB2519FBE43CFC22128E0112F194
:108DD40057C202C223128E011000081001051002AE
:108DE4001B80F51031ED10300D102604D22680E3DF
:108DF400D230C23180DDD231C23080D7227F35906B
:108E0400C06512817A90C08320300F90C09F2031BA
:108E14000990C07420260390C06C1F7E17128149EC
:108E240002F19B7F357E0190B9E312817C7F347E11
:108E34003A128F50744E12E8FC12F19B12F157C291
:108E4400027F347E3AD21775115975124E802675F9
:108E5400112E751227801E75113E75122F801675FE
:108E6400112B75122D800E75114E751253800675D7
:108E74001145751257128F50E511301702E5121281
:108E8400E8FC12F19B10000810010510020B80F59C
:108E9400D23C1017E3D21780DF028F4B4430F81214
:108EA4008EAAE8540F22C2218002D221A224922247
:108EB4009223128F50E830E709D23C7430302102FB
:108EC400745FF812E8FC12F19B10003410010510D5
:108ED400025D80F5D23C102266102367B439097410
:108EE4005F2021DF743080DBB45F04742D80D4B440
:108EF4002D04744180CDB45A04743080C60480C3F8
:108F0400D23C302406102237102338B44104742D87
:108F140080B1B42D04745F80AAB45F04743980A353
:058F2400B43009745A8D
:108F290020219B74398097148094B48908D223E84E
:108F390012E8FC800DF8C223800874898001E802D8
:108F49008EC7908F9A8003908F96C007EF2408FFF1
:108F590012E928D00702F19B128F50E830E704D2BA
:108F69003C7441F812E8FC12F19B10000810011141
:108F79001002CF80F5D23CB44104745A80E51480C4
:108F8900E2D23CB45A04744180D90480D60205F86F
:058F9900F802050000D4
:10F0EA0075A70090F11C75F02D84C2D5C2D16017A6
:10F0FA00D2D1146007D2D514600DC2D1E5F093FCC9
:10F10A00742D95F093FB22E5F093FB742D95F09303
:10F11A00FC220009121B242C353E474F58606870A8
:10F12A007880888F969DA4ABB2B8BEC4CACFD4D912
:10F13A00DEE2E6EAEDF0F3F6F8FAFCFDFEFFFFFF89
:10F1EC00D23D8002C23DED8BF0A430E70205F0C3A6
:10F1FC00E895F020D50425F025F0FEED8CF0A43038
:10F20C00E70205F0C3E995F030D10425F025F0FFB5
:10F21C00203D0B2487500122EF24CC40012202F226
:01F22C002DB4
:10EB7800203A7A7E1C7F5312F22D7F5912F22D1EF5
:10EB88007F5712F22D7F5512F22D7E2312F22D7F20
:10EB98005712F22D1E7F5912F22D7F5312F22D1F9C
:10EBA8007E2012F22D7F5A12F22D7E1E12F22D7F38
:10EBB8005212F22D121861E5BD20E0143006117FC3
:10EBC800357E1C90EC36E571700390EC4002E92824
:10EBD800E5716018E57012F0EA781F79567D091220
:10EBE800F1F0303A0312EC090DBD16F3227E1C7FBA
:10EBF8005390EC1F12E928200CD67E1F12DDF280FC
:10EC0800BEC0060E30D5021E1E12F22DD0061F30D1
:10EC1800D1020F0F02F22D070700386C446C380040
:10EC280005052070D8702005057088A88870080729
:10EC380010387CFE383838000807102844C62828C1
:02EC4800380092
:10DBC60090C0B17F717E2312817C121861E5BC7E04
:10DBD6003112E8B730121AC23C121861E5BCFB7567
:10DBE600F00AA4F904FAC23D12993912DE69303DF1
:10DBF6000122DAF712DD6B7C00EBF4042E4019AD3E
:10DC060003125EA2EFA2D1203C077E237F6502E5C8
:10DC160014AE16AF1702DD0CAD01125EA2EF12E6CE
:10DC260002203C077E237F6502E538AE16AF170259
:10DC3600DD307F567E0512DD977F3D12DDAA7F6FB0
:10DC460012DDAA12DDF27E0A7F4112DE257E227FD8
:10DC56005912DE2520120122129939857A1D855E18
:10DC66001C857B1B855F1A7AC0C23D12DE65203D8E
:10DC76005212DD6B7C007D14125EA274562F20D1E9
:10DC8600029F9FFF24CB40028037EF2488500280FA
:10DC960030EA1475F00384FE12F22DC3E51B957B62
:10DCA600FEE51A955F92D55004EEF404FEEEC3131A
:10DCB600FE24E0400C741F2E30D5029E9EFE12F20A
:10DCC6002DDAA8227F5212DCDC7F5A12DCDC7517B3
:10DCD60053751600802B7E0012F25D0EBE12F922DD
:10DCE6007F157E28742012E8FC7F1C7E2812F25DC8
:04DCF6000EBE40F925
:10DCFA00223012E712DCE675171575162DD23C0292
:10DD0A00DBDFC23D6002D23D92D175F080305C0407
:10DD1A00F5F08001A4A2E792D5E5F075F03284F817
:10DD2A00E5F075F00584C0E0E5F0A2D533C0E0E87F
:10DD3A00601E12E8E9EE2406FED0E0F8D0E012E810
:10DD4A00E9EE2406FE742C12E8FC0E0EE802E8E95D
:10DD5A007420303D07742B20D102742D12E8FC8008
:10DD6A00D4C3ED957AFFEC955EFE92D15003126012
:10DD7A001F227F1512DD837F327E3E12F22DDEFBDB
:10DD8A00227E0912F22D0EBE36F9227E0112F22DE2
:10DD9A000E0EBE3FF8227E3312F22D0EBE40F9223D
:10DDAA007E047D1112F22D0E0E0EDDF81F1F7E3538
:10DDBA0090C0BA305C057E3190C0BE02817C740589
:10DDCA00305C097E32740112E8B774067E3612E8B6
:10DDDA00B77E3A740012E8B77E3D02E8B77F1512A3
:10DDEA00F22D0F0FBF2DF8227F417E1F7D0F12F2F9
:10DDFA002D0F0F0FDDF8227F687D0380047F677D7A
:10DE0A000512F22D0FDDFA227F667D0780F37E1F51
:07DE1A007F5012F22D1F1FC3
:10DE2100BF3EF8227D0A12F22D0E0E0F0FDDF722F2
:10DE3100203D071248B47003D23D22056D12B19105
:10DE4100E4F5F7E4ABF7F5F7E4E5F7FA30E411EBC5
:10DE5100251DF51DE4351CF51C0519EA30E3010EFD
:10DE6100D2B28015780380027801203D071248B4B0
:10DE71007003D23D22D8F3056DE56D2409F56D12CD
:10DE8100B191E4F5F7E4ADF7F5F7E485F71BF5F7A4
:10DE9100E4E5F7FCD2B2543F30E50244C0CC54C0B3
:0BDEA1002323F51AE56D24F6F56D2231
:10EA9F007E017F0990EB1D12E9282051097E037F2B
:10EAAF0000743F02E8FCE4FEFFC3E54512E33DFDC1
:10EABF00940AED403D9464ED4002746312E7987E32
:10EACF00017F09E552240575F02D84AAF075F00534
:10EADF00A4CA75F00B842A90EB089312F0EABCB825
:10EAEF00027BB87D04EE2DF8EF2DF90D12F1ECDD60
:10EAFF00FB227E0312E8E980C6000C1622222D3974
:10EB0F00444F4F5A66707C7C87939EA9A9000909D0
:10EB1F000800410000000000888000000000410054
:10EB2F000800121875E5BCB4F8339004C3E0602CEC
:10EB3F00FA24F340277F137E0012F22D0F0F12F2EB
:10EB4F002D0E12F25D1F1F12F25D0EDAEC7F147E96
:10EB5F000012F22D0E12F25D0EBE12F5229005CCB0
:09EB6F00E0C3941240F60480C7D3
:10E33D00305D0A75F08AA42480E5F0340022207443
:10E34D00157F017E1190E3C512E9287F0A7E0AE54B
:10E35D002E540702E7AF7F087E1190E3D512E9280E
:10E36D0020730C7F0A7E1712F25D0E0E12F25D7F86
:10E37D00007E0BE57112E33D12E79E7F0C7E11E5E9
:10E38D0071602F0EE57064B4602864B475F032844A
:10E39D00C0F012E8E2CE2405CED0E075F00584C0C1
:10E3AD00F012E8E2CE2405CED0E023302D01040298
:10E3BD00E8E290A121028149070FFFFFC473BDAFB1
:10E3CD00A463B5FBCDE7FFFF030F0100FFFE038044
:10E3DD00306701227F3F7E00748812E8FCE55160B2
:10E3ED00F212187A85BCF01207A512E33D75F064A0
:10E3FD0084F87E06E5F012E7FDE860D77E0002E8BE
:10E40D00E912187AE5BE70012214600814603BE52C
:10E41D003F1340367F367E00747712E8FC2073017F
:10E42D002279BC8704098703125D3E7E05781DE6BF
:10E43D0060097E0012E8E2EE2405FE18E660071280
:10E44D00E8E2EE2405FE18E6801990B8B57F377E18
:10E45D000012817CAB60AC61125D411F7E09781D9D
:10E46D00E6600712E8E2EE2405FE18E612E8E2EE99
:03E47D002405FE75
:10E4800018E602E8E2202C012290E48F02E9280538
:10E490000EFFF0E01CF004F81CFFF0301201227FA8
:10E4A000637E0090B74612E9287F1512DD837F1F37
:10E4B00012DD837F2912DD837F177E06E53F30E082
:10E4C0000B90C0CE305C0390C0E2800990C0C33096
:10E4D0005D0390C0D81281497F2190B772207406E5
:10E4E00090B766028137E53770F9E53F20E0F430F8
:10E4F00073F190B77E1281377E1BAC4EAB4D12E6A6
:04E50000C302E74724
:10E66A00125D3E7F207E05751900781DC2D5E63001
:10E67A00D51712E8E2EE2405FE18B818F17E1F74C9
:10E68A0063305C02748202E8FC7005B8191880E2F3
:10E69A00D2D5CE24FACE7484301702742D12E8FC37
:10E6AA00EE2406FE80C8742012E8F880C8781C8020
:10E6BA000D7F007E23AC5EAB7A125D3E781DC2D51B
:10E6CA00E630D50C12E8E9EE2406FE18B818F12255
:10E6DA007005B8191680EDD2D53017E4CE24FACEDB
:10E6EA00742D12E8FCEE2406FE80D5742012E8FC94
:10E6FA0080D5125D3E781DC2D5E630D51612E8B730
:10E70A00EE2404FE18B818F10E745E305C02742709
:10E71A0002E8C67005B8191680E3D2D53017DACEEA
:10E72A0024FCCE742D12E8CAEE2404FE80CB742099
:10E73A0012E8CA80CBC23D12E7520F0F0E0E746365
:10E74A00305C02748202E8FC125D3E781DC2D5E696
:10E75A0030D50C12E917EE2408FE18B818F1227009
:10E76A0005B8191680EDD2D5301716740BCE24F8D9
:10E77A00CE12E917EE2408FE80D5740C12E9178030
:08E78A00D5303DCB740A80E597
:10EC4A007F797E24E55F30E70122AC5F1CAB7B1243
:10EC5A005D6CE51B700E742012E8FCEE2405FE12B2
:10EC6A00EC98800C12EC98E51B12E8E2EE2405FE03
:10EC7A00E51A12E8E2EE2405FE742C12E8FC0E0EE8
:10EC8A00E51912E8E2EE2405FE745E02E8FC742D32
:10EC9A00201702742B12E8FCEE2406FE22E55F30F0
:10ECAA00E70122AC5F1CAB7B125D6CE51B700E7436
:10ECBA002012E8CAEE2404FE12ECF1800C12ECF1E8
:10ECCA00E51B12E8B7EE2404FEE51A12E8B7EE24B3
:10ECDA0004FE742C12E8CA0E0EE51912E8B7EE24E7
:10ECEA0004FE742A02E8CA742D201702742B12E853
:06ECFA00CAEE2404FE2214
:10E504007F097E2530040512E5FE8028A275E57991
:10E51400C23D6002D23D92D175F080305C04F5F0CA
:10E524008001A4A2E792D5E5F075F03284F8E5F015
:10E5340075F00584C0E0E5F0A2D533C0E0E8602AB8
:10E5440012E917EE2408FED0E0F8D0E012E917EE45
:10E554002408FE0F0FE52B5403701F746012E8FCAF
:10E564001F1FEE2404FEE802E917740C303D067404
:10E574000A20D1010412E91780C9205904742E809D
:10E58400DC205804747F80D5748080D13004051257
:10E59400E5FE8028A275E579C23D6002D23D92D1A4
:10E5A40075F080305C04F5F08001A4A2E792D5E513
:10E5B400F075F03284F8E5F075F00584C0E0E5F01C
:10E5C400A2D533C0E07F3E7E1CE8602012E978D0FB
:10E5D400E0F8D0E07F3E7E2812E9787F447E3274F2
:10E5E4002E12E8FC7F3E7E37E802E978303DE07485
:10E5F4000A20D1010412E97880D59005CAE075F0AB
:10E604000A84F8E4C5F0C2D522301105E54AB40203
:10E6140050C39006E9E0957AFB9006E8E0955EFC2D
:06E62400500312602FEC10
:10E62A00C31360047B63800FEB13FB249C40F52427
:10E63A004F4004C20480079005CAEBF0D20490064A
:10E64A00E6E09006E8F09006E7E09006E9F0E55E7D
:10E65A009006E6F0E57A9006E7F02212E64880DEB8
:10DEAC00E54424F64001227800E552206607C3952C
:10DEBC0070500224B40475F00384F9E928FE24C4DC
:10DECC005001FE12DEEE12DEFA1E12F22DC3E9989C
:10DEDC00FE5003243CFE12DEEE1E12F22D08B81F7B
:10DEEC00DA22EE2420FE24C250032402FE22E8246F
:10DEFC00F1E8C2D55006D2D5E8F4241F23FF90DFF9
:10DF0C007C93CF0493FAE545F5F0A4ACF0FB125DDD
:10DF1C00CDE544F5F0A49BFBE5F09CFCEB2420FB49
:10DF2C00EC3400FC12DF5DFAE5458FF0A430E7021B
:10DF3C0005F0E5F020D502F4042A75F0052019034C
:10DF4C0075F00384FF24DF50027F20C374329FFFDF
:10DF5C0022EC24F0500BEB2460EC340090DFCC93DB
:10DF6C0022EB33FBEC33FCEB33EC3390DF9C932252
:10DF7C00FF00FF03FA0BF318EA2ADE40CF58BE73FA
:10DF8C00AB8D96A880C068D64FE835F51BFD00FF19
:10DF9C0000080B0E101214151718191B1C1D1E1F30
:10DFAC0020212223242526262728292A2A2B2C2DFA
:10DFBC002D2E2F2F30313132333334343536363732
:10DFCC00373839393A3A3B3B3C3C3D3D3E3E3F3F8E
:10DFDC004042444648494B4D4E5052535556585961
:10DFEC005B5C5D5F60616364656668696A6B6D6EDE
:10DFFC006F7071727374767778797A7B7C7D7E7FA3
:10E00C00808182838485868788898A8B8B8C8D8E90
:10E01C008F9091929394949596979899999A9B9C9A
:10E02C009D9E9E9FA0A1A2A2A3A4A5A6A6A7A8A9B7
:10E03C00A9AAABACACADAEAFAFB0B1B1B2B3B4B4E6
:10E04C00B5B6B6B7B8B9B9BABBBBBCBDBDBEBFBF20
:10E05C00C0C1C1C2C3C3C4C5C5C6C7C7C8C8C9CA65
:10E06C00CACBCCCCCDCECECFCFD0D1D1D2D2D3D4B3
:10E07C00D4D5D5D6D7D7D8D8D9DADADBDBDCDDDD09
:10E08C00DEDEDFDFE0E1E1E2E2E3E3E4E5E5E6E664
:10E09C00E7E7E8E8E9EAEAEBEBECECEDEDEEEEEFC6
:10E0AC00EFF0F1F1F2F2F3F3F4F4F5F5F6F6F7F72D
:10E0BC00F8F8F9F9FAFAFBFBFCFCFDFDFEFEFFFF9C
:10E0CC00E54524FD400122E552206607C3957050BA
:10E0DC000224B40475F00384241FFE24C2500324CC
:01E0EC000231
:10E0ED00FE12DDE7EEFD241EFE24C250032402FEC7
:10E0FD0012DDE7E544240275F00520190375F003E0
:10E10D0084F4042432FF24EE500F12E11CAE051EE0
:0AE11D001E7C0512F22D0EDCFA2222
:10E9B7007E00206615E5700475F0B484E5F075F007
:10E9C7000384FE6004C3743C9EFE745312E9E27430
:10E9D7005712E9E2744E12E9E274457F2F12E8CA32
:10E9E700BE00077E3C12E8CA7E00EE240875F03CA4
:10E9F70084AEF00F0F0F12F22D0E12F22D0F12F23E
:10EA07002D1E12F22DEE240775F03C84AEF0223055
:10EA1700745C301259E54AB4040122B4060122E5B8
:10EA27007112DF468F057C037E1E30662AE570046F
:10EA370075F00384241EFE24C6501C24FB500424B6
:10EA4700038013C00612EA5ED0E024C67C0160068C
:10EA57000C1460020C14FE12EA6A0EEE24C1400286
:10EA6700DCF5228D0712F22D0FEF24CE50F722E5A9
:10EA770053206607C39570500224B40475F00384CD
:10EA8700241FFE24C250032402FE12EA950E7F23A0
:08EA970012F22D0FBF2DF92230
:10F28D007E0E78ADE612E7FDEE2405FE742C12E835
:10F29D00FC0E0E0E18E612E7FDEE2405FE742C1280
:0AF2AD00E8FC0E0E0E18E602E7FD65
:10E127007F017E00745212E8FC7E06E51512E803B3
:10E137007F0A7E0178B8E67D0130E5027D03ED12A6
:10E14700E8E97E07E67D58A2E4922B50027D46ED72
:10E1570012E8FC7F017E1812F28F7F0A7E1378AED9
:10E16700E612E792EE2406FE743A12E8FCEE240566
:10E17700FEE53E12E792EE2406FE743A12E8FCEE44
:10E187002405FEE53F02E7927F797E00E54012E72E
:10E19700FD7E0A743B12E8F87E0CE54102E7FD7F3D
:10E1A700797E16743B12E8F87E18E53F12E7FD7F8B
:10E1B700797E0078AEE612E7FD7E0A743B12E8F836
:10E1C7007E0CE53E02E7FD305EE52043E27F6D7E93
:10E1D7000078AEE612E7FD7E0A743B12E8F87E0C83
:10E1E700E53E12E7FD7F757E00E53E75F00A84E5A2
:10E1F700F012E9170F0F7E08743A12E8F81F1F7E16
:10E207000DE53F75F00A84C0F012E917EE2408FE09
:10E21700D0E002E917851C1E851B1FAB1BAC1C3009
:10E227005D0A7A1B125DA47832125F46C3EB33FB9B
:10E23700EC33FC923D125D75303D087409F51DF510
:10E247001CF51B7F75E51D60157E2412E9177E2CD2
:02E25700E51CC4
:10E2590012E9177E34E51B12E917803D7E22E51C81
:10E26900601912E9177E2AE51B12E9177F787E31BA
:10E27900742E12E8F87F75E51A8019E51B12E91763
:10E289007F787E29742E12E8F87F757E2DE51A12A3
:10E29900E917E5197E3512E9177F777E3C12670584
:10E2A900851E1C851F1B227F397E1F12F22D0FBF71
:10E2B90040F9781F79567A007D1A12F0EA12F1F0C6
:10E2C900EA2406FABAAEF3781BC3E5119570500239
:10E2D90024B4FA604214603E14603A2450603A143F
:10E2E9006036EA24A540278A1E751D007D1912E3B0
:10E2F900020D30740312E3020D781F7956AA1DEA44
:10E3090012F0EA12F1F00AD3EA951E40F2228A1DB0
:10E31900751EB380D7080808087F367E1C90EC3636
:10E32900E571700390EC4012E9287F3CAE00908FB4
:04E339009602E92837
:10EE5E00787512EEAE7453201702744E207406E5C8
:10EE6E002E54074430AF1712EED87E3BE57DC454C6
:10EE7E000F12E8E92074077E07742012E8FC7878F8
:10EE8E0012EEAEE5172409FF7457201702744520C1
:10EE9E007402742012EED87E3BE57D540F02E8E931
:10EEAE00E6FD339217188604188603301703126096
:10EEBE003779177870125F418B13AF06AED27C0094
:10EECE007D64125EAF8F148D15227E0012E8FC7EDB
:10EEDE0007E51312E7AF7E19748112E8FC7E20E578
:10EEEE001412E7927E2B742E2073030E742C12E8EC
:08EEFE00FC7E2FE51502E792EE
:10F07A00E54A602E7A2420E00E7A26141460087A73
:10F08A0028141460027A297F667E01EA12E8FC20BD
:10F09A005505205406800B745B8002745C7E001256
:10F0AA00E8FC20110778A9B60007802130261EC285
:10F0BA002690B80D7F661281377F64A85AE54AB454
:10F0CA00060108E875F06484E5F012E20A20080FE8
:10F0DA00E537640260097F367E2E744112E8CA223F
:10ED000020144F740512F2FEEF33EE33F9EF0303D4
:10ED1000541FF5F090ED53E993A4C5F013C5F0131B
:10ED2000C5F013C5F013C5F0135403FCE5F013FB55
:10ED3000E9242093C9244093C39BC4540FFBE99C4E
:10ED4000C4FC540FF9EC54F02B2446F57BE934F65F
:10ED5000F55F22FFFFFFFFFFE6C5AD9C8F857D7746
:10ED6000726E6C6A696A6A6C6F747A828D9DB4D9AE
:10ED7000FFFFFFFAE9DCD3CEC9C6C3C0BEBBB9B73B
:10ED8000B5B4B2B0AFADABAAA8A6A4A2A09E9C9900
:10ED900096918C00381CE735D137246F00C5B3C17C
:10EDA000E61F66B60E68C21867AADBF4EDB94675B1
:03EDB00010A200AE
:10F2DE00D2A27408D2A1D2A300C2A3C2A1D2A3000B
:10F2EE00C2A3D5E0EF7405D2A300C2A3D5E0F822E5
:10F2B700C2A3D2A2D2A1D2A300C2A375F0083392EF
:10F2C700A1D2A300C2A3D5F0F5C2A175F003D2A3C2
:07F2D70000C2A3D5F0F822EC
:10D7F00012F2B7D2A300C2A3C2A175F008E4D2A36B
:10D8000000C2A3A2A233D5F0F5FE75F008E4D2A3BE
:10D8100000C2A3A2A233D5F0F5FFD2A300C2A32277
:10D82000E478806608B88BFB70012274D512D7F0BB
:10D830007881C3EE13FEEF13F692D118EE2460F652
:10D8400074D612D7F07888EF33CE33CE33CE33CEC2
:10D8500033A2D192E25407FCEEFB7A08125D96ECFB
:10D86000244FF608EBF674D912D7F0EF543F7882C4
:10D87000F67886EF33CE33CE33CE33CE335403F641
:10D8800008EEF618161608E6C4FF54F0F618E6C4BB
:10D89000CF540F2FF674DA12D7F0EF232354FC780D
:10D8A00083F67884EEF608EF54C0F67880E46608D4
:10D8B000B88AFBF62212D7F87889C3EF96FF18EEE4
:08D8C00096FEA2E7921650103B
:10D8C80012601F740FF8F9125DE3EF2CFFEE3DFEB6
:10D8D800788BEEF608EFF622E6182016072CF7E606
:10D8E8003D19F722C39CF7E69D80F66A405E805694
:10D8F800E050F04B0044803DC0384031D02BA0258B
:10D90800601F2018D014000F000AA001440158011C
:10D91800680178018801A001B401D001EC0210026D
:10D9280038026802A002DA030C034D78BE80208515
:10D938008E8A9D8F4D95BA9A97A0BEA631AC53B2E8
:10D948002AB801BD6AC1EDC4D1C78812D7F8788D4D
:10D95800EEF608EFF67887798C125DE37883799094
:10D9680012D8E07885798C125DE37881799212D8A3
:10D97800E0788DE624E4FE08E63392D13392D5545C
:10D98800FCFFEEA2D133A2D533FE780F7992125D57
:10D99800E378947990C3EC97F61819ED97F6799493
:10D9A80090D8F37F1F7D11EF93C3971F19EF9397BB
:10D9B8001F091DED600240EF0F90D913798DEF9389
:10D9C800F7090FEF93F7788E7994125DE390D933C6
:10D9D800EF93C39BFB1FEF939C2420FC7897E62BC7
:10D9E800F618E63CF618E436F6740612F2FEEEFC7B
:07D9F800EFFD740712F2FEBF
:10D9FF00C3ED9FFFEC9EFE78B7E6FD337C00500130
:10DA0F001CEF2DFFEE3CFE789CEF26F618EE36F657
:10DA1F002220140F789DE6B4050912DAC012DAF548
:10DA2F0012DB39222014577897799A12DB6A125F2A
:10DA3F00A7C3EE9420FE9245500312601F7C007D19
:10DA4F0005125EAF30450312601F8E618F60E531A6
:10DA5F00B40C2B12EE44E56120E71124F8500DFAB7
:10DA6F00C3E5609AF560E5619400F561121884E5ED
:10DA7F00BC2560F57AE5BD3561F55E12EE517897FC
:10DA8F00799AC3E697FB1819E697FC7A02125D960E
:10DA9F0012DAC012DAF520140312DB39789579986F
:10DAAF00E6F776000809E6F776000809E6F776004C
:10DABF0022799CE77700FB19E77700FC789DE6B4A5
:10DACF000506EB33FBEC33FCECA2E792D5500312C7
:10DADF00602F7A32125DA4ECFBEDFC30D50312609F
:0ADAEF002FECFEEBFF22EE2408FEF0
:10DAF9007406307511789DE6B40504740C8007F43A
:10DB09002406C323540FFD7C00125D82789FE6FC36
:10DB190008E6FBC374109DFA125DA4EFF8EEF91242
:10DB29005FA7E878A02FF6FF18EE39F62480FE22C9
:10DB39009275400312601F78BBE6F5F02438400364
:10DB490075F0E1EF33EE3378A8F6A485F07930E784
:10DB5900020579C276307508E57924F15002D2764A
:10DB690022E627FB1819E637FC1819E637FD227556
:10DB79006A0079C6876C09876B22756A2080F3125F
:10DB8900DB781298AB7F087871793A12DBA6029C90
:10DB99008A855E63857A62787379647F06E6F70819
:10DBA90009DFFA227864797380F1787379AF80EBB1
:0DDBB90078AF797380E5E6F008A3DFFA226B
:105D1C00E4FEFFFC7D0A791DE7540F2FFFE43EFEE5
:105D2C00B91902800619125D8280ED3017031260DA
:105D3C001F22305C2BEC339217500312602FEC2493
:105D4C00D950047C277B007AD2125DA4EB33CC3380
:105D5C00CD33CC33ED33FBEC33FC30170312602F17
:105D6C00EC339217500312602F7919125FBEF709AA
:105D7C00B91DF8A70322EFF88DF0A4FFEDC5F0CE06
:105D8C00A42EFEEC88F0A42EFE22EB8AF0A4FBE5F8
:105D9C00F0CC8AF0A42CFC22EB8AF0A4FBE5F0CC2E
:105DAC008AF0A42CFCE435F0FD22EB8AF0A4FBE590
:105DBC00F0CC8AF0A42CFCE435F0CD8AF0A42DFDB7
:105DCC0022EB8AF0A430E70205F0E5F0CC8AF0A4CF
:105DDC002CFBE435F0FC2286F0E7FDA4FAABF019BD
:065DEC00E786F0A42BFB8A
:105DF200E435F0FC18E68DF0A42BFBEC35F0FCE466
:105E020033FDE687F0A42CFCED35F0FD22EB89F0A2
:105E1200A4CBAEF08AF0A42EFEE5F03400FDEC89AE
:105E2200F0A42EFEE5F03DFDE433CC8AF0A42DFD76
:105E3200E5F03CCEFC22EB89F0A4CBAFF08AF0A4D3
:105E42002FFFE5F03400FEEC89F0A42FFFE5F03ED1
:105E5200FEE433CC8AF0A42EFEE5F03CFCED89F0A2
:105E6200A42EFEE5F03CFCE433CD8AF0A42CFCE544
:105E7200F03D8E058C068F04FF22C2D5EC30E7057B
:105E8200B2D5126027EE30E70DB2D512601F125E56
:105E9200AF1260278003125EAF30D50312601F225B
:105EA200C3EC13C0E0ED132FFFD0E03EFEBC000BAD
:105EB200BE0029EF8DF084FFADF022E4CCF975F03D
:045EC20008EF2FFFB7
:105EC600EE33FEEC33FCEE9DEC994005FCEE9DFEB8
:105ED6000FD5F0E9E4CEFD22EDF9F5F0EE8420D2FF
:105EE6001CFEADF075F008EF2FFFED33FD4007996E
:105EF6005006D5F0F222C399FD0FD5F0EA22EC3315
:105F0600EE3400FEEF3400FF7D007A007900780958
:105F1600C3ED9AFDEE9BFEEF9CFFB392D54009EDD3
:105F26002AFDEE3BFEEF3CFFA2D5E933F9ED33FD4A
:105F3600EE33FEEF33FFD8D92279007A00C38015FD
:105F460079007A00C3EA13FFE913FEE8132BFBEE90
:105F56003CFCEF3DFDE4F5D2F5D333FE7F19C3EEED
:105F660098FEE5D299F5D2E5D39AF5D3B392D5400A
:105F76000DEE28FEE5D239F5D2E5D33AF5D3A2D512
:025F8600EB33FB
:105F8800FBEC33FCED33FDDF0122EE33FEE5D233CB
:105F9800F5D2E5D333F5D380C3AD6FAC6EAB6DED01
:105FA800C454F0FEECC4FF540F2EFEEF54F0FFEB88
:105FB800C4540F2FFF22EC75F00A84FCEB54F02533
:105FC800F0C475F00A84C4CBC454F025F0C475F04D
:105FD8000A842BFBE5F022AC10AB11125FBEA904BA
:105FE800AD03FA7C197B99125D96AE04AF03EA758E
:105FF800F006A4F8AC12AB13125FBE2875F00A8441
:1060080085F014F8EF2BFFEE3CFEEF28FFE43EFE90
:10601800E43DFDE439FC22C3E49FFFE49EFE22E454
:10602800C39DFDE49CFC22C3E49BFBE49CFC22C3CF
:10603800E49BFBE49CFCE49DFD2275D4107B807AF4
:0C6048000079807800EAF5F0A4FCADF0CF
:10605400EBF5F0A4FEAFF0EB8AF0A4C333C5F03344
:10606400C5F092D52DFDC5F03EFEE430D501043FC8
:10607400FFB5150DEEB51409EDB51305ECB5120118
:10608400224006EA98FAEB99FBD5D40ABB00012218
:106094000ABA00010B22C3E913F9E813F8EA28FA53
:1060A400EB39FB80A478087B807D807C00EDF5F0E3
:1060B400A4FAE5F08EF0B5F007EA8FF0B5F001220E
:1060C4004003ED9BFDD827BDFF0122EDF5F0A4F9B7
:1060D400A8F0ED04F5F0A4C399FAE5F09813CA13F7
:1060E40029F9E83AF8C3E99FE89E50010D22C3EB71
:1060F40013FBED2BFD80B6C374689511FB740195F9
:1061040010FC8004AC10AB117A0B79B8125E0F80CE
:10611400177473F8F9E627FB0809E637FC0809E663
:0261240037FD45
:1061260030E703126037EB33FBEC33FCED3323FD32
:10613600242083F8ED241C83FFED241883FAED2434
:106146001483F9EF99F9E89AFA125E0FEF9DFFE8CA
:106156009EFE22FFFFFFB6FED7FD63FB5DF8C4F58A
:106166009BF1E3ED9EE8CFE379DD9ED743D06BC983
:1061760019C153B91CB079A7709E06943F8A237F34
:10618600B674FF6A045ECB535B47BB3BF130042316
:10619600FB17DE0BB2FF80C21DC232532CF8C3E5DB
:1061A600679576FBE5689577FCE5699578FD30E7B8
:1061B60005D26112603724F05003126271AA06A953
:1061C60007125E38EC2480E43DFBF9F51AE43EFC48
:1061D600FAF519E43F6002D232125E0F8B128C136D
:1061E6008D148E15C3E5649573FBE5659574FCE522
:1061F600669575FD30E705D262126037EBF9F51F3B
:10620600ECFAF51DED6002D23230320122125E0F39
:10621600EB2512F512EC3513F513ED3514F514EEE6
:106226003515F51540E102604212619D20323BEBC7
:10623600242E40D3EA2401CB3400FC7A07793D12A0
:106246005E0FC010C0118E108D118C128B13E4FCE2
:0E625600FD7E077FD012D384851203851302CC
:10626400D011D010BB0005BA0002D21D22B261C306
:1062740074809BFB74F59CFC74209DFD22204D6969
:10628400204866303F637F697E0112DD977E1F12CE
:10629400DE1275A7009004EDE0A2E792171392E7CF
:1062A400FC1582E013FB30170312602FBC003AEB9D
:1062B400603720E73420E63110E513201707C37454
:1062C4001F9BFE80027E1F12DE070EDBFA22FB20DC
:1062D40017097E00C374209BFB8008EB241FFE7407
:1062E400209BFB12DE010EDBFA2275A700758307E3
:1062F400E559C4440FF582E0A2E792522212DBB3BF
:106304001262EEC2E775F00A84FEAFF075A704537B
:1063140082F17864126377AE07786712637775A7A2
:1063240000E57DC4540FFEE57D540FFF78731263BE
:106334006BAE07787612636B74AF12611712622F1B
:106344008B148A131207D2ACCCAB017A0A125D9675
:10635400E5139B9004ECF0FBA3E5149CF0FCA2E78E
:10636400923DD23F02DBB9860308860408860518ED
:09637400188006E0FBE0FCE0FDEE
:10637D007A0A125DB620E70CEB2EF608E43CF6081F
:10638D00E43DF622C3EB9EF608EC9400F608ED947E
:10639D0000F622204D09204806C23F302A0522C2B0
:1063AD003380F6E54824F640F5E5580460F075A70E
:1063BD0000758307E559C42408F582E0FEA3E0FFCC
:1063CD001207D27437126463500B30381BC2387801
:1063DD00C5864680137432126463400C203809D28E
:1063ED003878C5A646754600740D126463404A128E
:1063FD006301303D38201122204D1F20481C2040C4
:10640D0019BCFF16EB24325011D24012185CE5BFB7
:10641D0075F019A4F536D22ED22F205238E55965D4
:10642D00586032204D2F20482CD23380282011095E
:10643D00204D06204803753600303319204D1220AB
:10644D00480F12AA000559C3E558955950038558B0
:10645D0059C233C2402229FBE435CCFCC3EB9FEC7F
:10646D009E22E558B4FF012285581175A704758346
:10647D0007E54824F65002805C201259202905209A
:10648D002A02805112DBB3E4F516F51775100012D0
:0C649D0064FBE510700312DBAD12651407
:1064A900302910E51B2517F517F51BE51C3516F5E1
:1064B90016F51C12652112DBAD0510C3E511951007
:1064C90050D175A70002DBB9E55AF51124F650033E
:1064D90075110A75A7047583067510001264FB12FD
:1064E90065141265210510C3E511951050EE75A7C5
:1064F9000022E510C4F582E0E0F564E0F565E0F519
:1065090066E0F567E0F568E0F5692275A7011269AB
:106519000D124AE775A70422E9F0E51CF0E51BF026
:1065290022E510C454F0F582E0F512E5822406F55F
:1065390082E0F511E0F51CE0F51B22E512B4261501
:106549007F757E34740D12E91720442575110012E8
:10655900E2B00266727F6D7E3BE012E8FCE5137ED5
:106569003512E8FCE5127E2F12E8FC20440312E202
:10657900B012E21C026672202852E558B4FF0122CB
:1065890075A704758307E559F51030330965586017
:1065990005204802051012652AE0F513305E072030
:1065A9004304E5376095E07F797E3D12E8CAE5133B
:1065B9007E3912E8CAE5127E3512E8CA30480B7FE7
:1065C9007F7E3512F22D0EBE40F98039201201224C
:1065D90075A704758306855B1012652A305E0A204B
:0265E900430766
:1065EB00E5377003026794E512700B7E3A7F79747E
:1065FB005D12E8FC800D75F06484E5F07E397F7ADE
:10660B0012E84AE537B4020512A8988045B4030294
:10661B008040E51C7006E51B24FB5036E511F96440
:10662B00B4602F20062CE537600D200C0AC3E995CA
:10663B0070F9500324B4F9E912F0EA781D79547D0E
:10664B001D90EC28E53F20E00390EC2F12F1F012A7
:10665B00E92875177975161930280375161DE5127B
:10666B00642660031266B575A7009006E3E511F08A
:10667B00A3121875E5BC75F01970040475F014A419
:10668B00951BFBE5F0951CFC9224500312602FEC3C
:10669B00F0A3EBF0C24FC263EC700EEB24E64002AA
:1066AB00D24FEB24C84002D26322E51C24ED402BD1
:1066BB00AE1CAF1B1268D77C007D32125EAFC005DB
:1066CB00EFAF17AE1612E803CE2405CE742C12E8EA
:1066DB00FC0E0ED0E02312E7FD801B1268CE126772
:1066EB000FCE2405CE742C12E8FCCE2402CEE87516
:1066FB00F0058412E8E2CE2404CE7422305D0274DD
:0D670B008302E8F8EE243D50047EC37F4B6E
:106718007C017DF4125EAFC004C005EF6007AF17BF
:10672800AE1612E803D007D0067C007D32125EAFA9
:10673800A805EFAF17AE16CE240ACE02E8E212681B
:10674800CEEE2450305D03EE24A150047EC37F4B6F
:106758007C017DF4125EAFC004C005EF6007AF177F
:106768007E2F12E850D007D0067C007D32125EAF33
:10677800C005EFAF177E3712E8B77E3B742C12E8DE
:10678800CA7E3DD0E075F0058402E8B77F6D7E2FA4
:10679800746312E8FCE51275F06484E5F07E351246
:1067A800E79212E2B002E21C30480320740122E4AE
:1067B800FCF5A79006E3E0F9A3E0FE24FE40EFA372
:1067C800E0FF7D78E5376008304FE3200C2A800B26
:1067D800121861E5BD20E010304F0DD206E5712496
:1067E800FE50151268C480107D3CE546600A7D1491
:1067F8001460057D0A1470B68911125D827D6F12CE
:106808005EA2BE00A9EF24E240A4AD07E51112F094
:10681800EA202404B2D5B2D1781F795612F1F0A833
:1068280006A907E511242D75F0B484E5F012F0EA05
:106838007407304F02740EFDFA12F1F0B2D5B2D1DE
:0768480012F1F0B2D5B2D14C
:10684F00DDF0AD0212F1F0850616850717B2D5B24D
:10685F00D112F1F085061E85071F7A03304F027A99
:10686F0006E511241675F0B484E5F012F0EAA816C7
:10687F00A917AD0212F1F0DDFBE51124EA40022465
:10688F00B412F0EAA81EA91FAD0212F1F0DDFBE56C
:10689F00377021304F1E90C186305D0390C1827FCB
:1068AF003C7E3312817C121861E5BD20E00612DEBA
:1068BF001812EBC722C3E99570500224B4F922E5F0
:1068CF001B2402FFE4351CFE305D1ABEC305BF4D0D
:1068DF00028012AC06AB077A1B125DA47832125FEE
:1068EF0046AE04AF03227873796412611912622FD6
:1068FF00751CC3751B4B2032048B1C8A1B2212681C
:10690F00F530320122AC19AE1AA91DAF1FB900051F
:10691F00BC00028010C3E913F9EF13FFC3EC13FCA3
:10692F00EE13FE80E8BF29005006BE290050012259
:10693F00C3EF13FFC3EE13FE80EB3E7FE3E3E3E30E
:10694F00E3E3E3E3E3E37F3E0C1C3C7C7C1C1C1C79
:10695F001C1C1C1C7F7F3E7FE3E3E3070E1C38707B
:10696F00E0E3FFFF3E7FE3E3030F0E0F03E3E3E3F9
:10697F007F3E070F1F3F77E7E7FFFF070707070771
:10698F00FFFFE0E0E0FEFF030303E3E37F3E1E3F74
:10699F0073E0E0E0FEFFE3E3E3E37F3EFFFFE3E3CB
:1069AF000303070E1C38383838383E7FE3E3E37FA4
:1069BF003E7FE3E3E3E37F3E3E7FE3E3E3E37F3FBB
:1069CF00030303E77E3C000000181818FFFF181898
:1069DF0018000000000000000000FFFF0000000092
:1069EF0000003FF00000381C38F00180C1F020F0AB
:1069FF00FC0038F03FE0000000007CC6C6C6C6C6EB
:106A0F00C6C6C67C1838781818181818187E7CC691
:106A1F00C60C183060C0C6FE7CC6C6061C0606C66D
:106A2F00C67C0C1C3C6CCCFE0C0C0C0CFEC0C0C00D
:106A3F00FC0606C6C67C3C66C0C0C0FCC6C6C67C8B
:106A4F00FEC6C6060C18303030307CC6C6C67CC6B3
:106A5F00C6C6C67C7CC6C6C67E060606CC780000B7
:106A6F0018187E7E18180000000000007E7E0000BF
:106A7F00000000000000000000000000C6E2E2D2AB
:106A8F00D2CACAC6C6C20000000000000000000043
:106A9F008080A0C0A000304020C08080C0A0A00097
:106AAF000060A0600000A040A05098D090882050B7
:106ABF00A850888850A8502060806000000040E0F7
:106ACF00400000000000800000E000000000000017
:106ADF0040002040800040A0A0A04040C04040E0C7
:106AEF00C02020C0E0E0204020E02060A0E020E0B7
:106AFF00C02020C06080E0A0E0E020404040E0A047
:106B0F00E0A0E0E0A0E020C00040004000008000D6
:106B1F0080002060E0602000E000E00080C0E0C066
:106B2F0080E0E0E0E0E0000000000040A0E0A0A076
:106B3F00C0A0C0A0C040A080A040C0A0A0A0C0E046
:106B4F0080C080E0E080C080806080A0A060A0A0B6
:106B5F00E0A0A0E0404040E0202020A040A0A0C046
:106B6F00A0A080808080E0A0E0A0A0A0A0E0E0E056
:106B7F00A040A0A0A040C0A0C0808040A0A0C06046
:106B8F00C0A0C0A0A060804020C0E040404040A016
:106B9F00A0A0A060A0A0A0A040A0A0A0E0A0A0A046
:106BAF0040A0A0A0A0404040E0204080E02020A8CE
:0D6BBF0070202070A8202008F030D01000B9
:106BCC0000F0A8A8000000E00000009020487088A9
:106BDC0098984000E0E0E000A0E0E0E04060301079
:106BEC0030604040E0404060909090909060206019
:106BFC002020202070609010204080F060901020A9
:106C0C0010906010305090F01010F080E010109048
:106C1C0060609080E0909060F010202040404060D8
:106C2C0090906090906060909070109060C0E0F0D8
:106C3C00F8F0E0C0000000000000000000000000C0
:106C4C00000050605000707050000078807008F0A8
:106C5C0000F8888888F800C0C8102040981800C038
:106C6C00B098B0C000602040000000000090D8FC3C
:106C7C00D8900000246CFC6C24000020A870A82084
:106C8C0000002020F8202000000000000000800000
:106C9C000000F00000000000000000606000081020
:106CAC002040800070888888888870206020202090
:106CBC002070708808102040F8F810201008887098
:106CCC0010305090F81010F880F0080888703040A0
:106CDC0080F0888870F808102040404070888870D8
:106CEC008888707088887808106000606000606028
:106CFC000000008000008000002040F840200000D0
:106D0C0000F800F80000002010F81020007088082F
:106D1C00102000200000000000000070888888F817
:106D2C008888F08888F08888F070888080808870E7
:106D3C00E09088888890E0F88080F08080F8F88077
:106D4C0080F0808080708880B8888878888888F8FF
:106D5C008888887020202020207038101010109007
:106D6C00608890A0C0A09088808080808080F88807
:106D7C00D8A8A88888888888C8A89888887088889F
:106D8C0088888870F08888F080808070888888A8CF
:106D9C009068F08888F0A09088708880700888705F
:106DAC00F82020202020208888888888887088886F
:106DBC008888885020888888A8A8A850888850205F
:106DCC0050888888888850202020F808102040801F
:106DDC00F800CCAC9CACCC0000CCD4E4D4CC0004FB
:106DEC00781828C800FC40A040182020180000008B
:106DFC00000000F800000000A040A0500078888837
:106E0C009868708840308870200000F0A8A8A8A866
:106E1C007848484848788870888080887020A8888E
:106E2C0098A8C88888805048FC485080304C5C60DA
:106E3C0060603C00E0F0080808F88044485C484476
:106E4C0080F880808080808078484848484888B89E
:106E5C00A8A8E8A8A8B88888888888F8085000707E
:106E6C00888888708080F088888888F888888888E6
:106E7C008888F09090909090F0A8A8A8A8A8A8F85E
:106E8C00888888F808080850008888888878A8A816
:106E9C00A8A8A8F8080000000000000000000000EE
:106EAC0000000088888888E8A8E8A8A8A870A8A886
:106EBC00A80000000000000000000000000000001E
:106ECC0000000000000000000000000000000000B6
:106EDC006000606000600060006060205020000076
:106EEC0000005090B890D090886050500070705056
:106EFC00008820208870000080C0A090F8003048E6
:106F0C00B4B44830003048B4B44830FC0098D020B9
:106F1C0058C800F8E8D880D8E8F8404050F85040FD
:0F6F2C0040A0C0A000203828A0C0A01038101826
:0B00000002005E000000000000000095
:03000B0002AA70D6
:10000E00206E06859950D26E32D26F32854F82E5C0
:05001E00143200000097
:1000230010990DC298206909206DE085994FD26D12
:01003300329A
:1000340085D01285835085824FF51485158275838A
:1000440004E515242140020515E599F0D26D8512C9
:07005400D085508380C0003D
:03005B000237F376
:10AA63008530F0C5F065308530F060F722C0D0C086
:10AA7300E0C0F0C0A775A700C083C08275D0087579
:10AA83008A00300503758A7A758CEA0532E53270DF
:10AA93000215320530E530640A6026201520E531C1
:10AAA300B40C0BE530B4010612AF6912ED00E531C9
:10AAB300B4180BE530B4060612AF6912ED0002AC10
:10AAC3008DC2AFD2C075C07AD2AFF5300531E53152
:10AAD30064197043F53120152CC225C22C7D0A74EC
:10AAE3000412F2FEEF33EE339005CCF0EE24F54082
:10AAF300142402400E24014008202005DDE1023722
:10AB0300F3D225D22CE5A6600215A678B5E660013E
:10AB13001678B6E6600116302E0BE5367007C22FA5
:10AB2300C22E12AE4EE5367004C24B800215367843
:10AB3300A9E660011678D8E66001160535E535709B
:10AB4300021535E590307B0B30E008D278C27BC22A
:10AB530000801A307C0B30E108D279C27CC20180BC
:10AB63000C307D0930E206D27AC27DC202E5904400
:10AB7300F8F47003753500304A09E53324FA5003BD
:10AB8300753305E5336005153302AC32E590F454B3
:0EAB930007700302AC32A2E09200A2E1920130
:10ABA100A2E2920230100320143D75330820001BED
:10ABB10020100C2011098013E59030E10E8006E58C
:10ABC1003724FC40F3E543541FF53320100375A6E9
:10ABD100FF202E5D301004E536705620100C201138
:10ABE10009E53524F55003753304D21BD2A5D2A64D
:10ABF10012AE4E75B44075B24078D8E67002053495
:10AC010020272E20682B202928202A25A210721106
:10AC1100501FE52054076019E53424375004C24A17
:10AC2100800F2401400B200026200119D27D7534AC
:10AC3100C8201558E531702412F2DE74E812F2B71B
:10AC4100802A02AD91E53724FC40E6D27C80DF30DA
:10AC510011DFE53724FC40D9D27B80D275F0038423
:10AC6100E5F070DE12D8B574E812F2B7E531B4063A
:10AC71000512DA208016B40C0512DA33800EB412F4
:10AC81000512DA208006B4180312DA3320141B806F
:10AC91001990ACB5E532C4540F93FAE532540F6004
:10ACA100096A70061216ED12171CE59030E1153095
:10ACB100E2128016010204040404050506070708D0
:10ACC10009090A0020100820110520103C807D2070
:10ACD10027F82068F52029F2202AEFE534243040B6
:10ACE100E9240750E5600B205E088590F020F20210
:10ACF100740190AD0393D2A5201002C2A512AE3902
:10AD0100806FC8A08269554646202F12E536603C07
:09AD110024AA500AE53675F01978
:10AD1A0084E5F06040D2A6201002C2A6D2A5202F58
:10AD2A000C7418304B02746412AE39803BE53675E8
:10AD3A00F00C30480375F00684A2E0744640E974CA
:10AD4A003780E5E52B5403600C20100E301106E520
:10AD5A004A6402600512AE54800312ADA9101B08A2
:10AD6A00A25892A5A25992A675A700D082D083D0E4
:10AD7A00A7D0F0D0E0D0D020200C201009C5A670B2
:10AD8A00030237F3C5A632C218B40202D21812D986
:10AD9A005330180874E412F2B702AC6D02AC68784A
:10ADAA00A7E5B4600924E04005760002AE54E53414
:10ADBA00702920412220751F300D1CE57924CE40D0
:10ADCA00167AFFE5B110E7010A2325B3F5B3EA3590
:10ADDA00B4F5B4C313F5B2E660021622C241207577
:10ADEA00028077C246E579FF605820120424FD509C
:10ADFA0051206502C21CD265EF24B050027F4FEF8A
:10AE0A0090AF199375C70375C6FC75B90185BFF074
:10AE1A00A4E5F0F624F44002760C301C2DE5BEC3FE
:10AE2A009FF5F0A4E5F024E0400375F020E5F0C2B8
:10AE3A001C79AA770375B300F5B4C31375B100F58D
:0CAE4A00B222C26578A77680D24179AAB6
:10AE56007703D21CE4F5B3F5B4F5B1F5B222C265B9
:10AE660079A1E57924CE500DE720E7E27628301C5B
:10AE7600DD743C80BE7680E720E7D3E57997404DC8
:10AE8600C24679AAE7FAE5792323B4C500400274DD
:10AE9600C42437300E31F42437300D15F7BA0302C7
:10AEA600FA0AC39AF5B175B300EAF5B4C313F5B25D
:10AEB60022101C07D21C76C802AE3B763274FF20E5
:10AEC6000E02749B02AE3BC313247E80CC75C7036F
:10AED60075C6FB75B901E5BD6026C395795004C2F8
:10AEE60046801D78A720461B301C11E57975F008B1
:10AEF600A42432F6E5792324AA02AE397605D24691
:10AF060002AE54301C077614747802AE397696C2B7
:10AF16004680EDFFF3E8DDD3C9C0B8B0A9A29A9484
:10AF26008F8A85817D7975716E6B6865625F5C5904
:10AF36005653504E4C4A48464442403E3C3A3836B8
:10AF460034333231302F2E2D2C2B2A292827262533
:10AF560025242423232222212120201F1F1E1E1DDB
:10AF66001D1C1CD2B5C28EAE8DAA8DAF8BAB8BE4E9
:10AF7600F58DF58BD28E3014012278B6BE0007EF20
:10AF860024E24002800806E624EC5002761420678C
:10AF960005E624F64005E4FEFAFFFB7C007D0A1276
:10AFA6005D827C007D5E125EA28F51EE600375515C
:0FAFB600FFEAFC7A33125D96EBF5F0A4E5F0CBE1
:10AFC5008CF0A425E0C5F035E0CB92D525F05006F0
:10AFD5000BBB0002D2D530E7060BBB0002D2D5EC85
:10AFE500F5F0A42BFBE5F03400FC30D5010C78A678
:10AFF500E6C39BFF18E608F6EB18F618E69CFE1864
:10B00500E608F6EC18F6301401227A0050040A120C
:10B01500601F7C007D6E125EA28FF078A2E6A4FB15
:10B02500ACF0125FBEEBBA0002F404FAE4F8FFEAF2
:10B0350030E70118E57960062075031FF4042AF549
:10B0450079EF38D27520E70860037579FF02DB5C7C
:10B05500C2750470F5E579F40460EFF57980EE12B8
:10B06500185778BBA6BC121875E5BE78A2F624F66B
:10B075005007E4F5BEF61255F7120BF6E5BEF54896
:10B0850024F65008E4F5BEF5481255F7E5BFF5433B
:10B0950024F3503924F3403512186B78A1A6BCE58A
:10B0A500BF789DF61424FB50087403F6F5BF1255BE
:10B0B500F778B7A6BE121861E5BDA2E39266A2E4D1
:03B0C5009267038C
:10B0C8005403C253B40102D25322740DF5BFF543A1
:10B0D8001255F780C0E56A700CE56B5403700612D0
:10B0E80098BD12B14775F08412B17F787086F70861
:10B0F800B880FAD2B275F08812B16D782575F00073
:10B10800758002C2B275F7D7E4F5F70000E5F7D20B
:10B11800B220E705D5F0E9D8E72275F08412B17FAF
:10B128008DF7A4D2B280CE75F08412B17F75F0008D
:10B1380075F7FFD5F0FAD2B222756BEC756A007517
:10B148008002C2B275F78475F70075F70075F700CD
:10B15800780075F7FF75F7FF75F7FF75F7FFD8F2F9
:10B16800D2B275F08112B17FD2B2808F75F05312CE
:10B17800B16D808775F003758002C2B285F0F785DE
:10B188006CF7856BF7856AF72275F003758002C244
:10B19800B285F0F7856FF7856EF7856DF722125443
:10B1A8004775382490B1FE12320B12EFD502F15BCD
:10B1B8001254477D0E90B21512B1C87D1890B22373
:10B1C80074A012EFC174A212EFC1E4FEFF12EFC126
:10B1D800ED12EFC1E493A312EFC12FFFE43EFEDDB1
:10B1E800F3EE12EFC1EF12EFC174B012EFC174B3F6
:10B1F80012EFC102F16124505352463130302C30E5
:10B208002C35373630302C382C312C300088000063
:10B21800040000000000000000000081020101009D
:10B22800010101000101010001000100000001000D
:10B2380000E10075160375170312B27B204C01223A
:10B24800D517F6D2A47F8CDFFEC2A412F15312B137
:0FB25800A612B1B812F153D516DC12F3127F32E1
:10B267007E0690BF6912814912283F12F19B300078
:10B27700FD0237F3E4F5A79004DFF0D582FCF01266
:10B287005447D269D2ACE4F515F87903106DF7D8B5
:10B29700FBD9F9E4F515F8F97A05E515700FD8FA31
:10B2A700D9F8DAF6C2ACC269D24CD23D227800791D
:10B2B70007106DF9D8FBD9F99005FF7453F0753273
:10B2C70010C2ACC269C24CC23D7A0312B613103B1E
:10B2D700D388017A0312B629103BC9E89940C57A89
:10B2E7000112B6AE70BE7A0212B6AE70B77A03120A
:10B2F700B6AE70B07A0112B6137A4712B601303B78
:10B3070004D23D800B7A0512B63C12B68AB43024BB
:10B31700E49005DDF09005E5F09005D779BCF0F5F0
:10B327005DF7A309F0F55CF79005F27427F0A374B5
:10B337000FF08059D25712B64E9005DDF09005E513
:10B34700F012B64E75F00AA4FA20D1010812B67AA7
:10B357002A75F00AA4C5F09005F2F0A3E5F0F0E431
:10B36700FCFBFEC21712B68AB42D05D21712B68D92
:10B37700B42E02800512B5F2DEF330170312602FE8
:10B387009005D8EBF0F55C1582ECF0F55D7A0212CA
:02B39700B613EB
:10B399007A5312B601303B04D23D80647A0212B668
:10B3A9003C12B67A147006FA532EE080139005DE2B
:10B3B9007402F0D274C2737A05146004D2737A07E6
:10B3C9009005CEEAF09005DDE05407C52E54F82526
:10B3D9002EF52E7E0C7DE612B63AC2D512B65175FF
:10B3E90083058D82F00D30D504DEEF8002DEE8AEF4
:10B3F9005DAF5C207303E4FEFF79BCA70609A707CC
:10B409007A0312B6137A4D12B601303B05D23D02CA
:10B41900B52B12B64EF53D12B651F53E12B651C5D1
:10B429003F0475F03C84E5F0653F60069005FF74C4
:10B4390044F012B68AB4562D7A0612B63CC22DE4EF
:10B44900F571F5707E049005D9F0A3DEFC20571341
:10B45900F57D7E067973F709DEFC7E089005CFF04D
:10B46900A3DEFC8074B441A512B63AC23C7FCF1268
:10B47900B564C4F57D12B68AB43102D23C7FD312C9
:10B48900B564257DF57D12B63A12B5DE7AB9125D3D
:10B49900A4C0007864125F46D0009005D9ECF0A3EF
:10B4A900EBF0125FBE8B71EC60037571FF12B63A57
:10B4B90012B5DE9005DBECFEF0A3EBFFF07C007D1E
:04B4C90014125EAF4C
:10B4CD00C22DED24F150010F240A5002D22DBFB42C
:10B4DD00027F008F70C23C12B64EF53C24E0500244
:10B4ED00D23C12B651F53B24F35002D23C12B65168
:10B4FD00F53AE53D24E85002D23CE53E24C4500225
:10B50D00D23CE53F24C45002D23C303C02800F7542
:10B51D00A7049005DF793A7E06E7F009DEFB203DB2
:10B52D000320740C532EE0E49005CEF09005DEF070
:10B53D0075A7049005F4E561F0E560F0E55EF0E5D2
:10B54D007AF0E579F0E52EF0E55FF0E57BF0E55179
:10B55D00F075A700029C8A12B651303C0224647526
:10B56D00F03CA4ACF0FB12B6512BFBE43CFC7A642E
:10B57D00125DA40812B6512BFBE43CFCE43DFD1218
:10B58D00B67AF912B68AC21724AF5005D2171260D7
:10B59D0037BFCF358D758C748B73301703126037B1
:10B5AD007A0A125DB6EB29FBE43CFCE43DFD7E001E
:10B5BD003017041260371E7583058F82EEF0A3EDF0
:10B5CD00F0A3ECF0A3EBF0E9228D788C778B7680ED
:02B5DD00C9E4BF
:10B5DF00FCFBFE12B68DB42E02800512B5F2DEF31F
:10B5EF0012B68DCD7A0A125D96CD540F2BFBE43C2B
:10B5FF00FC22C23B080808758304888208E06A6051
:10B60F0002D23B22C23B7583047800888208B8E0DF
:10B61F000280EEE0B424F4DAF2227800888208B8CF
:10B62F00E00280DDE0B42AF4DAF2227A01758304B5
:10B63F00888208B8E60280C9E0B42CF1DAEF221252
:10B64F00B63A758304888208E0B42C04D2D5E4227C
:10B65F00540FFA08A3E0B42E04EAD2D122540FCA31
:10B66F0075F00AA42AC2D12212B63A7583048882D1
:10B67F0008E0B42E0308A3E0540F2212B63A7583E4
:10B68F0004888208E02212B69FC4FA12B69F2A22BB
:10B69F00888208E020E603540F225407240922125F
:10B6AF00B6137AE6753800888208E0B42A0612B617
:10B6BF00956538226238DAEF74462212547375A7F3
:10B6CF00009004007EE07D03E0A312EFC1B40A04F2
:09B6DF00DD028002DEF202F165D9
:10005E00D2B47581C075AF017590F878FFE4F6D80B
:10006E00FDF4F5A6D220D2C075C07A75F83075D7DA
:10007E005075AE1375AF017581D87590F875EFBCDC
:10008E0075FDFFC2B7D2A412F157C2A47450123834
:10009E0016758951D28C75A882D2BC12997B12F238
:1000AE00DE12D82B12B064C22012EDB31236C57F09
:1000BE00407E0190B6F112814912549112F15712FD
:1000CE00EF0612F19B12F1917C1412F161300003D4
:1000DE000237E3DCF512B1A612B1B812F15775A6CC
:1000EE00FF12B23B12B0641236C512F19B12F153DD
:1000FE0012F19178B5761E12EDB312D820C215C248
:10010E00141236C590B7397F78128137205E0A7F78
:10011E00767E1290B74612E9287F4012F28D7F4903
:10012E007E0912E165E53F20E00805A6E5A670020E
:10013E0015A67F5312DD8B7F577E0B12E6BF12E79B
:10014E00477F602073102074097E2BE52E54071212
:10015E00E8E97E17800E7E0BAC5DAB5C12E6C31237
:10016E00E7477E311281D37F697E1212EC4E302525
:10017E00087E1290EF6F12E928E5A60303543FFDA7
:10018E00FE0D7F7312F22D0F12F22D1EDDF478B5D7
:10019E00E57124F64002761E307419E6602B7F72EC
:1001AE007E16744012E8CA7E17E612E8507E1F745F
:0701BE005312E8CA12F19B85
:1001C50010000C10010C10020C12B23B02010502CA
:1001D50037E3023A3E8061E53524C85046E5902074
:1001E500E241D0E0D0E0120229027D9DE53524D21E
:1001F5005031E59020E22CD0E0D0E08038E5352480
:10020500D25020E59020E21BD0E0D0E012F312306E
:100215006B0B7F0912812E12562F128606120229A8
:100225000205702212F31290C0227F00128137124C
:10023500F19B02F15012F180C215C214C227C268A7
:1002450012F19175370190B8281227259002557340
:100255000200EF0221F0020A08022AD2020570020A
:1002650005AD027D9D02027002052212F1917537DE
:100275000790BBCD1227259002807302023D02082C
:100285001D02085702088B0202A102041102027026
:100295000202700202BF0202A60256FF12B23B80A2
:1002A5002A7F517E00747212E8F812289C40BC1215
:1002B500554312EDB312B06480B17F49A25E120BB3
:1002C500E1925E120C0080A31255F712F191753779
:1002D5000290BD9E1227259002E07302027002185B
:1002E500A202190702195B0219B00219F4021A03D6
:1002F500020341020377021DC70203017F5B121847
:100305009812187AA8BE12032512F19B1000081046
:10031500010710020780EF18180880EA88BE80A838
:100325005300037F5A7E0590BDF1E875F00BA425B7
:0E03350082F582E5F03583F5830281497F4031
:1003430012189812187AE5BCF8E87F3F7E3212E85B
:100353000912F19B10000810010D10021280EA1817
:10036300B84AE6787D80E208B87EDE784B80DA888A
:10037300BC0202CD12F3127F0F90C2151281371205
:10038300283F12F19BC214C21512F150751065106B
:1003930000DFE53170F9E5106465700D855E148545
:1003A3007A15E4F512F513800C78A8E51326F513F6
:1003B300E43512F5127F1E7E19E51012E7AFC3E58F
:1003C3007A9515F517E55E9514F5167F287E0BAC27
:1003D30016AB1712E6C312E74712F19B12F161D570
:1003E30010ADAB17E516FC30E70312602F7A0A79DC
:1003F30000125E0FA912A813125F48EBF510243800
:1004030040037510C81218578510BC0202CD12F3B1
:100413001290B7847F017E0912814990B78D7F0ABC
:100423007E091281497F1312DD8375170012186646
:10043300E5BC1204F1E5BD1204F1E5BE1204F1E5D9
:10044300BF1204F190B7DD7F5F7E06128149122847
:10045300DE12F19B7517001204D11000081001156C
:1004630010024880F20517E51724F75003751700AB
:1004730075100080E2E5176408701512186675BCE4
:100483000175BD2375BE4575BF671255F70204118B
:10049300E51012050312F19B1204B1051053100766
:0604A300E51724FE4003F2
:1004A90053100380AC020270A9BCAABDABBEACBF9D
:1004B900E5171304F8E640085407C42510C480045E
:1004C90054702510F60287EE7800E875F009A42427
:1004D90017FF7E3B7D20E8651770027D89ED12E8E4
:1004E900FC08B809E502F19BF8C41204F7E8120503
:1004F900037E030517E51702E8E9540775F009A417
:1005090090B7952582F58250020583E51775F009A4
:10051900A42417FF7E0C02814912F19175370890C6
:10052900BE97122725900532730200EC02054E0290
:10053900142F0212E2020D0F02568D0205477F3772
:100549001220CD80D47F0A121898120BF61220724D
:1005590012F19B10000810010510020680EFB25A33
:1005690080EB120C0080B2C26812F19175370590C8
:10057900B96A1227259005827302023D0283870218
:1005890083CC0285650205700205A60284A702854F
:100599000D0221B902057002219F020B127F2E1252
:1005A90020CD80C312F19175370690BA45122725DF
:1005B9009005BD7302023D0221F60222580222D1A2
:1005C90002239E0223D00224470206020205FB02EF
:1005D90024900225350205E17F64121861E5BDA268
:1005E900E7120BE1121861E5BD92E7F5BD1255F767
:1005F90080B27F491220CD80AB1207BE12383D125E
:05060900F31212281994
:10060E00E55804607790BB171206AB129FD512F116
:10061E009B10000810011310021C80F50559C3E54C
:10062E0058955950D575590080D01559E55930E770
:10063E00C985585980C4E559B40F02802FB51F02E1
:10064E00802A75F007A42408F51775162774B825A7
:10065E0059F9870012069912F19B100028100128F3
:10066E0010020280F574B82559F9A700E53524FA71
:10067E00508878C7A6481207B512F31212F19B12D2
:10068E00F1530205AD1880CC0880C9E875F005A4B9
:10069E0085F01CF51BC0001266B5D0002212A066B4
:1006AE00B4FF0122751000751FFF12A07DE51064C6
:1006BE000F60171206E2401274B82510F8E675F0B6
:1006CE0005A485F01CF51B1267460510C3E5589569
:1006DE001050D722121BABF8602E6404602AE81467
:1006EE00B51025F51F121875E5BC70060475F014CB
:1006FE00800375F019A485F01CF51B1267467E2247
:10070E0090C1B612817CD322C322E558B4FF0122D8
:10071E00751000E510640F602EE51075F007A42427
:10072E0009FF74B82510F8E612079F75F00A84C009
:10073E00F07E2012E8507E28742C12E8CAD0E07E9B
:01074E002A80
:10074F0012E8B712075F0510C3E558951050C32282
:10075F00121BABF8603964046035E8146510702F14
:10076F00121875E5BC12079FF8C313923D7E1C1239
:10077F00E8667E28742C12E8CAE4303D067405B88A
:10078F000001147E2A12E8B77E18742312E8CA22D9
:10079F00305D1275F036A42432FBE435F0FC125FA5
:1007AF00BE125FBEEB221207C712811CDFFB2212A3
:1007BF0007C71288FEDFFB2275C70375C6F078B82E
:1007CF007F042275C70375C6F375B901E5BFB54838
:1007DF0031E55924F1402BE55975F00484A9F02433
:1007EF00F0F5C675B901C5F0A9BC600CA9BD1460C0
:1007FF0007A9BE146002A9BFE975F005A4F985F039
:10080F00CC22121875A9BD75CC00221255F712F122
:10081F009175370390BC2E12272590082D73020275
:10082F0070020B2B021D1C020B40020B4B022117F7
:10083F00021DE0020C0C021E14021E5A0221660257
:10084F001D96021E9F1255F712F19175370490BC39
:10085F00F212272590086773020270020B5A020BDF
:10086F0065020857020B7B020B86021A1D020857FE
:10087F00020B95020B70020BAF1255F712F1917527
:10088F00370B90BD4312272590089B73020270020D
:0B089F001ACB021ACB02092102095FEC
:1008AA000208C20208E50221FC021B70021C3B027C
:1008BA001BE4021CCC020BC9121861E5BF1470C1FB
:1008CA007F2E1218981F121861E5BDA2E6120BE1DD
:1008DA00121861E5BD92E6F5BD80A37F371218981C
:1008EA0012185CA8BFE812091912F19B100008102F
:1008FA00010D10021280EE18B802EA780A80E608A2
:10090A00B80BE2780380DE12185C88BF0208887F81
:10091A00367E2CE802E7987F1C121898121861A8F4
:10092A00BE12095312F19B10000810010D10021497
:10093A0080EF18B800EB780B80E708E824F450E160
:10094A00780180DD88BE0208887F1B7E35E875F055
:10095A0005A402E7927F25121898121861A8BF12FF
:10096A00099112F19B10000810010D10021480EF7A
:10097A0018B800EB780980E708E824F650E1780116
:10098A0080DD88BF0208887F247E3BE802E8E912FE
:10099A001857E5BF75F03CA4ACF0FDE5BE75F0054F
:1009AA00A42DFDE5F03CFC121861E5BF1460367514
:1009BA00F005A485BEF0A42DFFE5F03CFE7C007D89
:1009CA003C125EAFC005EF75F01884E5F07F2D7E0E
:1009DA002412E7927E30743A12E8FC7E35D0E01297
:0709EA00E79202F19B7F2D53
:1009F1007E0590C1D8128149121861E5BDA2E67F3A
:100A01002D12206402F19B12F312122819120A14FA
:100A110002023D7F177E0290B8881281497F4C7E89
:100A21000290B89E128149AC5DAB5C7F577E041287
:100A3100E73F12188485BC6285BD63E56124F840F7
:100A41004490B8A87F37128137AE61AF607C017DD9
:100A51005E125EAFC3741F9FFAAC63AB62EC33925C
:100A610017500312602F125D96AB047C0030170300
:100A710012602F74F52BFB74033CFC125D6C7F3705
:100A81007E1512E6B790B8B57F697E0F128149E5F0
:100A910060240FFBE43561FCA25C923BD25C7E1EBC
:100AA10012E6C3A23B925C7E30742012E8FC7E36D3
:100AB100742012E8FCE5602562FBE5613563FC7F8B
:100AC100227E0412E73FE56245637016742E7E3A7A
:100AD10012E8FC12F19B10000D1001151002260204
:100AE1000A3C742080E81562E562B4FF0C1563804E
:100AF100080562E56270020563E53524F55003756A
:100B01003301020A3C1218848562BC8563BD02551B
:100B1100F77F637E00747212E8F812289C40087F08
:100B21006312812E1255FE02057012186BE5BCA2EC
:100B3100E77F0A120BE4E5BC92E7F5BC02081A7FD5
:030B41001CA20DE6
:100B4400120BE1920D80097F25A20E120BE1920E89
:100B5400120C0002081D7F0AA20F120BE1920F80F3
:100B64002A7F13A208120BE19208801F7F52A20C65
:100B7400120BE1920C80147F25A20B120BE1920B55
:100B840080097F2DA209120BE19209120C000208C0
:100B9400577F49121861E5BDA2E3120BE1121861F7
:100BA400E5BD92E39266F5BD0208547F5B121861BD
:100BB400E5BDA2E5120BE1121861E5BD92E5924391
:100BC400F5BD0208547F6D121861E5BDA2E0120B59
:100BD400E1121861E5BD92E0F5BD020888120BF63A
:100BE4008F1F9217121898AF1F1F7E39128E4BA2B7
:100BF400172212187085BC2B85BD2122121870850E
:100C04002BBC8521BD0255F712186B85BE12120C40
:100C14002112186B8512BE1255F702081D75A6FF26
:100C240012F31212AA63740712F2FE8FF074061202
:100C3400F2FEEF2512C395F0A2E7923D4010FD2489
:100C4400CD50027D32AC05C3743F9DFD800FF4048A
:100C5400FD24C850027D37AC0574402DFD7F401241
:100C6400DD837E1212F22D0EBE1EF91F303D020FDF
:100C74000FEF6D70EDE536700A753606EC2513F549
:0C0C8400148C13120C9F12F19B1000073F
:100C90001001083002072215128002051280827F9F
:100CA000377E28742E12E8FC7F347E21740A303D92
:100CB000010412E917E514FC249C50027C637F3484
:100CC0007E2DEC12E20A7F437E1E12E6BF7E00E517
:100CD0001212E8567F057E0290BCC61281497F6DD4
:100CE0007E0190BCD112817C7F747E0490BCE212A4
:100CF000817C02281990B8C07F1B7E101281491296
:100D0000F19B12F150C214C21512F180020522D2D9
:100D100014D215E4F56EF56D756F02751501751435
:100D200001754280D233120D8EE51565146005857C
:100D3000151480F0C24D12F31212847D90BE67121A
:100D4000817A129B0478B8E60460AA751000D24E2E
:100D50001211E9304D07C24D12F157C202C23310D1
:100D6000000810012910024880F3E5151460C7D26D
:100D7000D5129A05E56F24FE400430339222129B6F
:100D80000478B8E630E6EA30D5221515801E1299AF
:100D9000E5E56F24F25005129A058010129B047845
:100DA000B8E630E6E9C2D50460C7051530338722BE
:100DB000E53514601324BE5003020D052419509D1F
:100DC00012284D12F19B8095E4F511F512122819A5
:100DD000E511451070087F7B90BA2F12817A12E1DD
:070DE000271211C385111257
:100DE70012F19BE51110001310013410020280F379
:100DF700E53524E65056D24D020D366004151180B4
:100E070015E5107003020EDD151012F3121211E72B
:100E17007407F511F5127F42129C5DDFFB80A72452
:100E2700F940157479951775F00D8414D395114011
:100E3700B20511129C26808E203CA8303DA50510D6
:100E470012F3121211E7129C26020DC8783A797133
:100E570012DBA4854E63854D62120FBD756C7F75DD
:100E67006BE8756AA512F3121228F012E127121126
:100E7700361215EA12168A1216CA12F19B100008CA
:100E870010011810023780F5120F99E56B241840EE
:100E970005120FAC801C129C5D8017120FACE56B1E
:100EA7002414500BE56A24135005120F998003127E
:100EB7009C2EE53524F550AD75330180A8787179FE
:100EC7003A12DBA485634E85624D754C0012F3120E
:100ED7001211E7020DCD12290C12F19B100005101B
:100EE700010580F8020DCDC25312547312284D74B8
:100EF7004012F005747812EFB5746312EFB574679A
:100F070012EFB5742312EFA81231A6E51512EF946C
:100F170078B8E6C4540344400412EFB512EFDCE49A
:100F2700F51412994D129A53747012F005E51412C4
:100F3700EF9475A700900401E012EFA8A3E012EF69
:080F4700A8A3E012EFA8A3E04B
:100F4F0012EFA8A3E012EFA8A3E012EFA812EFDCB4
:100F5F007F7B7E1DE51412E86612F19B1002287547
:100F6F00A70090042275134275120F753800E01216
:100F7F00EF94A3D512F812EFDCD513EC0514303C27
:100F8F009C12303F12F161020DCD74F1256AF56AA2
:100F9F00E56B34FFF56BE56C34FFF56C22740F25B0
:100FAF006AF56AE4356BF56BE4356CF56C22756C9C
:100FBF007F756BE812B144E5104511C2306002D263
:100FCF0030303B028060303011E51112994D129A8A
:100FDF0048129A9890055B121123E51112994D1240
:100FEF009A86900411756AA512111C056B7FEF127A
:100FFF001125129A98900411056B756A9412111CA1
:10100F00056B7F6C12112512B1417F8312112512CE
:10101F009A7B129A86900400E020E60990041175DD
:10102F006A8312112322303011E51112994D129A51
:10103F0048129A981210D5121120E51112994D12DB
:10104F009A861210D5756AA5121120129A9812104D
:10105F00D5056B756A4A121120129A7B129A8690E7
:10106F000400E020E65D1210D5756AEF1211201210
:10107F009A981210D5056B756A94121120129A7BEB
:10108F00129A86900400E020E6391210D5056B7590
:10109F006A39121120129A981210D5756ADE7F22C2
:1010AF0090061012112512B1417F83121125129A49
:0B10BF007B129A86900400E020E608F7
:1010CA001210D5756A83804E02B14175A701900648
:1010DA001005A7900411AE838E16AF828F17E0F524
:1010EA00451212D5F5441212D5F5537C007D2D1206
:1010FA005EAFED6414600685168385178212176F3A
:10110A001260A905A7EDF0A305A7A3E58324FA5069
:10111A00C5227F0080059006107FA575F08412B164
:10112A007FE0F5F7A3DFFAD2B202B0FDC06FC06E5E
:10113A00C06D756F7F756EE8756D0012B191751788
:10114A00237E00D2D57B0579FF7A007C1520D50154
:10115A001CE4F5F7E4ADF71212B620320CB5010023
:10116A005001F9B502004001FADCE6C3EA9904FA33
:10117A00E904F5F0EA141445F07003E4F9FAAF0152
:10118A00EA600612F22D0FDAFADB0B10D506D2D579
:10119A007B0580027B030EBE40ADD2B27E087F245F
:1011AA0012F22D7F2812F22D7E3712F22D7F241291
:1011BA00F22DD06DD06ED06F22E51275F00DA4FF1E
:1011CA0074739FFF7E00742012E8CAE51175F00D52
:1011DA00A4FF74739FFF7E00743F02E8CAC24EE404
:0F11EA0012994D12E127751779121206203C0C4D
:1011F900203D09304EF4E53524FA50EE22751201EE
:10120900129A53C23D75A700900400E0F5F0A2E5DB
:10121900923BB4FF03D23C22E5176479600320F6C0
:10122900F490042275160475130FE5165401441041
:10123900F514E0FD303B2AF545C083C0821212D572
:10124900F5441212D5F55312176FAC06AB0712DF2E
:101259005DFDD082D083D5130875130F741E121249
:10126900D7AE161212B620320312F22DA3303B224A
:10127900E58324F8501C0512E51224FC401F129A3C
:1012890053900400E030E604D23C801190042275AA
:10129900130FD5149D0516E51624C0508D12F19B28
:1012A900E51724F3F51724EE4002D23D22C232EDB0
:1012B90004601624FC501224A350027D5FEDC42360
:1012C900541FFFC3E5179FFF22D23222740F2582D4
:1012D900F582E43583F583E022D22B12141FD21450
:1012E90012EDB312F3121228F912E15A1215111262
:1012F90013F5751604751500E530651360FA853028
:1013090013533203E53270F01216ED12173C05152E
:10131900E51524C45006751500129C3D301A0312B8
:10132900179DE539600912139112136312F19B7528
:0B133900A6FF10000810011810020AA7
:1013440080BB301AB81214E38009201AB012B23BE1
:101354001214B6808E1214E3C237C22B020522E5A2
:101364001570030215377F0A147001221470077E6A
:1013740024E53E02E7921470097E1378AEE602E794
:101384009222146001227E35E53F02E792ED24E1CA
:10139400400574769D801A24E2400EED941E337548
:1013A400F00384FC74589C800804C313FCC3744485
:1013B4009CFCAE167F7612F22DEFB5040B1FEF24C2
:1013C400ED500812F25D80F51F80EBE516FE20E07B
:1013D400147F2612F22D7F3512F22D7F4412F22D46
:1013E4007F5812F22D0516E51624C0500375160415
:1013F400227F24740812E8B57F33740612E8B57F9F
:1014040042740412E8B57F56740212E8B57F65741D
:101414000112E8B57F74740002E8B5D215C21AC28D
:101424001F12B23B1214BDE4029121C22BC214124A
:10143400141F75A6FF758AFC758CFFE4F532F53927
:10144400D205D23712EDB312F312129C3D12E15AB7
:101454001215111215841228F979197B1E123B17E3
:1014640079557B1E123B1779917B1E123B1779CD60
:0E1474007B13123B1710002210012F100221D3
:10148200301A11E53924F14008E532240340058081
:10149200EF12179DE532240250FA80981214E3806D
:1014A200DF201ADC12B23B1214B680D41214E3C24B
:1014B20037020522201A57D21AD21F12185C85BC95
:1014C2004C85BD4D85BE4EE54C700FE54D54037005
:1014D20009753910E4F5520291217401129A26809D
:1014E200E6301A2AC21AC21F12185C854CBC854DFE
:1014F200BD854EBE1255F7E4129121D214E54C700F
:1015020008E54D540370028003121801C214227FB1
:101512000A7E007401205A02740312E8E27E057406
:1015220058201A02742D12E8FC7E0B7446202B02FE
:10153200742012E8FCC3E4954DFB740E954EFC4BEF
:10154200F5177A46205A027A17125DA48C038D048D
:10155200302B0CC3EC13CB13CBC313FCEB13FB12DA
:101562005FBEC0E07F017E00EB12E8037E0AD0E09E
:1015720012E8E2E517700A7F2F7E1090BA061281F8
:1015820049227F197E0590BE841281491215EA759F
:10159200A7008552827583057E3F7C00E0B504007A
:1015A2004001FC1582E582B4FF037582B3DEEDECE7
:0E15B200230475F0038423FD249C50027D6306
:1015C000ED75F00A84C0F07F237E2512E9170F0F16
:1015D0007E2D742E12E8FC1F1F7E32D0E012E91718
:1015E0007F267E0590BE8F02817C7D057F3A12DDCD
:1015F00095EF240FFFDDF778087F387E01E812E8C9
:10160000B7EF240FFF1818B8FEF17F3D02DDF47527
:10161000A700F5827583057E3FE92B203D012B95C0
:10162000324031E0FAC374769AFF1582E582B4FF46
:10163000037582B3E0FAC374769AFD1216551582CB
:10164000E582B4FF037582B3E0FAC374769AFD12A3
:101650001655DEC522BE3F0122203D1712F22DC3D2
:10166000ED9F70012240060F12F22D80E81F12F24A
:101670002D80E212F25DC3ED9F70012240060F1231
:10168000F25D80EF1F12F25D80E912B17C1216A4A8
:10169000FD7E001216A4FFFC1216B38C050EBE4090
:1016A000F2D2B222E4F5F7E4E5F704C313FAC37407
:1016B000769A2212F22DC3ED9F70012240060F127E
:0D16C000F22D80EF1F12F22D80E9C3E56BC3
:1016CD0094E8FCAB6A7A08125D967D0078A5125FEE
:1016DD003FAE037F259016E802E92803052070F838
:1016ED0030B226758001C2B275F72475F700E4E5B6
:1016FD00F7F545F5F775F700E4E5F7F544F5F775FA
:10170D00F700E4E5F7F553D2B212176F0260A97531
:10171D00A700758305855282EDC313F00552E5527E
:10172D00244C5003755200E532B401037539007530
:10173D00A7007583048539820539E53924F05004F5
:10174D0075391022EDF0E5822410F582E545F0E5BE
:10175D00822410F582E544F0E5822410F582E553EC
:10176D00F022E54530E702F404F5F0A4AEF0FFE514
:10177D004430E702F404F5F0A42FFFEE35F0FEE55A
:10178D005330E702F404F5F0A42FFFEE35F0FE22FE
:10179D00E53924F0407904600122E54E24F2406FD2
:1017AD00240C506BE54C704CE54D54037046740899
:1017BD0030100104302B024410205A024420301FF7
:1017CD0004C21F444075A7009005CEF0A3783A7F60
:1017DD000612DBBF7F07301010786A7F0312DBBF64
:0F17ED0078707F1012DBBF7F1A9005CE12184262
:1017FC007422129A2675A700900400205A0F758245
:10180C0010121820758220121820758230121820A0
:10181C0075390022E54C240E40047D0F800F04FD29
:10182C0074109DFCAF04121842EC129A26AF0512EC
:10183C001842ED029A2674061299867402129A10B6
:10184C00E0F5F7A3DFFAD2B2029B3775C6F4803508
:10185C0075C6F5803075C6F6802B75C6F780267573
:10186C00C6F8802175C6F9801C75C6FA801775C636
:10187C00FB801275C6FC800D75C6FE800875C6FF10
:10188C00800375C6FD75C70375B9012274721F12EA
:10189C00E8F80F02F19B7F0A1218987E2A12B23BCD
:1018AC00121875A8BF1218D61000121001051002DC
:1018BC001580F508E824E750EC781880E818E83033
:1018CC00E7E3780080DF88BF805F7F097E0590C0EA
:1018DC0099B80C0390C0931281497E27E53D2824CA
:1018EC000C75F01884E5F012E7927E33743B12E825
:1018FC00FC7E35E53E12E79202F19B7F131218989D
:10190C00120BF6121938100008100105100217807E
:10191C00F2105C07205D0BD25C80E8105DE5D25DB7
:10192C0080E1D25C80DD852BBC0202CD205C1020D6
:10193C005D1890C0EC7F127E2312814902F19B90BE
:10194C00C100205DF090C0F380EB90C0F980E67F81
:01195C001C6E
:10195D00121898121870A8BF1219921000081001D1
:10196D001110021A80F2E824F250031880EA780D63
:10197D0080E6E824E740030880DE781980DAE8F590
:10198D00BFF54380A37F1B7E26E412E8E9E82323FD
:10199D00B464087E26740112E8E9E47E2E12E79203
:1019AD0002F19B7F2512189812187FA8BCE8121916
:1019BD00EB12F19B10000810010D10021F80EEE8D4
:1019CD0024E050E9188006E824CF40E10812187F82
:1019DD0088BC1255F7D21512EDB380D180157F2436
:1019ED007E3724E202E8037F2EA20A120BE1920A4F
:1019FD00120C000202D07F37121861E5BDA2E4126D
:101A0D000BE1121861E5BD92E49267F5BD0202CDBE
:101A1D007F367E00747212E8F80F7E16743F12E85E
:101A2D00CA12186BA8BD121A9612F19B100008105D
:101A3D00010510021080EFE824875004240A80026B
:101A4D0024E8F880E17F377E16742012E8CA7E2CD8
:101A5D00743F12E8CA121A9612F19B100008100179
:101A6D001410022080EF18B80904787880E7B87850
:101A7D00E478E780E008B87904780A80D8B8E8D52A
:101A8D00787980D188BD020854E82487923DE850CA
:071A9D000224917F367E3028
:101AA400C313923B12E8037E3CE4303B02740512FC
:101AB400E8E27E1A90BFE0303D0390BFE412814912
:101AC4007F3C7E3A02F22D7F127E00747212E8F897
:101AD4000F7E20743F12E8CA12185785BE1085BFC6
:101AE40011121B5210000810011110021B80F21574
:101AF40011E511B4FFEB75111780E60511E511240A
:101B0400E850DE75110080D9121B527F137E2074B9
:101B14002012E8CA7E31743F12E8CA12F19B100009
:101B24000810011110021B80DF1510E510B4FFD856
:101B340075100B80D30510E51024F450CB751000FC
:101B440080C61218578511BF8510BE0208887F12FF
:101B54007E24E51112E7927E30743A12E8FC7E3559
:101B6400E51075F005A412E79202F19B7F49121863
:101B740098121BABF853BF1F121BB11000081001C1
:101B84000D10021280F218B8FF02780480EA08B837
:101B94000502780080E212185788BD1255F7B80084
:101BA4000302088B021C3B121857E5BD227F487EB6
:101BB4000590BFFA128149E8601CB4040A7E0590BE
:101BC400BFEF128149800C90C0061281497E38E82B
:101BD40012E8E902F19B90C0017E2912814980F349
:101BE400121BAB601D640460197F5B121898120B02
:101BF400F6121C1612187010000B10010810020CBB
:0C1C040080EF02088B105FE9D25F80E5E2
:101C1000852BBC020888121BAB601F6404601B7F0D
:101C20005A7E0590BFFA1281497E2390C00A305F28
:101C30000390C01112814912F19B22121BAB700359
:101C400002088B7F527E11121898121875A8BC12C8
:101C50001C7B12187510000810010810020880EF94
:101C60001880EC0880E912187588BC1255F7121814
:101C70007FE875F005A4F5BD020888121BAB604B28
:101C8000E875F03270040475F028A4ADF0FC305D06
:101C900011ACF0FB7A8A125DA4EB30E7050CBC00B6
:101CA000010DAE05AF047C007D64125EAFC005EF90
:101CB0007F517E1A12E7AF7E2C742C12E8FCD0E024
:101CC0007E2F12E792124DBF12F19B227F641218F1
:101CD00098121875A8BD121CFD10000810010F10F5
:101CE000021680F218E824CD50EC783280E808E83B
:101CF00024CD50E2780080DE88BD0208887F63E84A
:101D000023C2E012E33D75F06484C0F07E2612E841
:101D1000E97E2C742C12E8FCD0E080A47F1312180A
:101D20009812186BE5BCA2E7923DC2E7F8E8121DD5
:101D30006012F19B10000810010D10021280EE18C5
:101D4000B800EA783280E608B833E2780180DEE84D
:091D5000A23D92E7F5BC79A1F770
:101D5900021E117F6380027F12547F305C01237E53
:101D69002875F06484E5F075F00A84C0F012E8E2A1
:101D79007E2D742C12E8FCD0E07E2F12E8E20F7E53
:101D89003590C106305C0390C16202817C7F641288
:101D9900189812187AA8BDE8121D5C12F19B100060
:101DA9000810010D10021280EE18B8FFEA780F80B2
:101DB900E608B810E2780080DE88BD02081A7F5272
:101DC900121898121875E5BE7F517E2C128EA0F557
:101DD900BE79A2F70202CD7F37121898121870A89F
:101DE900BC5300037F367E32E812E8E912F19B10FA
:101DF900000810010710020780E718180880E2E5BB
:101E0900BC54FC48F5BCF52B02081A7F49121898F6
:101E190012187FA8BE121E4B12F19B100008100168
:101E29001110021A80EFE8240AF8242450E778DB1D
:101E390080E3E824F6F8247F40DB788180D788BEE8
:101E490080C6E8F424DC75F00A847F487E3B02E80A
:101E5900E97F5212189812187FA8BF121E9212F128
:101E69009B10000810011110021A80EFE82408F8ED
:101E7900245750E778A880E3E824F8F824A040DB49
:101E8900786080D788BF021E11E8F424A923C47F93
:031E9900517E3B3C
:101E9C0002E8E9123948754A00D210C211D214D2A4
:101EAC007575791475340012F3127F007E0290BCA4
:101EBC009D128149904DE87F087E2612E928E52B7A
:101ECC0054030F7E3912E8E912283412E59012A758
:101EDC008B12F19B10000810011A10022480C520EF
:101EEC007504057980BE1579E579B4FF05C2757561
:101EFC00790180B02075EB1579E57970A7D27580E2
:101F0C00A3C210C21402081D121870E5BE7F097E10
:101F1C003A02E8E9121875A8BF1218D6120BF6127D
:101F2C001938A8BF12199212187FE5BC1219EB7F51
:101F3C002DA20A1220647F36A26712206412187A2E
:101F4C00E5BC7F3F7E3212E809A8BE1203251218A9
:101F5C0057E5BC7F487E3212E809121875E5BE7F42
:101F6C00517E2C02E8E9120BF67F1BA20D122064A5
:101F7C007F24A20E12206412186BE5BC121D607F28
:101F8C0009E5BCA2E7122064A8BF12215212187AEC
:101F9C00E5BD121D5CE52B54037F367E3212E8E959
:101FAC0012187FA8BF121E92A8BE121E4B121861E7
:101FBC00A8BC022197120BF67F09A20F1220647F96
:101FCC0012A208122064121861E5BDA2E37F481228
:101FDC002064E5BDA2E57F5A1220647F51A20C1249
:101FEC0020647F24A20B1220647F2DA2091220648E
:101FFC0012186BA8BD021A9612185785BE1085BF11
:01200C0011C2
:10200D00121B52121861A8BE120953A8BF120991D2
:10201D00120999121870E5BE7F3F7E3A12E8E91257
:10202D00185CA8BF120919121857A8BD121BB112BE
:10203D001875A8BC121C7B121870121C161218757C
:10204D00A8BD121CFD121861E5BDA2E07F6C8007D2
:10205D00120BF67F48A25E744E400274597E3A020E
:10206D00E8FC120BF67F097E347401205A027403CA
:10207D0012E8E97F36802E1287FA7F73128451128F
:10208D0088497F6C1284607F2D801A121861E5BD1E
:10209D00A2E77F63122064121870E5BE7F097E3AB5
:1020AD0012E8E97F481220C37E1E90BA20305303F8
:1020BD0090BA1B028149121861E5BDA2E19253222B
:1020CD001218981F1220B212F19B10000810010572
:1020DD0010020D80EFE5BDB2E1F5BD1255F780E4BC
:1020ED0022128018EBF516F5147F6C128460127FA6
:1020FD00FC7F647E23E51612E866C3E5169514F59C
:10210D00167F731284517F2D809B7F2E121898128B
:10211D00186BA8BFE824FA5002780312215212F16D
:10212D009B10000810010D10021280E818B800E491
:10213D00780580E008B806DC780180D8799DE8F74D
:10214D00F5BF02081A7F2D7E2C7420B80502742E5F
:10215D0012E8FC7E32E802E8E97F5B12189812184B
:01216D006110
:10216E00A8BCE812219712F19B10000810010D1067
:10217E00021280EE18B800EA780380E608B804E28E
:10218E00780180DE88BC02081A7F5A7E2CE802E8AD
:10219E00E9D26875480A12B23BD21412384B128932
:1021AE0025123FDDC26B12020280F3D214751501A7
:1021BE001287B475B901E5BC20E71C1288E475A638
:1021CE00FF12893112283F12F19B12825110000F1B
:1021DE00500512837980E70515E515242050D102AC
:1021EE00057012220202023D1222020205AD1222D7
:1021FE000202088B12220E1218708548BE0255F785
:10220E0012383D12385712646F12F31290BABED2C2
:10221E004912A002129FBB1227EF12F19B1000145D
:10222E0010010510021B80F50548E548640A70028E
:10223E00F54880CF1548E54864FF7003754809805E
:10224E00C2854849123857E5582212B23B12383D22
:10225E00854849C250E558B40F02D25012646F80BF
:10226E003AD22775480A12384B12646F12F31212C3
:10227E009F2590BFB020290390BFBB1228CBC26A06
:10228E00123FDD106A0280E1C22712878C85494811
:10229E00122664123857D22912646F12F31290B9B3
:1022AE00D412A00020500E1228B512F19B1000106F
:1022BE001001AE80F812283F12F19B10000280FB35
:1022CE000205AD12383DE55830E7137F1B90BF9BDA
:1022DE007E0512814912F19B12F1530205AD12389F
:0722EE005712646F85594986
:1022F50012F31212282990BFBB12A000129FC5121B
:10230500F19B10000810010A10020C80F5122369D8
:1023150080DB12237680D612F31212282990BACECA
:1023250012A000129FC5129FC912F19B1000081040
:10233500010A10020C80F512238280DB12239080A3
:10234500D612262A12385712646F12F31290BF0064
:1023550012A00012286E12F19B1000051002888051
:10236500F80205AD0559C3E558955950037559004F
:10237500221559E55964FF7003855859220549D33B
:10238500E5491495584003754900221549E5496406
:10239500FF700585584905492212383DE55830E753
:1023A500057F240222DB12385712646F12F3129054
:1023B500BAD912A0001228C012F19B10000A100110
:1023C5000280F81226D380DE0205AD12383DE558AD
:1023D50030E7057F2D0222DBC26B7559FF12646F52
:1023E50012F312122819E55930E70312283490BA6E
:1023F500EB12A000129FD512F19BE55820E70610BD
:10240500000810011110021B80F00559C3955950A1
:10241500CF7559FF80CA1559E55964FE70C28558B4
:102425005980BDE55920E711D26B75A70075830763
:10243500C4F582E0B2E7F080A7306B031226810273
:1024450005AD12383DE55830E7057F360222DB122F
:10245500385712646F12F31290BAF712A0001228BF
:092465009C40091226C81226FD54
:10246E001224740205AD121875E5BD75F00584F5DC
:10247E00BCF5BDF5BEF5BF1207C71255F705C6DF91
:10248E00F92212383DE55820E7087F5190BB010232
:10249E0022DE12F31290BFC612A00012283F12F1D4
:1024AE009B125457D2AC10001FE55830E7F8306D30
:1024BE00F51225CA7E207F00501390C01812817C21
:1024CE0012F19B12F15380CAC2AC0205AD1B8B13E5
:1024DE0090B9F012817C12F19BC26B7B007514B81F
:1024EE001226BD1288B31288655025A814E8243828
:1024FE004004A60105140BC3E5139B50E678B812F1
:10250E0026FF306B0312860612385712646F8082D4
:10251E001287FAE51660E6D26B128910C003128795
:10252E00CBD003A91580C412383DE55830E7057F9E
:10253E005A0222DB12385712646F12F31290BB0C40
:10254E0012A00012286312F19B10003510010280B8
:10255E00F875460512259250157F007E3574079545
:10256E004612E86612F19B12F153D546E7D390BF9F
:10257E00D1500390C01812A00012F19B12F153809B
:10258E00B30205AD12545712EFF4745212F00574E3
:10259E005412EFB5E5580475590012EFE31282009C
:1025AE00401612878C1288E4128251400B0559C3D3
:1025BE00E558955950ECC322C2ACD322125457D2CF
:0D25CE00AC12F02D204CF1B440F712F032A9
:1025DB00B4400312F032B452E2F53812F032B45474
:1025EB00DA12F032FA60D424EF40D012F032E53830
:1025FB0070C912F03212F0321281E57B007E0312A9
:10260B0082DC50102050B412F032204C03B440F74F
:10261B00DEED80A71288C30B1281E5DAE0C322122C
:10262B00270AE55924C8F88602E54924C8F99860B9
:10263B0013146010500F18E608F618E86970F7A726
:10264B00021226FD22E559640F60F91908E618F607
:10265B0008E86970F7A70280E812270A78C8C25009
:10266B00E6B4FF02800708B8D8F6D25022B8D702DA
:10267B00D250A615807C78B812270CE4F9F5A77513
:10268B008307E9C4F582E030E70AE924B8F8243877
:10269B00400276FF09C3E5589950E71226C878B86F
:1026AB0079C8E6B4FF028002F70908E8243850F233
:1026BB00804079B877FF09E9243850F82279C87738
:1026CB00FF09E9242850F82212270AC23D78D7B611
:1026DB00FF04A900D23D18B8C7F5203D0279D819DF
:0826EB0078C8B6FF0122C3E824
:1026F300995007C6C7C6081980F478C81227177FF0
:102703000412811CDFFB2278C81227177F0412886A
:10271300FEDFFB2275C703E54875F004A42480F5AA
:10272300C62212F312C23C12813BE5376053146098
:102733004D14604514603D14603514602D146025FC
:1027430014600E146010146012146035146011804C
:102753003012205D802B12206F80261220EE802104
:10276300122004801C1220988017122084801212D9
:102773001FC1800D121F728008121F208003121FB9
:102783001412F19B12F15712281912AE5AA81F08FE
:10279300E814C23BB51D02D23B75F007203C03751C
:1027A300F009A4FF7E00303C0C7420303B02743EE1
:1027B30012E8CA800A740B303B02740A12E8E2D8AA
:1027C300CF12F19BE51D10000810011010021880B4
:1027D300B9651F7003751DFF051D80AE7005851F4C
:1027E3001D80A7151D80A375F003A4227F7B7E00A7
:1027F30090BF1812817CE54824F640087E0A90BFFA
:102803007E12817C2212847D7E05745B12E8C67E73
:102813001D745C02E8C61228087E3490BF29028129
:102823007C12847D80031228087E3190BF2D0281A3
:042833007C122808E3
:102837007E3190C02302817C12847D7E00800C1241
:10284700847D7E18800512847D7E2D90C0230281B1
:102857007C1228637E3190BA2A02817C12283F7E3F
:102867001A90BA2F02817C12283F80B912283F7E26
:102877001890B9DD02817C12283F7E1A90C0280289
:10288700817C12847D7E0090B9DD12817C7E31903F
:10289700C02802817C12283F7E1A90C02D12817CAD
:1028A70012F19BD3100006C310010280F6221228F2
:1028B7003F7E1A90BAC802817C12283F7E1890BAD0
:1028C700E402817C7F007E2012817C02F19B1284CE
:1028D7007D90C03202817A12847D90C04302817A52
:1028E70012847D90BE4502817A12847D90BE560285
:1028F700817A1228467E2C90BE7E301A057E009083
:10290700BE7802817C12847D90BEDA02817A125FE2
:10291700A10FBF00010E8E04EF799AF7FB7F017EAE
:1029270028A25C924EC25C12E6FCA24E925C78B87A
:10293700E654F070091F7E2890BE40128149E4FFDB
:10294700FE78ADE612E7FD7E0A742C12E8FC7E0CD9
:1029570018E612E7FD7E16742C12E8FC7E1818E6BE
:1029670012E7FD303D0A90BE3A7F147E0112817C4A
:10297700227F097E0178AEE612E7927E0D743A1245
:10298700E8FC7E1278BDE612E7927F097E2378BEC7
:01299700E659
:1029980012E7987E30743A12E8FC7E3508E612E7B2
:1029A800920886040886037F127E0012E6C312E7A7
:1029B8004778C4E612E33D7E2912E7AF7E3B748B6D
:1029C800305D010402E8FC780C7F1C7E02E812E806
:1029D8004A7E09742E12E8CA7E0CE51012E84AEF06
:1029E8002405FF7E1E12F22D0EBE3FF9EF2403FFD1
:1029F800D8D922C3740C951375F008A4241CFF7E43
:102A080017742012E8CAC3740C951175F008A42431
:102A18001CFF7E17743F02E8CA751600AD6FAC6ED6
:102A2800AB6D7403129991E4F5F7A4E5F7F9540F27
:102A38006046E4F5F7A4E5F76510703CE4F5F7A403
:102A4800E5F775F008A47F80CF9FFFE4F5F7A4E5CC
:102A5800F7D2B2241DFE12F22DE954F0601A1F12AB
:102A6800F22DEE6516700DEF651770081F12F22D26
:102A78001F12F22D8E168F17D2B21299AFED30E7D2
:102A8800A122AD6FAC6EAB6D7403129991E4F5F7AA
:102A9800A4E5F7540F601DE4F5F7A4E5F765107099
:092AA80013E4F5F7A4E5F765114C
:102AB1007009D2B28D6F8C6E8B6D22D2B21299AF2A
:102AC100ED30E7CBD32278B97998E6F70809E6F734
:102AD10022D215C210C21112F312129AC6303C133F
:102AE10090B8B87F1C7E0512817C12F19B12F150C7
:102AF10002023DC221C24D1299F0E56F20E7E112B9
:102B01009B0479B8E7540F60EEE764FF60D279B9AE
:102B11008710098711302109799887100987118059
:102B21000A12F312122978C23D800512F312D23D26
:102B31001229151228191229CF12F19B122A218567
:102B410011131229FB85111312F19B7998A7100912
:102B5100A711E59030E20FC221304D24C24D12F190
:102B61005712F191801AE53524AA500302023AE581
:102B71003524C3500B90BE2D7F7312813712F19B08
:102B81002021C810000810011C10023780BDE5117A
:102B910014F51170AD75110C1510E510B407005046
:102BA1008A051080A679B9E76510700609E76511F5
:102BB1006099E51104F511640D7087751101051017
:102BC100022B2C122A8A501DC3740C951175F00822
:102BD100A4241BFF7E0290BE2312814912F19B1295
:102BE100F157022B2C129B04122AC7E59020E21008
:082BF100E53524DC500AD22175
:102BF900D24D129AC6022AF812F3121228E71229A4
:102C09001579B8E75403600312297812DB7879B88B
:102C1900E764C3701712DB7812321912DB8812329B
:102C2900FE756A101298ABD2331234BE12F19B10A2
:102C3900001710013279B8E764C370A4100202804A
:102C4900EEE53524FA4099807C1299F0129B04E54F
:102C59006F20E70A79B8E7540F60EEB7FF8212993F
:102C6900D2129B04022BE91299D2129B0479B8E77C
:102C7900540F60F3B7FFED80D012289C40517FC0FC
:102C8900129B221299A2129B4C60F8B4FFBB78C622
:102C9900866C08866B756A0012B1741298AB1218AB
:102CA9008EE56C65BD701BE56B65BC7015E57064E0
:102CB900FC700F78BEE66577700808E665787002E3
:102CC9008049022BE97995A76F09A76E09A76D7944
:102CD90095876F09876E09876D129B0412DB78123D
:102CE900DB881232FE756A101298ABC2331233B503
:102CF90090B8D1D23C12813B12278A902D087302D9
:102D09002BE9023F26022D90022C827F6C12812E24
:102D190012F153D2201299F0E56F30E70F1280B506
:102D29001255F71256D51256B7022AD2129B04121F
:102D390099D212188EACBFADBE85BDBF85BCBE7819
:102D4900C686BD0886BC1255F712B174E56C6C7065
:012D59000D6C
:102D5A00E56B6D700812B16A12B0FD801F12B12FB7
:102D6A00E56B54036403700612B16A12B0FD129740
:102D7A00FAE56B5403700312B17480CF7F00129B83
:102D8A0022C220022BE912F3127F6490C1FB128146
:102D9A00377F7990C20812813712F19B751600109D
:102DAA00000A10010910020280F505160516C25321
:102DBA0012DB8875370090B8ED122725902DCA735B
:102DCA00022CD8022DB8022FBD022FC2022DB80242
:102DDA002DF1022DF6022DB8022E34022E38022EC3
:102DEA003C022E43022E4712547380031254687811
:102DFA000A122F16740B12EFB3122F5E12EFDC12A7
:102E0A002F971298AB1299081297E0129C3D123034
:102E1A00A6D5150C75150A122FA71231CB12EFDCA5
:102E2A00100204E57F70DB022CD8780A8006780449
:102E3A00800278011254738009780A80027801129C
:102E4A005468122F16740B12EFA8122F5EE548125F
:102E5A00EF94E5165403443012EFB5742A12EFB515
:102E6A0012EFB512EFDC122F971298AB12990812D3
:102E7A0097E0129C3D1230A6D51548854815122FA9
:102E8A00A7E51C12EF94E51B12EF94E51B2548F504
:102E9A001BE4351CF51CE4A27792E7A27492E0A227
:102EAA007392E112EF94AD75AC74AB73E57DC41205
:102EBA002ED7AD78AC77AB76E57D122ED71231E9F5
:0A2ECA0012EFDC100204E57F709F98
:102ED400022CD8540F2375F00584F8C3EB33FBECB4
:102EE40033FCED33FDC3EB33FBEC33FCED33FD205E
:102EF400E713EB28FBE43CFCE43D12EF94EC12EF07
:102F040094EB02EF94C3EB98FBEC9400FCED94007B
:102F140080E8884812284D90BE1D12817A12F19BD8
:102F2400E4F54AF549756A207515011298AB1297B4
:102F3400E0D5150E854815E5492401F549E4354ADF
:102F4400F54AE57F70E5744012F005747812EFB528
:102F5400746312EFB5742302EFA81231A6799AE7CD
:102F640012EF9412DB88E53A12EFA8E53B12EFA8C2
:102F7400E53C12EFA8E53D12EFA8E53E12EFA8E507
:102F84003F12EFA8740112EF94E54A12EF94E54959
:102F940002EF9412DB83E4F51CF51BF514F51375AD
:102FA400150122753800E51412EF94E51312EF941D
:102FB4000513E5137002051422125473800312548E
:102FC4005D12284D12310012F15B756A20751501EE
:102FD40075A6FF754A0112984F1297E0129C3D1294
:102FE40030A6D5150975151E1230CA12F1651231B5
:102FF400CBE57912EF94E412EF94E57112308B1261
:09300400EF94E57012EF94E57BF6
:10300D0024ACFFE55F340912EF9AEF12EF94E5154A
:10301D0020E036857D56E412EF94E52EC412EF9A2A
:10302D0012EFEB12F16510020630559B12303F0284
:10303D002CD8744012EFB5744512EFB5744F12EFE2
:10304D00B5744612EFB502EFEBE556123065C4FAD2
:10305D00E57D1230652A80BFFBC41230722323CB6D
:10306D001230722B22540FFC24F650027C0090304B
:10307D0081EC932200000101010202030303FA24F3
:10308D0040400A24804003EA3322D2E72274FF2213
:10309D0020E703C3132224C022E53F701F7F7B7EF0
:1030AD000078AEE612E850EE2404FE743A12E8CA37
:1030BD00EE2404FEE53E12E84A12F19B22C015C033
:1030CD0016D212128FCFC212D016D01578AEE612CC
:1030DD00EFA8E53E12EFA8E53F12EFA8E54512EF88
:1030ED0094E55212EF94740A12EF9474C012EF9497
:1030FD0002EFEB744012EFB5745412F005744E12DA
:10310D00EFB5743012EFB5E5165403443012EFB538
:10311D001231A6742312EFA8E53D12EFA8799AE7B4
:10312D0012EF9412DB8878ABE60812EFA8E60812CE
:0D313D00EFA8E60812EFA8E612EFA8E53EA5
:10314A0012EFA81236ACE51212EFA8E51112EFA899
:10315A00740112EF9490C05412320B756A101298CF
:10316A00AB740212EF94E412EF94787B12EF8D782D
:10317A007D12EF8D787712EF8DE4FEFF780712EF5C
:10318A008D12EF8DE57412EF94E57512EF94E41247
:10319A00EF94E412EF9412EF8D02EFEB75C703750B
:1031AA00C6FF75B901C217751D0085BC1C85BD1BFC
:1031BA0085BE1A85BF19125D1CEE12EF94EF02EF5D
:1031CA0094E57512EF94E57412EF94E57312EF9497
:1031DA00E57812EF94E57712EF94E57612EF94E52D
:1031EA001664016011E55E12EF94E57A12EF94E538
:1031FA0016640260012278BCE612EF9408E602EF38
:10320A009475A700E493700122A312EFB580F5121A
:10321A00DB88857946787A796412DBA47464126152
:10322A00178E471232FE756A20D23D1298AB129958
:10323A0008123335303D09307406C23D8E1E8F1F89
:10324A00E57F602BE54C24FFF54CE54D34FFF54D49
:10325A00454C600512980180D2751D3C1298AB123C
:10326A0099081297E0123335E57F6003D51DED12F8
:10327A0033969033AE12E928203D0DAE1EAF1F12D1
:10328A0033969033A712E928E546FD700B90C18A60
:10329A00305D1190C186800C04700E90C186305D3D
:0632AA000390C1827F3891
:1032B000024DBAE4FFFC7E05305D047E027FB3124E
:1032C0005EA2AC06AB07125D6C7F38C23DE51C60A8
:1032D00007D23D7E2C12E8B7E51B203D026007D2E5
:1032E0003D7E3012E8B7E51A203D026007D23D7EF0
:1032F0003412E8B7E5197E3812E8B7024DBFE54051
:1033000075F03CA42541FFF54CE435F0FEF54D7C0D
:10331000007D10125EAF0F8F4BAF4CAE4D7C007D29
:103320003C125D827C00AD4B125EAFEE4F70010F20
:103330008F4C8E4D2278647973C2D112334CFF7852
:10334000677976D2D112334CFE02F22DC3E796FB99
:103350000809E796FC0809E796FDA2E792175003D3
:1033600012603775135A30D10E751320B217AA4761
:10337000125DB6AB04AC05E546600B04600BAA46D3
:10338000125DCDEB03FBEB03FBEB543FFBE5132B93
:103390002017029B9B22EE141430E701E4FEEF1489
:1033A0001430E701E4FF2205057088A88870050540
:1033B0002020F8202012F3127E1E7F1C12F22DDF37
:1033C000FB12F22D7E1E7F1C12F22DDEFB7E1D7F76
:0633D0001D12F22DDEFBD0
:1033D6007F007E2178ADE612E84A7E29742E12E837
:1033E600CA7E2D18E612E84A7E35742E12E8CA7E89
:1033F6003918E612E84A7F077E21745412E8CA7E1D
:1034060025744F12E8CA7E2D78AEE612E84A7E355C
:10341600743A12E8CA7E39E53E12E84A78AE1236A8
:10342600AC7F0E7E21744C12E8CA7E25744112E8E8
:10343600CA7E2DE51212E84A7E35743A12E8CA7E33
:1034460039E51112E84A7F157E25744412E8CA7ED2
:103456002DE54012E8507E35743A12E8CA7E39E509
:103466004112E84A7F217E0190C15512817C7E0E71
:10347600AC77AB7612E6FC7E2B85795F85787B127E
:10348600ECA77F287E0190C15912817C751D2B7592
:103496001E10E5741236607E25742F12E8CA751D5B
:1034A6002D751E2BE5751236607F367E0290C1455E
:1034B60012817CE57212364A12358E20330312369B
:1034C6003B12DB83AE4DAF4C7C007D40125EAFBF3E
:1034D60000010F0FAC07AD07E4FED23D1298AB1208
:1034E600990812352EE57F602CE54C24FFF54CE556
:1034F6004D34FFF54D454C600512980180DE751D73
:103506003C0E1298AB129908123533E57F6006120D
:1035160097E0D51DED7F783033027F3612DD951F9B
:083526001F7E00743002E8CAA8
:10352E00DD03AD040E7F783033027F36E55E20E793
:10353E002EE57A8549F0A4A9F0E57A854AF0A4290A
:10354E00F9E435F0FAE55E8549F0A429E435F02A70
:10355E00FAE55E854AF0A42A30330113CF9FFF129D
:10356E00F22D103D18C3EF9B50131BEF6B600E8FA7
:10357E00018B0712F22D1FEF6970F8AF01AB072216
:10358E0090C10A305C0390C123754A40754900AF63
:10359E0076E577FE20E76B7005EF24105064EF247C
:1035AE00A8EE34FD401190C10F305C0390C1277519
:1035BE004A1975499A8075EF2450EE34FB401190EC
:1035CE00C114305C0390C12C754A0C7549CD805CDA
:1035DE00EF24A0EE34F6401190C117305C0390C179
:1035EE0031754A067549668043EF24F0EE34F1409A
:1035FE001390C11A305C0390C136754A0475494464
:10360E00802A8028EF2490EE34E8401190C11D30BE
:10361E005C0390C13B754A0275498F800F90C120A3
:10362E00305C0390C140754A0175499A227F401261
:10363E00817A7F4612DD957F5F02DD957E2112E352
:10364E003D12E8667E2F90C15D305D0390C162022F
:0D365E00817CAE1E75F064305C0375F032A7
:10366B0084C0F0F87004EE2404FEE51D12E8CAEEE7
:10367B002404FEE8600712E8B7EE2404FED0E075E0
:10368B00F00A305C0375F00584A8F012E8B7EE245D
:10369B0004FE742C12E8CA0E0EE8305C012302E81B
:1036AB00B7E53E2541F51124C45003F511D3E6359A
:1036BB0040F51224E85002F5122212AE54C2101239
:1036CB00F3127F057E0990B6E81281497F127E06C0
:1036DB009036F512E9287F2B7E0190375D12E92891
:1036EB007F267E2A9037CF02E928113007FE1FE094
:1036FB0001E101F80F00061B00F80C00180E007C0E
:10370B0010007006003C2000E006003E4001E00483
:10371B00001E8003C004001F0003C000000F000741
:10372B008000000F800780000017800F000000272B
:10373B00C00F00000043C00F00000083E00F00200B
:10374B000301F00700C00F01F80383007F87FE0120
:10375B00FC000E3E180000030000000018000003E0
:10376B0000000000380000000000000030000000E6
:10377B0000000000FC761F0E1C6030ECFCBC3F17F9
:10378B002DF0F978613866264F619A706070C60E1D
:10379B001EE330E06060C60C1CC360C0E0618C0CA3
:1037AB0018C7C0C0C0E18C1C39C611C0C4C19C99DC
:1037BB0031963180C8C1FF1E31E7E180F0C0EE1CAD
:1037CB0031C38180061238E18034D340659640794D
:1037DB00E640C3448082230012F3127F3E7E179093
:1037EB00BF6512814912F19BD2A47F8CDFFEC2A46C
:1037FB00C2AFD2C075C0107581D874FE12381612C4
:10380B00F157E4F5F9F5FBC2B480F7D2A6C2A512C5
:10381B00AE3912F15702AE5A75C703E54875F0047D
:10382B00A42480F5C6C23C75B901E5BC047002D274
:10383B003C22121870E5BEF54824F650037548007B
:10384B00753400753704C228D229D22A75C703E50F
:10385B004824E75003754800E54875F004A424801C
:10386B00F5C6751607751700C23C123898123898B2
:10387B001238981238988517581558755900E5481D
:10388B00B40A09E5586005F46002055922203C1D75
:03389B0075B901FB
:10389E0005C6AABCABBDACBEADBFEA1238B9EB12C1
:1038AE0038B9EC1238B9ED1238B922203C07F515AB
:1038BE00B4FF03D23C22C0C7C0C61287B475A7049A
:1038CE00851683E517C4F8F58275B90105C6E5BC02
:1038DE00F0C582F82406F92403C582E5BDF0E5BEE5
:1038EE00F0E5BFF075B90105C6E5BCF0E5BDF0E544
:1038FE00BFF08516838982E4F075B90105C685BCD3
:10390E001385BD14E4F0F08882E5BEF0E5BFF075D6
:10391E00B901E5BCF0E5BDF0E5BEF0E5BFF075839D
:10392E0006E51723541E24B0F582E513F0E514F0D6
:10393E0075A700D0C6D0C705172212B06478BEA6F0
:10394E004808E4F6F55908761808F6D23608760ACD
:10395E0008F6060876BEC237C22BC21AC21FC25460
:10396E00C255129B6F12384BC229C22AC207C227F8
:10397E00C268121861E5BDA2E59243C24AE4F52E73
:10398E00F534F536F52F78B6F678B5F678A9F678DB
:10399E009EF678B8A65E08A67A12E665C26BC233AA
:0239AE00C2381D
:1039B000C240C223C2221239D075460278C5A6463B
:1039C000C23AD221C219C226E4F542F541F540229D
:1039D000E45407205E09B4040040027403801B1203
:1039E0001866C313A9BC600C14A9BD600714A9BE56
:1039F0006002A9BFE94001C45407F5372212383DDF
:103A000012646F1207BE12F31212286EE55804708A
:103A10000A7F327E0590BF9B12814990C1F212A0AD
:103A2000021207187F7290C1E712813712F19B10C2
:103A3000000510020480F8D322C3220200EF1218FE
:103A400061E5BD20E7051239FD40F0123948129DAD
:103A5000E012B23B789F7680754A001297B1D2107F
:103A6000C211C213C212123EC712544775A61E12CB
:103A7000EDB312D82020250CE59054057009E535EA
:103A800024E25003023B74E5322418400D75F00C1B
:103A900084E5F070E0123FE080DB7532F012B23B5B
:103AA000E53124F39205201203123E20123B302010
:103AB000371A12A6D1200A0312B6CA123FE0128F9B
:103AC0009E123FE0129DE3123FE0803779247B1184
:103AD000123B1712F31212EB3112E34B12E6BB1238
:103AE000E5041215841215111228F979607B1D1254
:103AF0003B17799B7B1D123B1779D67B0E123B1728
:0F3B0000123FE030120E301A0B8009E532241606
:103B0F0050F212179D023A69D3E9953250FAE556F1
:103B1F00D23D12160FE552F556C23D12160F02F1A5
:103B2F009B301238E54024EE40267A0AC3E53F95D4
:103B3F004B601D402824E24017305405C254757F56
:103B4F0001E54B0475F03C8485F04B1297C0DADC2D
:103B5F0079BCE7D2E7F57F09877EC27722F4042488
:103B6F00E250ED80D412F3127F2A7E0E90C05812CD
:103B7F00814975A6FFC2101012137F367E0890BAC6
:103B8F000D12814912F19B12F1500200EFD2211256
:103B9F00B23B1297C07F1E7E0B90BF7412814912E9
:103BAF00F19B123BC77F3E7E0790BBAC128149123F
:103BBF00F19B12F14A0237F3D2201214E3C237D22B
:103BCF0015D214120BF675B90575B902129939D2BF
:103BDF005512982D7D0012B122129943E56A6005A6
:103BEF001297E080F712188E85BEBC85BFBD856B1E
:103BFF00BE856CBF75B90575B90285BD6C85BC6B8B
:103C0F00756A20129939123C9A857A621299437516
:103C1F006A001298AB7570FC854077854178851FD7
:103C2F00797818797A12DBA412B1741297D812F13D
:103C3F006579B877C309A77109A77209A77309A78F
:103C4F007409A77509A77709A778129943756A10A0
:103C5F001298AB7F087810797212DBA685627C858B
:023C6F005E7D78
:103C710079C0A71509A71409A77409A77509A7721F
:103C810009A77309A76C09A76B129AC6125FA18EC7
:103C91007E8F7F129AED0297D878107F0EE4F60896
:103CA100DFFCF564F565F567F5687515FC751AC0F7
:103CB100751DC0756640756940754A0112984F308F
:103CC1005503023D501297E0E571B510004002F531
:103CD10010E4F511E512207502E513C3957950063C
:103CE100207545857913D3E57A9514E5156480FF30
:103CF100E55E64809F400C857A14855E15857B1690
:103D0100855F173074B3C2D178647973123D2E7810
:103D1100677976123D2ED2D178187973123D2E78BB
:103D21001B7976123D2E809185791280B9D3E79661
:103D31000809E7960809E66480FFE764809F20D1BF
:103D410001B3400AE7F61819E7F61819E7F622E574
:103D51001AB4C00E7873791812DBA47873796412DF
:103D6100DBA478187964C2D1123DC17418126117AD
:103D71008E47AE1EAF1F781B7967D2D1123DC1C3EA
:103D8100E51F9FE51E9E50048E1E8F1F7EFF7FFF45
:043D9100AC1EAD1F98
:103D9500125EAF7A04EF8AF0A4E5F0CE8AF0A42E85
:103DA500FEE435F0BEFF011E60051460057EFF8E42
:103DB5001F22EE7E0020E7F77EFE80F3C3E697FB29
:103DC5000809E697FC0809E697FD1818191930E760
:103DD50003126037C3EB33FBEC33FCED33FDEB3300
:103DE500EC33FBED33FC30D105AA47125DCD0BBB9F
:103DF50000010C751E03751FFFEC24FC40048C1E8E
:103E05008B1FE627FB0809E637FC0809E637A2E71A
:103E150013F618EC13F618EB13F62210131978B5F0
:103E2500E624FA401AE57124F64008E57924F640BF
:103E35000280330606802F12F161E59030E2DFD271
:103E450020753612D22EE4F534F55A129BA1123E96
:103E5500D5C2191239D012AA0012AA2DD212853F45
:103E65004B205E02D2281239C8307335E53F20E079
:103E750030E55D455C602A75A7009006FAE0255C93
:043E8500F0FBA3E0CB
:103E8900355DF0FCA3E03400F0FDA3E02401F0F877
:103E9900A3E03400F0F9125F488C4E8B4D2275A7D0
:103EA900009006FDE0F9A3E04960F2121884C3E529
:103EB9004D9560F5BCE54E9561F5BD0255F775A7C1
:103EC900009006FA7F05E4F0A3DFFC22D214123F2A
:103ED9001BE6F008DFFB857A62123F117570FE78E8
:103EE9003A797112DBA41297DD123F1185627A8546
:103EF9005E7B7570C01297DD123F1BE0F608DFFB91
:103F090075A700D254C2142274FF7870F608B880DD
:103F1900FB2275A7049004F078707F102212F31227
:103F290012F19BC258C259123948753901754A01B3
:103F390012DB8312984F1261158E47C210D211D22B
:103F490014D212129BA112AA0012AA2D12EDB37556
:103F5900A6FF753609753200E59020E206E535249D
:103F690005400CE59054057019E53524E25013C25B
:103F790011C21212F31212F19B12F15312F19102B2
:103F89002CD8C221E54AB40202D22112984F128FCD
:103F99009E30260F1264D1129DE3753606E5367000
:103FA900FCC226129DE0123FE0E54A20E021B4025E
:0F3FB90009753900E53670F98092E53960FAFD37
:103FC80024E24002053912984F2026C9DDF880E91D
:103FD80075390080E475370410003A100116100294
:103FE80016E52F5407600312AE4E20784C20790A4C
:103FF800207A1F220241F2024139E5376009146034
:10400800091460090242AD02421302427EC27902DB
:1040180042D402416C20110C3037091214E3753474
:1040280000C27822E53724FC500FE53764076003A7
:1040380002434A02430E0241032011FAE59020E2AE
:10404800028056753400201203D2132278A9E67034
:1040580017C226767DE5377005106B02D26BD277D2
:10406800753614D22E029B96E5376043146040B42F
:104078000227200B24E6249B401F2414501C12AA5C
:104088000090BF447F207E0812814912F19B75364B
:1040980008D22E78A9E624ECF622241940FB241431
:1040A80050F712AA0012AA2D90BF4E7F2980D72060
:1040B80028E7E54824F640E1E5580460DC7F5D7EAA
:1040C80010E6249B40D324145015C2330559C3E588
:1040D8005895595005855859D22690BF3280A92441
:1040E8001940B6241450B2E5596002155910260635
:1040F800E5596002155990BF3B808D1078012275F3
:0F4108003900E53424384007754A017534002228
:10411700700AE54A30E0F2754A0280F014600875CB
:104127004A0612AA2D8006754A0412AA007539019B
:1041370080DA302909C229D22A7559008005302A28
:104147001BD229129FB1129F7FE53524AF4004751A
:10415700340022753700C229C22A80F320684E3006
:104167002703D26A2220110A3037071214B6C27AFF
:104177008015D2221244E612F19B107A0122E5340F
:10418700243840071239D075340022700FAA37122D
:1041970039D06A70F274011239D180EB041239D127
:1041A70024FC50E3E537B40706D22880DA8036C20C
:1041B70028E53724FC2324BEF879C4E7F9A7480982
:1041C700A75979C4E8F78648088607E537B405058F
:1041D700754818D2361238578F59E537640670027A
:1041E700D20702418E1244C202446CE537601D14A7
:1041F700600F14601114600BE53724F9400B02437C
:10420700C480740242AD0242FD02439120110A208C
:104217001207C279123EA78012D223124CA6107938
:104227000122E534243840077546017534002278A9
:10423700D87020304A0BC24AE624F85004B24380B3
:104247000AD24A7614E54624FE40DDE54660D915D4
:064257004680D8B600D538
:10425D00B40500500C04F54624FA50C97546058086
:10426D00C424F950051285A480BB100FB8D20F805D
:10427D00B4D223E53464C86003124CA61079012230
:10428D00E534243750097011105B3CD25B80381037
:10429D000802D208124CA6802E100C2BD20C8027AF
:1042AD00D223124CA610790122D24BE5342437408B
:1042BD0002801424FC402824047010C258C25920D6
:1042CD001105D22E75360775340022D258C25914F5
:1042DD00700280F3C258D2591460ECD25880E812A3
:1042ED00186BE5BCB2E7F5BC79A1F71255F780D78D
:1042FD0078B8A65E08A67A2011CD753605D22E8027
:10430D00C630122B129FEB055BE55B75F00B84E558
:10431D00F0F55BE55A24F64009E55A955B500375B7
:10432D005B00129FEF12F19BE5346003D534D2751B
:10433D00340022D229D22A75480A024432C24010D2
:10434D0007F1302903024432129FAD129FC1102A8A
:10435D001BC2330559C3E558955920E7025008751E
:10436D005900E548B41816E558B4FF037559001205
:10437D009FD512F19BE5346003D534C122D22A12A8
:10438D009FB180EE301223129FEB155BE55B30E79A
:10439D000C755B0AE55A24F64003855A5B129FEFB4
:0343AD0012F19B6F
:1043B000E5346003D534DA75340022D229D22A7567
:1043C0004817804CC2401007F2202944129FAD12BA
:1043D0009FC1102A22C2331559E55930E71C855870
:1043E00059E558B4FF03755900E548B41802800A2E
:1043F000D22A129FB1800E855859E558B4FF037533
:104400005900129FD512F19BE5346003D534B522D3
:1044100020106220115F7F180548E5486418700875
:10442000F54830270375480A123823303C2DDFE861
:10443000802620105A2011577F181548E54830E78C
:1044400005754817800A64097006302703754817F8
:10445000123823303C05DFE275480A1238571264DF
:104460006FE532244C5005129F7F8003129F257503
:10447000340002F19B1244A97F15E5486B70048A51
:104480004880020548123823303CD0DFED80CC1242
:1044900044A97F15E5486A70048B488002154812CC
:1044A0003823303CB6DFED80B27A007B09E537B4C3
:1044B0000401227A0A7B17B40601227418FAFBF56C
:1044C000482275A704758307E559C4F582E0E0F535
:1044D00073E0F574E0F575E0F576E0F577E0F578F2
:1044E00075A70002646FE59020E23EE53424375062
:1044F0003812452A124507205E4F7F2C90B7A7122D
:07450000457190B7B0806A1D
:10450700E534243775F009A42435FF205E0624BE60
:1045170050027F3EEF249B50027F627E32748912E5
:10452700E8FC2275A7049000317E087F3AE4F0DFAB
:10453700FDE5822446F582E43583F583DEED75A734
:1045470000227F2C121866E5BD12455AE5BE1245BA
:104557005AE5BFF8C4124560E8540775F009A490FE
:10456700B7952582F58250020583EF2409FF028162
:01457700370C
:109DDD00029E9A12F312E53724FC40F4B4FE1420CF
:109DED00110EE590F45407600122E532247450EF12
:109DFD0002A6DD12F31212EA9F12EB3112E34B129F
:109E0D00E6BB12E5047E197F3612E48512F07A1254
:109E1D00E49BC206E53760051460338053C23A12E5
:109E2D009F3E124D61124EF61251DC126F3B126FB6
:109E3D0063124A14E54864186009E54824F6500396
:109E4D001252C712A67312E1CE124DFC8014D23AF3
:109E5D00129F64124580124DCB12DCFB12A67312B9
:109E6D00E18F1267B012EB78126281126580801259
:109E7D00129F4A12DC3812EC4A12DCCA12A6731277
:109E8D00E1A630101412E40E12E3DD800C12F31271
:109E9D00E53724F9401E129F273022091244E6E5CA
:109EAD00347002C222302309124CA6E5347002C26E
:109EBD002302F19B12281975170012EE5E7F121204
:109ECD00DD8330124A75100075A70475830612657F
:109EDD002AE51075F009A42415FFF5177E00E5128B
:109EED00602F75F06484E5F00F12E84A1F7E0EE5D1
:109EFD001112E3937516231266E60510C3E55A9504
:109F0D00104006E51024F550BF301203129FEF806C
:109F1D0088745D12E8FC80D5C2493029051227EFFF
:109F2D00800312281990B9D412A002202A76029F1C
:109F3D00D5301223305E2030501D02A2E9301217A9
:039F4D00305E067D
:109F5000200B1102A94A12DD7C7F1712F28D7517B2
:109F60002002EE5E12EA1612E9B7301211205105F6
:109F700012EA76800612E0CC12DEAC125BDE22E43E
:109F8000FEFFE54824F6400D90BF7E12817C7E16D0
:109F9000E54802E8B7B40E0690BF8402817C90BF0A
:109FA0008B12817C7E12E54824F702E8507D2080E8
:109FB0000C7D3F302A077D633029027D3C7F008085
:109FC000247D2080127D3E800E7D3CE54975F007A2
:109FD000A42406800A7D3FE55975F007A42409FFF3
:109FE00064027001FF7E1CED02E8CA7D2080027DC4
:109FF0003FE55B75F009A42416FF7E09ED02E8CA6F
:10A00000C24912A066B4FF012275100012A07D792A
:10A0100020E030E702792F304917121BABFAB40465
:10A0200008E510700C79658008EA146510700279F3
:10A0300023E97E1812E8CA7E20E51230E70890BABC
:10A040000D12817C8016E51112A0F31267462010D4
:10A0500005201102800630120312A0A50510C3E5E9
:10A0600058951050A7227E207F0012817C129F7F7E
:10A070007E007F0690A12512E928E5582275A704E5
:10A0800075830712652AE51075F007A42409FFF50A
:0DA09000177E00E51212E8CA7805EE2404E0
:10A09D00FEE012E8CAD8F62212A1B012A1C6FD7CCC
:10A0AD0000AE1CAF1B125EA2BE003A8F00C3E57A54
:10A0BD009513FFE55E9514FE402B7C007D28125E06
:10A0CD00AFC3EF98401F75F0058404FB24F95002CF
:10A0DD007B067E2CAF170F12F22D0F12F22D0F12E1
:10A0ED00F22D0EDBEF2264B4602464B475F032847B
:10A0FD00C0F012E8B7CE2404CED0E075F00584C0D0
:10A10D00F012E8B7CE2404CED0E02302E8B790A138
:10A11D002102817C2D2D2D000140FFFFFFE0FFFF6F
:10A12D00FFFFC25030124220283FE558F4603A201C
:10A13D004803200934D250E559F5103033096558DC
:10A14D006005204802051012A17A12A1D675A70448
:10A15D009006DCE512F0E511F0E517F0E510F0756D
:10A16D00A7049006E0ECF0EBF075A7002275A704AC
:10A17D0075830712652A7813E0F608B819FA900668
:10A18D00D07811E6F008B819FAE51CF516F0E51BC4
:10A19D00F515F012A1B09006DAE514F0E513F0759F
:10A1AD00A7002275A704758306E51023541E24B05D
:10A1BD00F582E0F513E0F5142212186BE5BD248746
:02A1CD00E5BDEE
:10A1CF00923B500224912212A1C675F005A485F08E
:10A1DF0012F511E4F519FEF51CF51D129939C23D62
:10A1EF00C2567F3C12DE31303D05751900807DDF90
:10A1FF00F3E5596558700A301007EE24D35002D298
:10A20F00568C1B8D1AE519FD24E250DEAE1CAF1DD6
:10A21F007C00125EA2EFF51924F650CEAC1BAD1ADE
:10A22F0012DD6B20D1108E048F05E51975F0A7A4F0
:10A23F00AEF0FF125EA2AC12AB117AA0125DCDEBA5
:10A24F0033FBEC33FC20D11AEF9BEE9C5014C3E58B
:10A25F001213FCE51113FBC3EF9BEE9C4004AC06FD
:10A26F00AB07204807203B048C128B119006E2E5C8
:10A27F0019F012A2BEAC16AB157AC8125DA4A912C2
:10A28F00A811125F48ED7005EC249E50057C807B71
:10A29F000822C3E57A305602E55C9513FFE55E3080
:10A2AF005602E55D9514FEC3EF9BFBEE9CFC22AEC0
:10A2BF0016AF157C00E519FD24F6501A125EA27C2C
:10A2CF00007D06125D827C007D05125EA28F10EE6E
:09A2DF00F51724E950037517FF7F
:10A2E8002212DD7C12A30612A34912E66A12A36F9A
:10A2F80020480912A45D12A48D02A4F080747F176F
:10A308007E2020480E748A204D101262EE500E7482
:10A318002F8007746A305F02746712E8FC75A7041F
:10A328009006D07811E0F608B819FA7F177E007801
:10A3380012751905E60812E8FCEE2406FED519F494
:10A348002275A7049006D8E0F516E0F515E0F51497
:10A35800E0F513E0F512E0F511E0F517E0F510E08F
:10A36800FCE0FB75A700227F187E26AC14AB130215
:10A37800E6FC9006E4E0F51CA3E0F51B7F2A304ECE
:10A3880013121861E5BF90BFE8B4010390C1E11250
:10A39800813780420F7E00745312E8CA9005CBE0E3
:10A3A800F830E705E53F30E0091F7E00E8540F125A
:10A3B800E8E29004EEE0FEF51EA3E0FFF51F12A40C
:10A3C80005E51E24E9500C7E06742B12E8FC7E0C71
:10A3D80012E8FC12A435C20375172A7516271266EF
:10A3E800B5202415205F15D2037F2A7E1E90A42352
:10A3F800304E0390A42C02E928205FEB227C007DDC
:10A408003C125EAFA805EF7F2A7E0812E8037E1291
:10A41800743B12E8F87E14E802E7FD0707384C9E03
:0FA42800BAF264380707387CE6C2E67C38AC1C11
:10A43700AB1B7A48305D027A27125DA4A91EA81FBC
:10A44700125F48ED4C60027BFF7F207E28EB12E80D
:10A45700097E3902A9DD7F2B90BF9112817AE5171A
:10A46700F46022AE17AF107C007D3C125EAFA805EA
:10A47700EF7F2A7E0C12E8037E16743B12E8F87E03
:10A4870018E812E7FD22AE12AF117C007D0A125EBA
:10A49700AFA805EF7F207E3012E8037E3A742C12B6
:10A4A700E8FC7E3CE812E8E20F7E29744502E8CA20
:10A4B70074858007748720560274867E2912E8FC0B
:10A4C700301707742D7E3A12E8FC227C007D0A12B1
:10A4D7005EAFA805EF7F2A7E3012E8037E3A742C20
:10A4E70012E8FC7E3CE802E8E212A621E54824F6E1
:10A4F700500512A4D280B9E559046558600D12A41D
:10A50700D212A4B7E559655860AA22A217923D8EC8
:10A517001E8F188515179006D0E0F5118558101570
:10A52700101251BCC3E51195105002F404F924A68A
:10A537005005C374B399F9E975F00584F924EE5011
:10A5470002791190A661E993F5F01207D2E5CC7074
:10A5570004E930E702747F23A4A9F0E51B2517FD62
:10A56700E51C3516FEC3ED99F515EE9400F5167545
:10A57700A700758306E55823541E24B0F582E0A38F
:10A58700F513E0F51412A621203D2C2017291218E7
:10A597006BE5BD2487E5BD5002249175F007A4FB48
:10A5A7009518E5F0951E400FEB9FE5F09E4008EFEC
:10A5B7009518EE951E500EA23D9217AE1EAF1812BB
:10A5C700A4D202A4B7306B1012A5BEE53F20E00766
:10A5D70074867E2212E8FC2275A7009006E0E51635
:10A5E700F0A3E515F012A4D212A4BB74857E231242
:10A5F700E8FC85581012A17A12A30612A3498C16FB
:10A607008B1512A36F12A28412A16C12E66A900630
:10A61700E2E0F51912A2BE02A45DC3E57A30560244
:10A62700E55C9513FFE55E305602E55D9514FE92F5
:10A6370017500312601FAC16AB157AC8125DA4A998
:10A6470006A807125F487E037FE7ED700CEB24181E
:10A65700EC34FC4004AE04AF032200172E43576CC2
:10A667008092A4B6C5D3DFE6EDF3F8FD305E4F3038
:10A67700504C75A7009006E0E0A3FCE0FBECA2E7D6
:10A687009217402024FE50047F3B8022AE04AF0384
:10A697007C007D14125EAF74542F2017029F9FFF1A
:10A6A7007462800C12602FEC24FE50E07F6D743DC5
:10A6B7007E0012E8CA7E017D197C0312A6C6227F9E
:10A6C7003D12F22DEF2DFFDCF822E537B40206E547
:10A6D70034243750292212F31212EA9F12E34B1245
:10A6E700A85D12DBC612E1B612A8B51265807F20FD
:10A6F7007E2B12E48512EB3112F07A1244E612E552
:10A707009012A78B125B7802F19B20041EE579FD5E
:10A7170024A050027D5FED24CD401E744520750CAA
:10A727002DFFF51212A7601FBF44F922C39DFFF545
:10A737001212A7600FBF46F92220750EED2413FFF2
:10A74700F51212A7600FBF78F922C374779DFFF542
:10A757001212A7601FBF12F922EF24BA4008243350
:10A76700FCC374329C1404FC24D750047C23800956
:10A77700EC2375F005842413FC7E0512F22D0EECF4
:10A78700B506F822E59020E206E5342437400312A7
:10A79700A7117F457E047D1212F22D0EDDFA7F434D
:10A7A7007E00746412E8CA7F4F7D1212A8467F3B71
:10A7B7007D1212A8467F597D1612A8467F317D1655
:0EA7C70012A8467F637D1A12A8467F277D1ACE
:10A7D50012A8467F6D7D1E12A8467F1D7D1E12A8FC
:10A7E500467E057F1912F22D0FBF72F97804E579BF
:10A7F50024CD50027809E8305C0123F87F1B12A8AC
:10A80500357F6B12A83518305C01187F2512A835E5
:10A815007F6112A83518305C01187F2F12A8357F8B
:10A825005712A83518305C01187F3912A8357F4DAD
:10A835007E00E875F00A847004E802E8B7E802E8EB
:10A8450050EF6512600C7E04EE20E00712F22D0E2B
:10A85500DDF62212F25D80F790C0A77F287E2C12CC
:10A86500817C7E3B12E713AC5EAB7A7F307E19C2EA
:10A875003D12E75290BF957F5D7E2D12817C78B9A0
:10A88500C3E57A9618FBE55E96FC7F507E19D23DAE
:10A8950002E752E51164B4700122E51112F0EA787D
:10A8A50031790F7D0B12F1F01F1E90A94502E928A1
:10A8B500E5716012E57012F0EA7831790F7D0412C6
:10A8C500F1EC0DBD0AF97F0112A91D7F1D12A91D0D
:10A8D5007E2312A9277E3F12A9277E247F1712A95E
:10A8E500317E397F0212A9317E247F0712A93B7E72
:10A8F500397F1C12A93B7E317F0212F22D7F1C127B
:10A90500F22D7F0F7E2412F22D7E3E12F22D7F0C4A
:10A915007E2E90EC1F02E9287E2A12F22D0EBE39FA
:10A92500F9227F0812F22D0FBF17F9227D0612F2C8
:10A935002D0E0FDDF9227D0612F22D0E1FDDF922F7
:10A945000303E0A0E012DD7C7F1890B7E512817A61
:10A955007F217E01744112E8CA7F2A7E0174531259
:10A96500E8CA9005BEE0F51AA3E0F519A3E0F51EC7
:10A97500A3E0F51D851A1C85191B75172012A9FA68
:10A98500E519251DF51BF51DE51A351EF51CF51EEA
:10A9950075172912A9FA9005BA12A9EAAC1AAB19CA
:10A9A50075172012A9B89005BC12A9EAAC1EAB1DFB
:10A9B500751729EC7006EB24CD4001227A48305DED
:10A9C500027A27125DA4125F48ED4C600122AF1791
:10A9D5007E07EB12E7AF7E1A0F90C16A305D0390D8
:10A9E500C16D02817CE0FEA3E0FD129D19C3EB9DC4
:10A9F500F8EC9EF9227516270266E6129D1975A7D1
:10AA0500049005B478737F06E6F008DFFBECF0EB05
:10AA1500F0E0E0E0FCE0FDE0FEE0FFEF2DFFEE3CC6
:0EAA25009005C0F0EFF0801275A7049005BAFE
:10AA3300E0FBE0CBF0EBF0E0E0E4F0F075A7002200
:10AA430075A7049005B478647F06E0F608DFFB750C
:10AA5300A7001268F59005BEE51CF0A3E51BF022E4
:10457800D23C799E77008002C23C129939E4F5104A
:10458800F511F512F513F514F515F516F517C23DE5
:104598001248C5203D1F1248C5203D19E51F30E5CA
:1045A8001130E40E1245EF303C08799EE724F550AF
:1045B8000122D510DBAE14AF157C00AD12125E7C63
:1045C8008F55AE16AF177C00AD13125EA21260A90C
:1045D8007E00E55530E7011E2DFFE43E30E7027FFF
:1045E80000740A2FF55622C235E51CAF1DBFFF0522
:1045F8000FD235F404FABF003F532CF8E518AF1971
:10460800BFFF050FD262F404BF002D20E72A205B0C
:104618000123FF24AA4021E51AAE1BBEFF050ED2D6
:1046280061F404BE00128547F0A4E5F020E70920F4
:104638005B0123FE24AA5001227C807B80305166D6
:10464800302163C006C0078AF0E545A4AEF0FFE557
:1046580056205B011375F009A4ACF0FD125EA2743C
:10466800FFBE0001EFFA24C050027A3FD007D006FF
:10467800E55212F0EA303504B2D5B2D1EA8CF0A492
:1046880030E70205F0748025F020D10495F095F00C
:0A469800FCEA8BF0A430E70205F005
:1046A200748025F030D50495F095F0FBC3EC2F20F3
:1046B2006203C39F9FFFEB2E306103C39E9EFE20C9
:1046C2003C64200C0512475C406412473E405F1276
:1046D200F22DE51EFD24FB50550E12F22DED24F6AF
:1046E200504C1E1F12F22DED24F150421E0F12F2F9
:1046F2002DED24EC50380F12F22DED24E7502F1F30
:104702001F0E0E12F22DED24E250231E0F0F12F295
:104712002DED24DD50180E12F22DED24D8500F1E6F
:104722001E1F1F02F22D12473E4003799E0722E907
:10473200242AFFE82461FE12475C401DEF246040FA
:1047420018243F5013EE2460400F243F500AEF24F8
:10475200D6FFEE249FFEC322D322532CF8432C040F
:10476200EE10E706D2E7F404D261FE24D340EAEF6A
:1047720010E706D2E7F404C262FF24D340DBEFB5B0
:1047820006005003CED26070057480FE8062FF2462
:0D479200FD5060904848938EF0A4AAF033CB
:10479F00CA33CA33CA33CA33CA33FA904872938FB3
:1047AF00F0A433C5F033CA90489393FB1248109589
:1047BF0070500224B412F0EAEA8BF0A430E702053D
:1047CF00F0C3748095F020D50425F025F0FEEA8C17
:1047DF00F0A430E70205F0C3748095F030D10425C2
:1047EF00F025F0FFC3227A01EE6F70097B16BF022E
:1047FF00BB7A0380B7BF01047B0080B07B0D0A80BA
:10480F00ABE52C540723C390481A73800E800E809B
:10481F0024801E8010800A80108012EB22742D9B42
:10482F0022742D2B22745A9B22745A2B2274879B2D
:10483F002274872B2274B39B22FFFFCCAA92807124
:10484F00665D554E4944403C383533302E2C2A286E
:10485F00272524232221201F1E1D1C1B1A1A19185D
:10486F001817178181818282838384858687898A3D
:10487F008B8D8F90929496989B9D9FA2A4A7A9AC85
:10488F00AFB1B4B400010203040405060708090A16
:10489F000A0B0C0D0D0E0F0F101111121313141410
:1048AF00151516161612983312B191E4F5F7E4E5C3
:1048BF00F7D2B264C022203D071248B47003D23D34
:1048CF0022056D056D12B1917D008DF7E485F71FFF
:1048DF008DF7C3E5F79573F5188DF7E4E5F7957444
:1048EF00F5198DF7E4E5F78DF7C3E5F79576F51A2A
:0C48FF008DF7E4E5F79577F51B8DF7E4E5
:10490B00E5F78DF7E4E5F7F51E8DF7C3E5F7957A37
:10491B00F51C8DF7E4E5F78DF7E4E5F7D2B2543FDC
:10492B0030E50244C0955EF51D156D156DE510243F
:10493B00784001227E00AF55EF30E7011E0512E5EE
:10494B001FA2E592D5400EE515951EF515E51494BD
:10495B0000F514800BE515251EF515E43514F5143B
:10496B007800E51E600620D50318F404C39FF5F00C
:10497B00E89E30E701220513E5F0A42517F517E5AE
:10498B00F03516F51622303D03D23D221248B460A5
:10499B00F81248B460F3E546600A1248B460EA12B4
:1049AB0048B460E5056D056D056D12B1917D008D07
:1049BB00F7C3E5F79573F5188DF7E4E5F79574F5FF
:1049CB00198DF7E4E5F78DF7C3E5F79576F51A8DB5
:1049DB00F7E4E5F79577F51BD2B2156D156D156DEF
:1049EB0022307424129939C23D75101E1249912040
:1049FB003D167902124A58400CA806A907124731F6
:104A0B00400312F22DD510E422200F4030123D202E
:104A1B0006CF304806200C03204FC6E546790260CE
:094A2B0014790614600F791614C9
:104A3400600A79361460057976147017129939C2B0
:104A44003D7896124991203D0A124A58400312F2C9
:104A54002DD8F022532CF8AB18E519FC33926212CE
:104A64004AAABC002BEB89F053F00784FF24DF40F3
:104A74001FAB1AE51BFC339261124AAAAA47125DC6
:104A8400CDBC000CEB89F053F00784FE24DF500208
:104A9400D32274562F2062029F9FFF741F2E306111
:104AA400029E9EFEC322500312602FE920E40122DD
:104AB400C3EC13FCEB13FBE920E50122C3EC13FC6C
:104AC400EB13FBE920E60122C3EC13FCEB13FB22FE
:104AD40074542F2062029F9FFF741D2E3061029E2A
:104AE4009EFE2279B4203249201D46EFB50600927D
:104AF40060AC06AB074004AC07AB06904B36EC2326
:104B040004938BF0A4A9F0EC23938BF0A429F990DF
:104B14004B9693C9904C96E52C54079313E9500196
:074B2400F4904C9EF9E52C12
:104B2B005407932975F0B484A9F022FFFFFFFF7F90
:104B3B00FF55553FFF33332AAA24921FFF1C7119CF
:104B4B00991745155513B1124911110FFF0F0F0E80
:104B5B00380D790CCC0C300BA20B210AAA0A3D099B
:104B6B00D8097B092408D30888084207FF07C10727
:104B7B00870750071C06EB06BC06900666063E062A
:104B8B001805F405D105B005900572000000000072
:104B9B0001010101010101010102020202020202F3
:104BAB0002020303030303030303030404040404C7
:104BBB00040404040505050505050505050606069B
:104BCB000606060606060607070707070707070771
:104BDB000808080808080808080809090909090944
:104BEB00090909090A0A0A0A0A0A0A0A0A0A0B0B1C
:104BFB000B0B0B0B0B0B0B0B0C0C0C0C0C0C0C0CF2
:104C0B000C0C0C0D0D0D0D0D0D0D0D0D0D0D0E0ECA
:104C1B000E0E0E0E0E0E0E0E0E0F0F0F0F0F0F0FA2
:104C2B000F0F0F0F0F10101010101010101010107E
:104C3B00101011111111111111111111111111125A
:104C4B001212121212121212121212121313131335
:104C5B001313131313131313131313141414141414
:104C6B0014141414141414141414151515151515F3
:104C7B0015151515151515151515161616161616D3
:104C8B00161616161616161616161600FFFF00FF2A
:104C9B000000FF002EB5875B2D5A88E537606C143A
:104CAB006036B402507F347E12E53424375046F818
:104CBB00904DE812E928E824FC501179A1E77E0514
:104CCB0090BCA820E70390BCB10F803A24040F7E60
:104CDB002312E8E9D26480627F357E02E534243703
:104CEB00401410641090BBA330081B1281497E1A2C
:104CFB0090BF64801122700590BBB5800990B812EB
:104D0B00200C0390B81D12814980C97F35E53424EE
:104D1B0033402A2404501B7D0F600C7D1E1460074A
:104D2B007D3C1460027D78ED305D02C3137E2B1247
:104D3B00E7AF7E0090BBB612814902F19B7E052442
:104D4B00FE500590B9FA800990B7F5200F0390B883
:104D5B000112814980E4E546604A14603C14602EE0
:104D6B0014602014601290C19E205D41904DE17F34
:104D7B00367E3412E928803C90C19E305D0390C191
:104D8B009A802A90C19A305D0390C196801F90C182
:104D9B0096305D0390C192801490C192305D039068
:104DAB00C18E800990C18A305D0390C1867F367EAB
:104DBB003312817C7E3C7422305D02748302E8FCEA
:104DCB00305D0890C176305BE4800690C17E205B3D
:104DDB00DC90C17A80D70508B28D8DB5BA09100663
:104DEB00000A10F248922492249224F2480A1006E8
:0E4DFB0000305E5220434F20284CE55864FFE4
:104E09006046E54824F640407F3FE55804F9C23D35
:104E1900124E52121BAB601AB404047401D23D75D0
:104E2900F003A4243CB5070A7E3A303D027E3612CF
:104E39004E540F0F0FD9D7E55975F003A4243EFF3F
:104E4900124E520F0F124E52227E3D12F22D0EBEFD
:104E590040F922C248C249305E56202853E55864B9
:104E6900FF604DE54824F64047121BAB6042D2492A
:104E7900B40402803B1465597036D248304E31E58E
:104E8900596558602B307428124EBF121861E5BF5E
:104E9900B4011DE5BD20E618202416205F129006F6
:104EA900E4E0700CA3E024CE400624255002055905
:104EB90022305FFC80E820113375A7009006E4E0FA
:104EC9007028A3E0302402F404305F02F4042404BF
:104ED900F924F74015E924FC4003D26C2270012221
:104EE900306C097536A7D22ED22FC26C22305E08DB
:104EF900307405E558B4FF0122C244C24D780075EB
:104F0900A70475830712523E88188A1E8E168F17BA
:104F1900C23EC23BE54824F65003024FCFD23EE5DC
:104F29005860F7E8655970F22048EF12508430D183
:074F39003BAE16AF17A818EC
:104F4000E54670551207D2E5CC49604DD244E5CC18
:104F50007033E924CD402EE975F038A4ACF0FB1293
:104F60005FBE125FBEEBFDF511124FE5304D2CC256
:104F700006C23B8043E546705C1207D2E5CC700563
:104F8000E924CD50501259AF75A704758307A818AE
:104F900012523E8A1E8E168F178037121861E5BD99
:104FA000A2E0B3923B50113074281247314026A939
:104FB00007A806D20612DE18125001124FF812503E
:104FC00041890788061E1F90523912E92880063051
:104FD000D103125019A81808C3E558984003024F8E
:104FE0000875A7002274562F2062029F9FF9741F34
:104FF0002E3061029E9EF822E51865586001227DE0
:10500000057A00EA12F0EA12F1F00A0AED24F24001
:10501000020A0AEA244C50EB22AE16AF17124AD409
:105020001E303E021E1EE51E12E8CAEE2404FEE5F6
:105030001212E8CA303E09EE2404FEE51312E8CA53
:1050400022E5186558603CC001C000C012C013853D
:1050500018101251BCD013D012D000D001E510307E
:075060003B07C395705002ED
:1050670024B412F0EA203B07AE16AF17124FE5E55E
:10507700112402FD7A0612F1F01DDAFA22121BAB97
:10508700B40457E8705412187FE5BD604D78C6A682
:105097001308A61208A62C12DBB375A7047583079D
:1050A7007510011264FB12DBAD15101264FB12615F
:1050B700158E628F6312619D8B1C8A1B12DBB920D0
:1050C700320E12516C203B08D24D1271461250E23B
:1050D70078C6861308861208862C2212187FAABD66
:1050E7007C027BB3125DCD8C128B13AA1DA91F12F4
:1050F7005E0FA91CA81B125F488C1D8B1FAC12AB3F
:1051070013AA19A91A125E0FA91CA81B125F488CB3
:10511700198B1AE56E251AF9E56D3519F8C3E56E91
:10512700951AFBE56D9519FAC3E554951FFDE56FD3
:10513700951DFCE554251FFFE56F351DFEE52C2366
:10514700652C30E206ECCEFCEDCFFD75A70490058B
:10515700C2E8F0E9F0ECF0EDF0EAF0EBF0EEF0EF9A
:10516700F075A70022D23BC3E5649573C5659574B6
:0E517700F564E5669575600404600822E56441
:1051850024E0500822E5642420400122C3E5679508
:1051950076F567E5689577F566E5699578600904BC
:1051A500600122E566F48002E5668562F0A474E09C
:1051B50025F04002C23B2212DBB375A704758307B5
:1051C5001264FB12DBAD05101264FBC02C126514D2
:1051D500D02C891002DBB930125120064E780075AB
:1051E500A70475830612523E30D139124AD4E546DA
:1051F50024FE500A0E0F90523412E9288026EA70D8
:1052050007745D12E8C6801C75F06484ADF0700FFC
:10521500ED75F00A847008E5F00E12E8B780051EFA
:10522500ED12E84A08C3E55A9850B475A700220361
:105235000340A040030340E040D2D1E8C4F582E03A
:10524500FA797312529730D146AF06532CF8EDBF59
:10525500FF07F40460390FD262BF00331253CB400D
:105265002E797612529730D126E5822403F582E015
:10527500F512E0F513EEA2E713FEED13BEFF07F4FA
:1052850004600C0ED261BE00061253E8400122C232
:10529500D122C3E09709FDE09709FEE09760090474
:0352A500700AEE9E
:1052A80030E7068007EE30E703C2D122E546600EFC
:1052B80014600BF9EDCEA2E713CE13D9F8FD227CCA
:1052C800007B44E54660207C007BCC1460197C019F
:1052D8007B981460127C037B3014600B7C067B6027
:1052E8001460047C0C7BC08C148B157AE9125DA4C5
:1052F800A847125F468C168B1775C70075C60475CC
:1053080010DF75B901E5BC20E76FF51385BD1205FF
:10531800C605C675B901532CF8C3E5BE9573FBE500
:10532800BF9574FC05C675B901E5BC9575FD5005BA
:10533800D262126037C3E5159BE5149CE49D4033A7
:105348008C198B18C3E5BD9576FBE5BE9577FCE512
:10535800BF9578FD5005D261126037C3E5179BE50C
:10536800169CE49D400D8C1B8B1A125392E5322437
:1053780028401305C6E5C68006E5C62404F5C670B0
:105388000205C7D510012202530AAE19AD181252F0
:10539800B4ED1253CBAE1BAD1A1252B4EE13ED138B
:1053A8001253E8124AD4E54624FB50080E0F9052D7
:0B53B8003902E9281EE51312E8CAEED6
:1053C3002404FEE51202E8CA75F0067FFDA946B97A
:1053D300000575F0027FFF84C5F02F500205F0C56C
:1053E300F0FF24DE228547F0A430E70205F0E5F064
:1053F300A946B9000280050475F00384FE24E02267
:10540300E537B4020122E5377002D2396402700233
:10541300C239E53724FC799EE76005640B600C22F2
:10542300D27E20081E401C107F1022D27F2008133A
:105433004011107E01227537012275370020390390
:105443007537022275FB0075F9FF802775FBFF7521
:10545300F9FF801F1220C32053F2125488759E85D2
:10546300759D2D8014125488759E84759D2D800919
:10547300125488759E83759D09C2AC759852C26D8E
:10548300C26EC26F22C25375FBFF75F90022C23D83
:105493001254F6203D012275BC4175BD3075BE30F6
:1054A30075BF301228297F5A90B7021281377F6463
:1054B30090B70E1281377F6E1254FB7E20A8BC1268
:1054C3008F6188BC7E26A8BD128EAA88BD7E2CA8BB
:1054D300BE128EAA88BE7E32A8BF128EAA88BF12C1
:1054E300288912F19B1000051002B880F81255F7B5
:1054F30012F3121218897F4B7E0890C166128149FC
:105503007E20E5BC12E8FC12552E7E26E5BD12E88E
:08551300FC1255377E2CE5BEA9
:10551B0012E8FC1255377E32E5BF12E8FC12553704
:10552B0002F19B24BF500E24E6400A2224D05005E2
:10553B0024F6400122D23D2275C70375C6FE1280A8
:10554B00B51255F775C6FC75BC2675BD6475BEA93D
:10555B0075BF701255F775C6FB1280B575BC64121A
:10556B0055F775C6FA75BC1475BD1475BE0075BFBD
:10557B000C1255F775C6F975BC4E75BDBF75BE00DF
:10558B0075BF191255F775C6F875BC0A75BD7E75D2
:10559B00BE0075BF011255F775C6F775BC0175BD19
:1055AB002375BE4575BF671255F775C6F675BC02F8
:1055BB0075BDAB75BE0175BF011255F775C6F512FA
:1055CB0080B575BE0275BF0A1255F775C6F4128009
:1055DB00B575BCE11255F775C6F31280B11255F7CC
:1055EB0015C61255F715C61255F715C675B90575BB
:1055FB00B902227515001287B475B901E5BC648137
:10560B0060031280980515E515242050E975C70332
:10561B0075C68075B90505C6E5C6241C50F512562E
:10562B002F028606E4F5C7F5C674261280B675BD43
:10563B004E125649125646E41256461280B6125571
:10564B00F705C6227F3E7E00E54B12E8667E10E52D
:10565B004C12E8667E20E54D12E8667E30E54E1270
:10566B00E866227F467E00E56C12E8667E10E56BED
:10567B0012E8667E20E56A12E8667E30E57F12E866
:0E568B0066227F2E12189812289C40167F2D42
:1056990012812E1256B012185CE4F5BCF5BD75BE28
:1056A900021255F70205227F0E756F0280057F02EF
:1056B900756F00E4F56EF56D740612998674D8124B
:1056C90099BED2B2129B37056FDFED22E4F56CF576
:1056D9006B756A00E56B700C7F797E32E56C12E8B8
:1056E9000912F19B12B16AE56B2404F56BE4356C80
:1056F900F56C30E7DF2212570502027012F3127FB0
:105709005A7E0590BF7412814912F19B12B23BD2A5
:1057190020C210D214D215C25512188E85BF6C85BD
:10572900BE6BE56B540360051297FA80F5856CBF73
:10573900856BBE75B90575B902129AC6125FA17B50
:1057490017756F7FE4F56EF56D758002C2B275F756
:1057590053856FF7856EF7856DF7A4D2B212B10341
:10576900BB172B756A007539FC75F08412B17F7C03
:1057790007783986F708DCFBD2B2756A1E75F084A2
:1057890012B17F8EF7A48FF7A4D2B2756A0012B155
:105799006A12B0FDE56E2404F56E7C041297FADCFA
:1057A900FBDBA612188E85BEBC85BFBD856BBE8589
:1057B9006CBF75B90575B90279B877C309A73A09F4
:1057C900A73B09A73C09A73D09A73E097700097727
:1057D900180977050977CE09772709773B09775B98
:1057E90009770009A7BD09A7BC129AC6029AEDD28A
:1057F90014D215125806C214C21502023D756F0063
:10580900756E00756D0074031299BE784075A70016
:10581900900700E4F5F7C2B2C2B2E5F7F0A3D8F3F6
:10582900D2B212F31285354B856F4C856E4D856D5D
:105839004E7F0012565175A70090070078107F0916
:10584900E8540370020F0FE0F54BA3E0F54CA3E019
:10585900F54DA3E0F54EA3C083C082125651D08204
:10586900D083EF2407FFD8D812F19B10000910014B
:105879002F10020280F522100214E5352496400209
:10588900800C756D00536EFCE56E24FC800AE56D95
:1058990024C0F56DE56E34FFF56EE56F34FF8026A3
:1058A900100214E53524964002800C756D00536E84
:1058B900FCE56E2404800AE56D2440F56DE56E343F
:1058C90000F56EE4356F540FF56F02580FD214D2FC
:1058D900151258E4C214C21502023D756F00756EA7
:1058E90000756D0012B191784075A700900700E42A
:1058F900F5F7E4E5F7F0A3D8F6D2B212F31285353D
:105909004B856F4C856E4D856D4E7F0012565175D6
:0F591900A70090070078107F09E8540370020F71
:105928000FE0F54BA3E0F54CA3E0F54DA3E0F54EF1
:10593800A3C083C082125651D082D083EF2407FFC0
:10594800D8D812F19B10000910012F10020280F51F
:1059580022100214E53524964002800C756D005320
:105968006EFCE56E24FC800AE56D24C0F56DE56EDD
:1059780034FFF56EE56F34FF8026100214E53524F8
:10598800964002800C756D00536EFCE56E24048011
:105998000AE56D2440F56DE56E3400F56EE4356F6B
:1059A800547FF56F0258ED20740122D24475A70088
:1059B800758307E559C454F02407F582E0F51A24E5
:1059C8004C40E7A3E0F512A3E0F5131207D289389B
:1059D800121861E5BDA2E0923BE51A4006957050A9
:1059E8000224B4F51A203B05D20612DE18E51A1275
:1059F8005B12E5152437F51DE43514F51CE517246D
:105A080037F51FE43516F51E85CC12853813AC1210
:105A1800AB137A04125D9675380124FA401A0538DA
:105A28002402401405382401400E053805382401A5
:105A38004006053805380538C3E51A945A5002243B
:0E5A4800B4F51AC23BC23CC23D751B00A23B26
:105A5600823C406D203B2CE51A75F008A4951BFB93
:105A6600E5F0303D04940180029400FC5008EB24DC
:105A7600A0FBEC3405FC125B19125AC8923B40039A
:105A8600125AEB203C2CE51A75F008A4251BF9E404
:105A9600303D010435F0FAE994A0FBEA9405FC5088
:105AA60004AB01AC02125B19125AC8923C400312B5
:105AB6005AEBE51B2538F51B5094203D04D23D805A
:105AC6008D22E51F2517FEE51E35167016EE24916C
:105AD6004011E51D2515FFE51C35147006EF2491D0
:105AE600400122D3228E027C8A7B3B125DA4ED24E8
:105AF60002FE8F027C8A7B3B125DA4ED2439FF02F5
:105B0600F22D12610880311260FB804675F008A400
:105B1600ACF0FB751900C3EB9468F9EC9401FA40FC
:105B2600080519AC02AB0180ED8C108B11531903DB
:105B3600E51920E0CD1260FB125B6DAF05E5192477
:105B4600FE500312601F8E168F17E51920E0B8125B
:105B56006108125B6DAF05E5191460061460031247
:105B6600601F8E148F1522AC06AB07AA12A913026A
:055B76005E0F125C5AF5
:105B7B00203D4974857F227E0812E8FC7E08301791
:105B8B003CAC1EAB1FEB2418EC34FC402F125D75A4
:105B9B00E51B60077F207E0812E9177F207E10E54A
:105BAB001A12E9177F237E17742E12E8F87F207ED6
:105BBB001BE51B7011E519C2E012E917227F207E4D
:105BCB000E740A02E917E51975F0058475F005A442
:105BDB0002E917125C5A203D5E74857F227E3A12D1
:105BEB00E8FC301753AC1EAB1FEB2418EC34FC4015
:105BFB0046EC7033EB249C402E7E2D125C4C125FD6
:105C0B00BEC0E07F2A7E2EEB12E9177E39D0E0C2B0
:105C1B00E012E9177F347E3712F22D1E12F22D1F80
:105C2B0012F22D0E02F22D7E30125C4C125FBEEB87
:105C3B007F2A7E3112E20A227F2A7E39740A02E918
:105C4B00177F2912F25D0FBF34F90EBE40F322D23B
:105C5B003D30126612186BE5BDF51C75F00AA4F801
:105C6B0024E15002781EE4FCFBFEFFC23D12993981
:105C7B00125CC6203D44D8F8751DCEE51C14600996
:105C8B00751D9C146003751D6AC217EC30E705D2B5
:105C9B001712602F8C018B00E9487003D23D22EE66
:055CAB007008EF251D4B
:105CB0004003D23D22AC06AB077A1C125DA4125FF2
:105CC000488C1E8B1F22203D071248B47003D23D22
:105CD00022056D12B191E4F5F7C2B2C2B2ADF7F58B
:105CE000F7C2B2C2B2E5F7FAD2B230E4E3ED2FFF69
:105CF000E43EFEE56D2408F56D12B191E4F5F7C2BE
:105D0000B2C2B2ADF7D2B2EA30E508EB2DFBEC340B
:0C5D100000FC22C3EB9DFBEC9400FC2285
:08F335000000000000000000D0
:00000001FF
